:020000040000FA
:0400000006EF00F017
:020008001000E6
:10000C00D6ECB6F01269936A94809482949E949C78
:10001C00949894949496949A929092929294929694
:10002C009298929A010E0E6F899089928994899672
:10003C008998899A8B948B968B988B9A8B9C8B9E98
:10004C00A3ECB0F0A3ECB0F0A3ECB0F08B8E8A6A0A
:10005C0048ECAEF00E53D8A45FEF19F00000E0ECC2
:10006C00A6F000008A6AC7ECB8F0100E816E76EC30
:10007C0091F0100E816E34ECBAF0100E816E080EF9
:10008C00816E100E816E080E816E01EC7EF0100EEA
:10009C00816E080E816E0000000000008A46100E72
:1000AC00816E16ECBBF0080E816E83ECB0F0100E76
:1000BC00816E080E816E000000000000100E816E33
:1000CC004CECB0F0000000008A6AC7ECB8F0100EDF
:1000DC00816E76EC91F0100E816E100E816E3FECFD
:1000EC00BAF0100E816E080E816E00000000100E2A
:1000FC00816E080E816E01EC7EF0100E816E080E82
:10010C00816EA1ECB0F08A46100E816E21ECBBF032
:10011C00080E816E18EC91F000008A6AC7ECB8F0FA
:10012C00100E816E76EC91F0100E816E080E816EC1
:10013C00100E816E4CECBAF0100E816E080E816EB2
:10014C000000000000000000100E816E080E816E91
:10015C0001EC7EF0100E816E080E816EBEECB0F0DC
:10016C008A46100E816E2EECBBF0100E816E080EBE
:10017C00816E18EC91F000008A6AC7ECB8F0100E92
:10018C00816E76EC91F0100E816E080E816E00007F
:10019C000000100E816E55ECBAF0100E816E080E38
:1001AC00816EB2ECB0F0100E816E080E816E01EC17
:1001BC007EF0100E816E080E816EC7ECB0F08A4690
:1001CC00100E816E37ECBBF0080E816E100E816E36
:1001DC00080E816E18EC91F000008A6AC7ECB8F03A
:1001EC00100E816E76EC91F0100E816E080E816E01
:1001FC000000000000000000100E816E5AECBAF0F6
:10020C00100E816E080E816EC2ECB0F0100E816E75
:10021C00080E816E6FECB0F000004CECB0F08A462A
:10022C0000008A428DECB0F08A4600008A426FECE6
:10023C00B0F0000000008A6A5BECB0F000008A8627
:10024C006FECB0F0000000008A4600008A428DEC92
:10025C00B0F08A4600008A4245ECB0F06FECB0F08A
:10026C000000100E816E080E816E4CECB0F08A46C8
:10027C00100E816E3CECBBF0080E816E000000008D
:10028C00100E816E080E816E18EC91F000008A6AD7
:10029C00C7ECB8F0100E816E76EC91F0100E816EFA
:1002AC00080E816EB2ECB0F0100E816E67ECBAF0F5
:1002BC00100E816E080E816E45ECB0F0100E816E42
:1002CC00080E816E6FECB0F000004CECB0F08A467A
:1002DC0000008A428DECB0F08A4600008A425BEC4A
:1002EC00B0F08A6A8DECB0F0000000008A865BECFE
:1002FC00B0F08A4600008A428DECB0F08A460000CD
:10030C008A4245ECB0F06FECB0F00000100E816E3C
:10031C00080E816E4CECB0F0000000008A46100E06
:10032C00816E49ECBBF0080E816E000000000000ED
:10033C000000100E816E080E816E18EC91F000001A
:10034C008A6AC7ECB8F0100E816E76EC91F0100E44
:10035C00816E080E816EC2ECB0F0100E816E70ECE6
:10036C00BAF0100E816E080E816E4CECB0F00000ED
:10037C00100E816E080E816E6FECB0F000004CEC2C
:10038C00B0F08A4600008A428DECB0F08A4600003C
:10039C008A424CECB0F0000000008A6A97ECB0F096
:1003AC00000000000000BEECB0F08A864CECB0F00F
:1003BC00000000008A4600008A428DECB0F08A46AC
:1003CC0000008A4245ECB0F06FECB0F00000100E6B
:1003DC00816E080E816E51ECB0F000008A46100E52
:1003EC00816E52ECBBF0080E816EB2ECB0F0100EC8
:1003FC00816E080E816E18EC91F000008A6AC7ECD1
:10040C00B8F0100E816E76EC91F0100E816E080E25
:10041C00816E45ECB0F0100E816E75ECBAF0100EDA
:10042C00816E080E816E51ECB0F0100E816E080ECC
:10043C00816E6FECB0F000004CECB0F08A4600001E
:10044C008A428DECB0F08A4600008A42C2ECB0F0D1
:10045C008A6A56ECB0F08A886FECB0F000000000AD
:10046C008A6A56ECB0F08A86C2ECB0F08A4600007C
:10047C008A428DECB0F08A4600008A4245ECB0F01E
:10048C006FECB0F00000100E816E080E816E56EC11
:10049C00B0F08A46100E816E57ECBBF0080E816EE0
:1004AC00C2ECB0F0100E816E080E816E18EC91F05B
:1004BC0000008A6AC7ECB8F0100E816E76EC91F0F1
:1004CC00100E816E080E816E4CECB0F00000100E18
:1004DC00816E7CECBAF0100E816E080E816E51ECC0
:1004EC00B0F000000000100E816E080E816E6FECF3
:1004FC00B0F000004CECB0F08A4600008A428DEC63
:10050C00B0F08A4600008A420000000000008A6AAF
:10051C0051ECB0F08A8897ECB0F08A6A51ECB0F0EC
:10052C008A860000000000008A4600008A428DEC9A
:10053C00B0F08A4600008A4245ECB0F06FECB0F0A7
:10054C000000100E816E080E816E56ECB0F00000AB
:10055C0000008A46100E816E5EECBBF0080E816EB8
:10056C0045ECB0F0100E816E080E816E18EC91F017
:10057C0000008A6AC7ECB8F0100E816E76EC91F030
:10058C00100E816E080E816E51ECB0F00000100E52
:10059C00816E00000000080E816E56ECB0F0000079
:1005AC000000100E816E080E816E6FECB0F0000032
:1005BC004CECB0F08A4600008A428DECB0F00000A2
:1005CC0000008A6A4CECB0F08A885BECB0F08A428E
:1005DC0056ECB0F0000000008A465BECB0F08A6A82
:1005EC004CECB0F08A868DECB0F0000000008A462E
:1005FC0000008A4245ECB0F06FECB0F00000100E39
:10060C00816E080E816E5BECB0F00000100E816EF6
:10061C0000000000080E816E4CECB0F000000000F1
:10062C00100E816E080E816E18EC91F000008A6A33
:10063C00C7ECB8F0100E816E76EC91F0100E816E56
:10064C00080E816E83ECB0F000000000100E816E7D
:10065C00080E816E6FECB0F000004CECB0F08A46E6
:10066C0000008A4283ECB0F000008A6A45ECB0F0DE
:10067C008A8851ECB0F08A428DECB0F08A4651EC8D
:10068C00B0F08A6A45ECB0F08A8683ECB0F00000DA
:10069C008A4600008A4245ECB0F06FECB0F00000E6
:1006AC00100E816E080E816E83ECB0F0000000001D
:1006BC00100E816E080E816E18EC91F000008A6AA3
:1006CC00C7ECB8F0100E816E76EC91F0100E816EC6
:1006DC00080E816E83ECB0F000000000100E816EED
:1006EC00080E816E6FECB0F000004CECB0F08A4656
:1006FC0000008A427EECB0F000008A6AC7ECB0F0D1
:10070C008A884CECB0F000008A4297ECB0F0000004
:10071C00000000000000000000008A464CECB0F025
:10072C0000008A6AC7ECB0F08A867EECB0F000005C
:10073C008A4600008A4245ECB0F06FECB0F0000045
:10074C00100E816E080E816E83ECB0F0000000007C
:10075C00100E816E080E816E83ECB0F0000000006C
:10076C00100E816E080E816E000000000000100E4D
:10077C00816E4CECB0F0000000008A6AC7ECB8F057
:10078C0000008A6A000085EC91F0100E816E080E54
:10079C00816E6FECB0F000004CECB0F08A460000BB
:1007AC008A4279ECB0F000008A6AC2ECB0F08A8818
:1007BC0045ECB0F08A4297ECB0F00000000000006D
:1007CC0051ECB0F000008A4645ECB0F08A6AC2ECFD
:1007DC00B0F08A8679ECB0F000008A4600008A42BC
:1007EC0045ECB0F06FECB0F00000100E816E080E0E
:1007FC00816E27EC91F0000000008A6A4CECB0F09E
:10080C00000000008A6AC7ECB8F000008A6A000099
:10081C0085EC91F0100E816E080E816E6FECB0F0CD
:10082C0000004CECB0F08A4600008A426FECB0F04D
:10083C0000008A6AC2ECB0F08A88C7ECB0F08A4239
:10084C0097ECB0F000000000000065ECB0F08A46B8
:10085C00C7ECB0F08A6AC2ECB0F08A866FECB0F0EC
:10086C0000008A4600008A4245ECB0F06FECB0F014
:10087C000000100E816E080E816E27EC91F00000C6
:10088C0000008A6A4CECB0F0000000008A6AC7ECE9
:10089C00B8F000008A6A000085EC91F0100E816EB1
:1008AC00080E816E6FECB0F000004CECB0F08A4694
:1008BC0000008A426AECB0F000008A6AC2ECB0F028
:1008CC008A88C2ECB0F08A4297ECB0F000000000CD
:1008DC0000006FECB0F0000000008A46C2ECB0F0F3
:1008EC008A6AC2ECB0F08A866AECB0F000008A46E4
:1008FC0000008A4245ECB0F06FECB0F00000100E36
:10090C00816E080E816E27EC91F0000000008A6A5F
:10091C004CECB0F0000000008A6AC7ECB8F00000A4
:10092C008A6A000085EC91F0100E816E080E816EC3
:10093C006FECB0F000004CECB0F08A4600008A423C
:10094C0065ECB0F0000000008A6ABEECB0F08A885A
:10095C00C2ECB0F08A4297ECB0F00000000000004E
:10096C007EECB0F0000000008A46C2ECB0F08A6A5F
:10097C00BEECB0F08A8665ECB0F0000000008A4650
:10098C0000008A4245ECB0F06FECB0F00000100EA5
:10099C00816E080E816E27EC91F0000000008A6ACF
:1009AC004CECB0F0000000008A6AC7ECB8F0000014
:1009BC008A6A000085EC91F0100E816E080E816E33
:1009CC006FECB0F000004CECB0F08A4600008A42AC
:1009DC0065ECB0F08A6ABEECB0F08A88BEECB0F080
:1009EC008A4297ECB0F00000000000008DECB0F0F3
:1009FC00000000008A46BEECB0F08A6ABEECB0F093
:100A0C008A8665ECB0F08A4600008A4245ECB0F06C
:100A1C006FECB0F00000100E816E080E816E27ECAA
:100A2C0091F0000000008A6A4CECB0F0000000006D
:100A3C008A6AC7ECB8F000008A6A000085EC91F075
:100A4C00100E816E080E816E6FECB0F000004CEC55
:100A5C00B0F08A4600008A425BECB0F000008A6A73
:100A6C0000000000000000008A6A00008A88000074
:100A7C0079ECB0F0000000008A426AECB0F00000A3
:100A8C00000051ECB0F00000100E816E79ECB0F06B
:100A9C00000000008A6A00008A6A00000000000062
:100AAC0000008A865BECB0F000008A4600008A42A7
:100ABC0045ECB0F06FECB0F00000100E816E080E3B
:100ACC00816E27EC91F0000000008A6A4CECB0F0CB
:100ADC00000000008A6AC7ECB8F000008A6A4CEC8F
:100AEC00B0F000000000100E816ECDECB0F00000F4
:100AFC00000065ECB0F051ECB0F0000051ECB0F03F
:100B0C00000000008A4200008A6AB2ECB0F0100EBD
:100B1C00816E93EC7CF08A426AECB0F0000000002D
:100B2C0051ECB0F00000100E816EF6EC7CF08A6A8D
:100B3C00B2ECB0F08A8600008A4651ECB0F00000AE
:100B4C00000051ECB0F0CDECB0F00000000065EC12
:100B5C00B0F00000000000008A6A4CECB0F000001D
:100B6C0000008A6AC7ECB8F000008A6A00005FECEB
:100B7C0091F0100E816E080E816E6FECB0F00000DB
:100B8C004CECB0F08A4600008A4256ECB0F08A6A0F
:100B9C00B2ECB0F08A880000100E816E93EC7CF001
:100BAC008A426AECB0F00000000051ECB0F000009A
:100BBC00100E816EF6EC7CF08A8800008A6AB2EC2A
:100BCC00B0F08A8656ECB0F08A4600008A4245ECBA
:100BDC00B0F06FECB0F00000100E816E100E816E54
:100BEC0009EC91F0000000008A6A4CECB0F00000B7
:100BFC0000008A6AC7ECB8F000008A6A00005FEC5B
:100C0C0091F0100E816E080E816E6FECB0F000004A
:100C1C004CECB0F08A4600008A4251ECB0F0000077
:100C2C008A6AB2ECB0F08A88000000000000100E56
:100C3C00816E93EC7CF08A426AECB0F0000000000C
:100C4C0051ECB0F00000100E816EF6EC7CF08A884E
:100C5C000000000000008A6AB2ECB0F08A8651EC09
:100C6C00B0F000008A4600008A4245ECB0F06FEC10
:100C7C00B0F00000100E816E100E816E09EC91F038
:100C8C00000000008A6A4CECB0F0000000008A6A98
:100C9C00C7ECB8F000008A6A00005FEC91F0100E0F
:100CAC00816E080E816E6FECB0F000004CECB0F071
:100CBC008A4600008A424CECB0F0000000008A6AC0
:100CCC00B2ECB0F08A88A1ECB0F0100E816E93EC0F
:100CDC007CF08A426AECB0F00000000051ECB0F0FD
:100CEC000000100E816EF6EC7CF08A88A1ECB0F05E
:100CFC008A6AB2ECB0F08A864CECB0F000000000CE
:100D0C008A4600008A4245ECB0F06FECB0F000006F
:100D1C00100E816E100E816E09EC91F00000000037
:100D2C008A6A4CECB0F0000000008A6AC7ECB8F09C
:100D3C0000008A6A00005FEC91F0100E816E080EC4
:100D4C00816E6FECB0F000004CECB0F08A46000005
:100D5C008A424CECB0F000008A6AA1ECB0F08A88B0
:100D6C00B2ECB0F08A42100E816E93EC7CF08A42A9
:100D7C006AECB0F00000000051ECB0F00000100E76
:100D8C00816EF6EC7CF08A428A46B2ECB0F08A6A4C
:100D9C00A1ECB0F08A864CECB0F000008A46000062
:100DAC008A4245ECB0F06FECB0F00000100E816E92
:100DBC00100E816E09EC91F0000000008A6A4CEC78
:100DCC00B0F0000000008A6AC7ECB8F000008A6A34
:100DDC0000005FEC91F0100E816E080E816E6FECCE
:100DEC00B0F000004CECB0F08A4600008A4245ECB2
:100DFC00B0F08A6AB2ECB0F08A88A1ECB0F08A420A
:100E0C0000000000100E816E93EC7CF08A426AECBC
:100E1C00B0F00000000051ECB0F00000100E816E3C
:100E2C00F6EC7CF08A42000000008A46A1ECB0F09F
:100E3C008A6AB2ECB0F08A8645ECB0F08A460000C3
:100E4C008A4245ECB0F06FECB0F00000100E816EF1
:100E5C00100E816E09EC91F0000000008A6A4CECD7
:100E6C00B0F0000000008A6AC7ECB8F0100E816E7A
:100E7C0000005FEC91F0100E816E080E816E6FEC2D
:100E8C00B0F000004CECB0F08A4600008A42C7EC8F
:100E9C00B0F08A6AA1ECB0F08A88A1ECB0F08A427A
:100EAC000000000000000000100E816E93EC7CF03E
:100EBC008A42BEECB0F08A466AECB0F000008A427E
:100ECC00BEECB0F0100E816EF6EC7CF08A420000A5
:100EDC000000000000008A46A1ECB0F08A6AA1EC88
:100EEC00B0F08A86C7ECB0F08A4600008A4245EC26
:100EFC00B0F06FECB0F00000100E816E100E816E31
:100F0C0009EC91F00000100E816E4CECB0F000007A
:100F1C0000008A6AC7ECB8F0100E816E00005FEC1E
:100F2C0091F0100E816E080E816E6FECB0F0000027
:100F3C004CECB0F08A4600008A42BEECB0F08A6AF3
:100F4C00B2ECB0F08A88A1ECB0F08A42A1ECB0F01F
:100F5C00100E816E93EC7CF08A42BEECB0F08A46A7
:100F6C006AECB0F000008A42BEECB0F0100E816E5C
:100F7C00F6EC7CF08A42A1ECB0F08A46A1ECB0F021
:100F8C008A6AB2ECB0F08A86BEECB0F08A460000F9
:100F9C008A4245ECB0F06FECB0F00000100E816EA0
:100FAC00100E816E09EC91F00000100E816E4CEC6D
:100FBC00B0F0000000008A6AC7ECB8F0100E816E29
:100FCC0000005FEC91F0100E816E080E816E6FECDC
:100FDC00B0F000004CECB0F08A4600008A42B2EC53
:100FEC00B0F08A6AA1ECB0F08A88A1ECB0F08A4229
:100FFC00BEECB0F0100E816E93EC7CF08A42BEEC2D
:10100C00B0F08A466AECB0F000008A42BEECB0F058
:10101C00100E816EF6EC7CF08A42BEECB0F08A4683
:10102C00A1ECB0F08A6AA1ECB0F08A86B2ECB0F018
:10103C008A4600008A4245ECB0F06FECB0F000003C
:10104C00100E816E100E816E09EC91F00000100EE6
:10105C00816E4CECB0F0000000008A6AC7ECB8F06E
:10106C00100E816E00005FEC91F0100E816E080E78
:10107C00816E6FECB0F000004CECB0F08A460000D2
:10108C008A42A1ECB0F08A6AA1ECB0F08A88A1EC9B
:10109C00B0F08A42C2ECB0F0100E816E93EC7CF092
:1010AC008A42BEECB0F08A466AECB0F000008A428C
:1010BC00BEECB0F0100E816EF6EC7CF08A42C2EC05
:1010CC00B0F08A46A1ECB0F08A6AA1ECB0F08A8646
:1010DC00A1ECB0F08A4600008A4245ECB0F06FEC0F
:1010EC00B0F00000100E816E100E816E09EC91F0C4
:1010FC000000100E816E4CECB0F0000000008A6A0B
:10110C00C7ECB8F0100E816E00005FEC91F0100E81
:10111C00816E080E816E6FECB0F000004CECB0F0FC
:10112C008A4600008A4200000000000000008A6A23
:10113C00A1ECB0F08A88A1ECB0F08A42C7ECB0F018
:10114C00100E816E93EC7CF08A42BEECB0F08A46B5
:10115C006AECB0F000008A42BEECB0F0100E816E6A
:10116C00F6EC7CF08A42C7ECB0F08A46A1ECB0F009
:10117C008A6AA1ECB0F08A86000000000000000032
:10118C008A4600008A4245ECB0F06FECB0F00000EB
:10119C00100E816E100E816E09EC91F00000100E95
:1011AC00816E4CECB0F0000000008A6AC7ECB8F01D
:1011BC00100E816E00005FEC91F0100E816E080E27
:1011CC00816E6FECB0F000004CECB0F08A46000081
:1011DC008A420000000000008A6A00000000000043
:1011EC0000008A88A1ECB0F08A424CECB0F0100EF2
:1011FC00816E93EC7CF08A42BEECB0F08A466AECCD
:10120C00B0F000008A42BEECB0F0100E816EF6EC2D
:10121C007CF08A424CECB0F08A46A1ECB0F08A6AC1
:10122C0000000000000000008A86000000000000A2
:10123C008A4600008A4245ECB0F06FECB0F000003A
:10124C00100E816E100E816E09EC91F00000100EE4
:10125C00816E4CECB0F0000000008A6AC7ECB8F06C
:10126C00100E816E9CEC91F0100E816E080E816E4A
:10127C006FECB0F000004CECB0F08A4600008A42F3
:10128C00000000008A6A00000000000000008A884C
:10129C00A1ECB0F08A424CECB0F00000100E816E64
:1012AC0093EC7CF08A42BEECB0F08A466AECB0F06B
:1012BC0000008A42BEECB0F0100E816EF6EC7CF0B1
:1012CC008A424CECB0F000008A46A1ECB0F08A6A7D
:1012DC0000000000000000008A86000000008A4622
:1012EC0000008A4245ECB0F06FECB0F00000100E3C
:1012FC00816E100E816E36EC91F0100E816E4CECFE
:10130C00B0F0000000008A6AC7ECB8F0100E816ED5
:10131C009CEC91F0100E816E080E816E6FECB0F0AB
:10132C00000051ECB0F000008A6A000000000000E0
:10133C0000008A88A1ECB0F08A424CECB0F00000BE
:10134C000000100E816E93EC7CF08A42BEECB0F083
:10135C008A466AECB0F000008A42BEECB0F0100E87
:10136C00816EF6EC7CF08A424CECB0F00000000090
:10137C008A46A1ECB0F08A6A000000000000000070
:10138C008A8651ECB0F06FECB0F00000100E816E5C
:10139C00100E816E36EC91F0100E816E4CECB0F0AC
:1013AC00000000008A6AC7ECB8F0100E816E9CEC4D
:1013BC0091F0100E816E080E816E6FECB0F0000093
:1013CC0051ECB0F08A6A00000000000000008A882E
:1013DC00A1ECB0F08A4251ECB0F0100E816E93EC9F
:1013EC007CF08A42BEECB0F08A466AECB0F00000A9
:1013FC008A42BEECB0F0100E816EF6EC7CF08A42A4
:10140C0051ECB0F08A46A1ECB0F08A6A0000000002
:10141C00000000008A864CECB0F0000000006FEC7D
:10142C00B0F00000100E816E100E816E36EC91F053
:10143C00100E816E4CECB0F0000000008A6AC7EC14
:10144C00B8F0100E816E9CEC91F0100E816E080EAF
:10145C00816E6FECB0F000004CECB0F000000000BE
:10146C008A6A00000000000000008A88A1ECB0F03D
:10147C008A4251ECB0F00000100E816E93EC7CF0BF
:10148C008A42BEECB0F08A466AECB0F000008A42A8
:10149C00BEECB0F0100E816EF6EC7CF08A4251EC92
:1014AC00B0F000008A46A1ECB0F08A6A000000009F
:1014BC00000000008A864CECB0F000006FECB0F03D
:1014CC000000100E816E100E816E36EC91F0100E35
:1014DC00816E4CECB0F0000000008A6AC7ECB8F0EA
:1014EC00100E816E9CEC91F0100E816E080E816EC8
:1014FC006FECB0F000004CECB0F000008A6A000019
:10150C000000000000008A88A1ECB0F08A4251EC87
:10151C00B0F000000000100E816E93EC7CF08A425B
:10152C00BEECB0F08A466AECB0F000008A42BEEC29
:10153C00B0F0100E816EF6EC7CF08A4251ECB0F0FB
:10154C00000000008A46A1ECB0F08A6A000000009E
:10155C00000000008A864CECB0F06FECB0F000009C
:10156C00100E816E100E816E36EC91F0100E816EA5
:10157C004CECB0F0000000008A6AC7ECB8F0100E1A
:10158C00816E9CEC91F0100E816E080E816E6FECEA
:10159C00B0F000004CECB0F08A6A000000000000D3
:1015AC0000008A88A1ECB0F08A4256ECB0F0100E24
:1015BC00816E7EECB0F000008A42BEECB0F08A4640
:1015CC006AECB0F000008A42BEECB0F0100E816EF6
:1015DC007EECB0F000008A4256ECB0F08A46A1ECEA
:1015EC00B0F08A6A00000000000000008A8645EC1A
:1015FC00B0F06FECB0F00000100E816E100E816E2A
:10160C0036EC91F0100E816E4CECB0F00000000046
:10161C008A6AC7ECB8F000008A6A9CEC91F0100E54
:10162C00816E080E816E29EC80F0100E816E100E0A
:10163C00816E36EC91F000008A6A4CECB0F0000040
:10164C0000008A6AC7ECB8F000008A6A9CEC91F042
:10165C00100E816E080E816E0DEC81F0100E816EF5
:10166C00100E816E36EC91F000008A6A4CECB0F0F2
:10167C00000000008A6AC7ECB8F000008A6A9CEC93
:10168C0091F0100E816E080E816EC5EC81F0100E7B
:10169C00816E100E816E36EC91F000008A6A4CEC73
:1016AC00B0F0000000008A6AC7ECB8F000008A6A4B
:1016BC009CEC91F0100E816E080E816EB4EC82F0F1
:1016CC00100E816E100E816E36EC91F000008A6A5D
:1016DC004CECB0F0000000008A6AC7ECB8F00000D7
:1016EC008A6A9CEC91F0100E816E080E816EADEC46
:1016FC0083F0100E816E100E816E36EC91F00000AE
:10170C008A6A4CECB0F0000000008A6AC7ECB8F0B2
:10171C0000008A6A9CEC91F0100E816E080E816EAE
:10172C002AEC84F0100E816E100E816E36EC91F066
:10173C0000008A6A4CECB0F0000000008A6AC7EC2A
:10174C00B8F000008A6A4CECB0F000000000100EFB
:10175C00816E97ECB0F000008A6A56ECB0F0000095
:10176C00100E816E00008A6A56ECB0F00000100E6C
:10177C00816E100E816EE4EC84F0100E816E100EF2
:10178C00816E56ECB0F0000000008A6A100E816E7B
:10179C0056ECB0F00000100E816E97ECB0F000002B
:1017AC00000000008A6A4CECB0F0000000008A6A6D
:1017BC00C7ECB8F000008A6A9CEC91F0100E816EB8
:1017CC00080E816ED3EC85F0100E816E100E816EBA
:1017DC0036EC91F000008A6A4CECB0F0000000008E
:1017EC008A6AC7ECB8F000008A6A9CEC91F0100E83
:1017FC00816E080E816E4EEC86F0100E816E100E0E
:10180C00816E36EC91F000008A6A4CECB0F000006E
:10181C0000008A6AC7ECB8F000008A6A9CEC91F070
:10182C00100E816E080E816EA2EC7EF0100E816E91
:10183C00100E816E36EC91F000008A6A4CECB0F020
:10184C00000000008A6AC7ECB8F000008A6A9CECC1
:10185C0091F0100E816E080E816E46EC7FF0100E2A
:10186C00816E100E816E36EC91F000008A6A4CECA1
:10187C00B0F0000000008A6AC7ECB8F000008A6A79
:10188C009CEC91F0100E816E080E816E46EC7FF090
:10189C00100E816E100E816E36EC91F000008A6A8B
:1018AC004CECB0F0000000008A6AC7ECB8F0100EE7
:1018BC00816E9CEC91F0100E816E080E816E9AEC8C
:1018CC0088F0100E816E100E816E36EC91F0100EB9
:1018DC00816E4CECB0F0000000008A6AC7ECB8F0E6
:1018EC00100E816E9CEC91F0100E816E080E816EC4
:1018FC0048EC89F0100E816E100E816E36EC91F072
:10190C00100E816E4CECB0F0000000008A6AC7EC3F
:10191C00B8F0100E816E9CEC91F0100E816E080EDA
:10192C00816E61EC8BF0100E816E100E816E36ECB8
:10193C0091F0100E816E4CECB0F0000000008A6A41
:10194C00C7ECB8F0100E816E9CEC91F0100E816E0D
:10195C00080E816E61EC8BF0100E816E100E816E94
:10196C0036EC91F0100E816E4CECB0F000000000E3
:10197C008A6AC7ECB8F0100E816E9CEC91F0100ED8
:10198C00816E080E816E61EC8BF0100E816E100E64
:10199C00816E36EC91F0100E816E4CECB0F00000C4
:1019AC0000008A6AC7ECB8F0100E816E9CEC91F0C6
:1019BC00100E816E080E816E30EC8AF0100E816E66
:1019CC00100E816E36EC91F0100E816E4CECB0F076
:1019DC00000000008A6AC7ECB8F0100E816E9CEC17
:1019EC0091F0100E816E080E816EA4EC8AF0100E30
:1019FC00816E100E816E36EC91F0100E816E4CECF7
:101A0C00B0F0000000008A6AC7ECB8F0100E816ECE
:101A1C009CEC91F0100E816E080E816EA4EC8AF095
:101A2C00100E816E100E816E36EC91F0100E816EE0
:101A3C004CECB0F0000000008A6AC7ECB8F0100E55
:101A4C00816E9CEC91F0100E816E080E816EA4ECF0
:101A5C008AF0100E816E100E816E36EC91F0100E25
:101A6C00816E4CECB0F0000000008A6AC7ECB8F054
:101A7C00100E816E9CEC91F0100E816E080E816E32
:101A8C00A4EC8AF0100E816E100E816E36EC91F083
:101A9C00100E816E4CECB0F0000000008A6AC7ECAE
:101AAC00B8F0100E816E9CEC91F0100E816E080E49
:101ABC00816EF6EC86F0100E816E100E816E36EC97
:101ACC0091F0100E816E4CECB0F0000000008A6AB0
:101ADC00C7ECB8F0100E816E9CEC91F0100E816E7C
:101AEC00080E816E74EC87F0100E816E100E816EF4
:101AFC0036EC91F0100E816E4CECB0F00000000052
:101B0C008A6AC7ECB8F000008A6A9CEC91F0100E5F
:101B1C00816E080E816E04EC8DF0100E816E100E2D
:101B2C00816E36EC91F000008A6A4CECB0F000004B
:101B3C0000008A6AC7ECB8F000008A6A9CEC91F04D
:101B4C00100E816E080E816E04EC8DF0100E816EFD
:101B5C00100E816E36EC91F000008A6A4CECB0F0FD
:101B6C00000000008A6AC7ECB8F000008A6A9CEC9E
:101B7C0091F0100E816E080E816EB2EC8DF0100E8D
:101B8C00816E100E816E36EC91F000008A6A4CEC7E
:101B9C00B0F0000000008A6AC7ECB8F000008A6A56
:101BAC009CEC91F0100E816E080E816E27EC8EF07D
:101BBC00100E816E100E816E36EC91F000008A6A68
:101BCC004CECB0F0000000008A6AC7ECB8F00000E2
:101BDC008A6A9CEC91F0100E816E080E816E96EC68
:101BEC008EF0100E816E100E816E36EC91F00000AE
:101BFC008A6A4CECB0F0000000008A6AC7ECB8F0BE
:101C0C0000008A6A9CEC91F0100E816E080E816EB9
:101C1C0011EC8FF0100E816E100E816E36EC91F07F
:101C2C0000008A6A4CECB0F0000000008A6AC7EC35
:101C3C00B8F000008A6A4CECB0F000000000100E06
:101C4C00816E97ECB0F000008A6A56ECB0F00000A0
:101C5C00100E816E00008A6A56ECB0F00000100E77
:101C6C00816E100E816E8AEC8FF0100E816E100E4C
:101C7C00816E56ECB0F0000000008A6A100E816E86
:101C8C0056ECB0F00000100E816E97ECB0F0000036
:101C9C00000000008A6A4CECB0F0000000008A6A78
:101CAC00C7ECB8F000008A6A9CEC91F0100E816EC3
:101CBC00080E816E12EC90F0100E816E100E816E7B
:101CCC0036EC91F000008A6A4CECB0F00000000099
:101CDC008A6AC7ECB8F000008A6A9CEC91F0100E8E
:101CEC00816E080E816E8FEC90F0100E816E100ECE
:101CFC00816E36EC91F000008A6A4CECB0F000007A
:101D0C0000008A6AC7ECB8F000008A6A9CEC91F07B
:101D1C00100E816E080E816EA0EC8BF0100E816E91
:101D2C00100E816E36EC91F000008A6A4CECB0F02B
:101D3C00000000008A6AC7ECB8F000008A6A9CECCC
:101D4C0091F0100E816E080E816E52EC8CF0100E1C
:101D5C00816E100E816E36EC91F000008A6A4CECAC
:101D6C00B0F0000000008A6AC7ECB8F000008A6A84
:101D7C009CEC91F0100E816E080E816E90EC8CF044
:101D8C00100E816E100E816E36EC91F000008A6A96
:101D9C004CECB0F0000000008A6AC7ECB8F0100EF2
:101DAC00816E9CEC91F0100E816E080E816E6FECC2
:101DBC00B0F000004CECB0F08A6A000000000000AB
:101DCC0000008A8800000000000000008A4256ECE7
:101DDC00B0F00000100E816EF6EC7CF08A42BEEC86
:101DEC00B0F08A6A6AECB0F000008A86BEECB0F003
:101DFC00100E816E93EC7CF08A4256ECB0F0000031
:101E0C008A4600000000000000008A6A0000000002
:101E1C00000000008A8645ECB0F06FECB0F00000DA
:101E2C00100E816E100E816E36EC91F0100E816EDC
:101E3C004CECB0F0000000008A6AC7ECB8F0100E51
:101E4C00816E9CEC91F0100E816E080E816E6FEC21
:101E5C00B0F000004CECB0F08A6AA1ECB0F08A88CB
:101E6C0000000000000000008A4256ECB0F0100E9A
:101E7C00816EF6EC7CF08A42BEECB0F08A6A6AECB9
:101E8C00B0F000008A86BEECB0F0100E816E93ECC0
:101E9C007CF08A4256ECB0F08A460000000000004C
:101EAC0000008A6AA1ECB0F08A8645ECB0F06FECC9
:101EBC00B0F00000100E816E100E816E36EC91F0B9
:101ECC00100E816E4CECB0F0000000008A6AC7EC7A
:101EDC00B8F0100E816E9CEC91F0100E816E080E15
:101EEC00816E6FECB0F000004CECB0F000008A6A30
:101EFC00A1ECB0F08A8800000000000000008A42CB
:101F0C0051ECB0F000000000100E816EF6EC7CF08D
:101F1C008A42BEECB0F08A6A6AECB0F000008A86A5
:101F2C00BEECB0F0100E816E93EC7CF08A4251EC5A
:101F3C00B0F0000000008A46000000000000000025
:101F4C008A6AA1ECB0F08A864CECB0F06FECB0F081
:101F5C000000100E816E100E816E36EC91F0100E9A
:101F6C00816E4CECB0F0000000008A6AC7ECB8F04F
:101F7C00100E816E9CEC91F0100E816E080E816E2D
:101F8C006FECB0F000004CECB0F0000000008A6A7E
:101F9C00A1ECB0F08A8800000000000000008A422A
:101FAC0051ECB0F00000100E816EF6EC7CF08A4221
:101FBC00BEECB0F08A6A6AECB0F000008A86BEEC27
:101FCC00B0F0100E816E93EC7CF08A4251ECB0F0C4
:101FDC0000008A4600000000000000008A6AA1ECA4
:101FEC00B0F08A864CECB0F000006FECB0F0000062
:101FFC00100E816E100E816E36EC91F0100E816E0B
:10200C004CECB0F0000000008A6AC7ECB8F0100E7F
:10201C00816E9CEC91F0100E816E080E816E6FEC4F
:10202C00B0F0000051ECB0F08A6AA1ECB0F08A88F4
:10203C0000000000000000008A4251ECB0F0100ECD
:10204C00816EF6EC7CF08A42BEECB0F08A6A6AECE7
:10205C00B0F000008A86BEECB0F0100E816E93ECEE
:10206C007CF08A4251ECB0F08A460000000000007F
:10207C0000008A6AA1ECB0F08A864CECB0F000004B
:10208C0000006FECB0F00000100E816E100E816E2F
:10209C0036EC91F0100E816E4CECB0F000000000AC
:1020AC008A6AC7ECB8F0100E816E9CEC91F0100EA1
:1020BC00816E080E816E6FECB0F0000051ECB0F048
:1020CC0000008A6AA1ECB0F08A88000000000000D1
:1020DC0000008A424CECB0F000000000100E816E43
:1020EC00F6EC7CF08A42BEECB0F08A6A6AECB0F096
:1020FC0000008A86BEECB0F0100E816E93EC7CF082
:10210C008A424CECB0F0000000008A46000000004F
:10211C00000000008A6AA1ECB0F08A8651ECB0F0A5
:10212C006FECB0F00000100E816E100E816E36EC6C
:10213C0091F0100E816E4CECB0F0000000008A6A39
:10214C00C7ECB8F0100E816EB9EC91F0100E816EE8
:10215C00080E816E6FECB0F000004CECB0F08A46CB
:10216C008A420000000000008A6AA1ECB0F08A8864
:10217C00A1ECB0F08A424CECB0F0100E816EF6EC93
:10218C007CF08A42BEECB0F08A6A6AECB0F00000D7
:10219C008A86BEECB0F0100E816E93EC7CF08A4215
:1021AC004CECB0F08A46A1ECB0F08A6AA1ECB0F02D
:1021BC008A860000000000008A468A4245ECB0F096
:1021CC006FECB0F00000100E816E100E816E4FECB3
:1021DC0091F0100E816E4CECB0F0000000008A6A99
:1021EC00C7ECB8F0100E816EB9EC91F0100E816E48
:1021FC00080E816E6FECB0F000004CECB0F08A462B
:10220C0000008A420000000000008A6AA1ECB0F0D5
:10221C008A88A1ECB0F08A4245ECB0F0100E816EC9
:10222C00F6EC7CF08A42BEECB0F08A6A6AECB0F054
:10223C0000008A86BEECB0F0100E816E93EC7CF040
:10224C008A4245ECB0F08A46A1ECB0F08A6AA1EC67
:10225C00B0F08A860000000000008A4600008A4226
:10226C0045ECB0F06FECB0F00000100E816E100E6B
:10227C00816E4FEC91F0100E816E4CECB0F00000C2
:10228C0000008A6AC7ECB8F0100E816EB9EC91F0C0
:10229C00100E816E080E816E6FECB0F000004CECED
:1022AC00B0F08A4600008A420000000000000000E6
:1022BC008A6AA1ECB0F08A88A1ECB0F08A42C7EC33
:1022CC00B0F0100E816EF6EC7CF08A42BEECB0F0F1
:1022DC008A6A6AECB0F000008A86BEECB0F0100E90
:1022EC00816E93EC7CF08A42C7ECB0F08A46A1EC8C
:1022FC00B0F08A6AA1ECB0F08A8600000000000001
:10230C0000008A4600008A4245ECB0F06FECB0F059
:10231C000000100E816E100E816E4FEC91F0100EBD
:10232C00816E4CECB0F0000000008A6AC7ECB8F08B
:10233C00100E816EB9EC91F0100E816E080E816E4C
:10234C006FECB0F000004CECB0F08A4600008A4212
:10235C00B2ECB0F08A6AA1ECB0F08A88A1ECB0F0D3
:10236C008A42BEECB0F0100E816EF6EC7CF08A4224
:10237C00BEECB0F08A6A6AECB0F000008A86BEEC63
:10238C00B0F0100E816E93EC7CF08A42BEECB0F093
:10239C008A46A1ECB0F08A6AA1ECB0F08A86B2EC65
:1023AC00B0F08A4600008A4245ECB0F06FECB0F019
:1023BC000000100E816E100E816E4FEC91F0100E1D
:1023CC00816E4CECB0F0000000008A6AC7ECB8F0EB
:1023DC00100E816EB9EC91F0100E816E080E816EAC
:1023EC006FECB0F000004CECB0F08A4600008A4272
:1023FC00BEECB0F08A6AA1ECB0F08A88A1ECB0F027
:10240C008A42B2ECB0F0100E816EF6EC7CF08A428F
:10241C00BEECB0F08A6A6AECB0F000008A86BEECC2
:10242C00B0F0100E816E93EC7CF08A42B2ECB0F0FE
:10243C008A46A1ECB0F08A6AA1ECB0F08A86BEECB8
:10244C00B0F08A4600008A4245ECB0F06FECB0F078
:10245C000000100E816E100E816E4FEC91F0100E7C
:10246C00816E4CECB0F0000000008A6AC7ECB8F04A
:10247C00100E816EB9EC91F0100E816E080E816E0B
:10248C006FECB0F000004CECB0F08A4600008A42D1
:10249C00C2ECB0F08A6AA1ECB0F08A88B2ECB0F071
:1024AC008A420000000000000000100E816EF6EC65
:1024BC007CF08A42BEECB0F08A6A6AECB0F00000A4
:1024CC008A86BEECB0F0100E816E93EC7CF08A42E2
:1024DC0000000000000000008A46B2ECB0F08A6AEE
:1024EC00A1ECB0F08A86C2ECB0F08A4600008A42B9
:1024FC0045ECB0F06FECB0F00000100E816E100ED9
:10250C00816E4FEC91F0100E816E4CECB0F000002F
:10251C0000008A6AC7ECB8F000008A6A00005FEC21
:10252C0091F0100E816E080E816E6FECB0F0000011
:10253C004CECB0F08A4600008A4245ECB0F08A6A56
:10254C00A1ECB0F08A88A1ECB0F08A420000000047
:10255C000000100E816EF6EC7CF08A428DECB0F02F
:10256C0000000000100E816E93EC7CF08A4200009B
:10257C00000000008A46A1ECB0F08A6AA1ECB0F031
:10258C008A8645ECB0F08A4600008A4245ECB0F0F1
:10259C006FECB0F00000100E816E100E816E09EC25
:1025AC0091F0000000008A6A4CECB0F000000000D2
:1025BC008A6AC7ECB8F000008A6A00005FEC91F000
:1025CC00100E816E080E816E6FECB0F000004CECBA
:1025DC00B0F08A4600008A424CECB0F08A6AB2EC49
:1025EC00B0F08A88A1ECB0F08A420000100E816E27
:1025FC00F6EC7CF08A428DECB0F000000000100E7E
:10260C00816E93EC7CF08A4200008A46A1ECB0F01B
:10261C008A6AB2ECB0F08A864CECB0F08A460000C4
:10262C008A4245ECB0F06FECB0F00000100E816EF9
:10263C00100E816E09EC91F0000000008A6A4CECDF
:10264C00B0F0000000008A6AC7ECB8F000008A6A9B
:10265C0000005FEC91F0100E816E080E816E6FEC35
:10266C00B0F000004CECB0F08A4600008A424CEC12
:10267C00B0F0000000008A6AA1ECB0F08A88B2ECDD
:10268C00B0F0100E816EF6EC7CF08A428DECB0F05E
:10269C0000000000100E816E93EC7CF08A88B2EC86
:1026AC00B0F08A6AA1ECB0F08A864CECB0F0000075
:1026BC0000008A4600008A4245ECB0F06FECB0F0A6
:1026CC000000100E816E100E816E09EC91F000006E
:1026DC0000008A6A4CECB0F0000000008A6AC7EC7B
:1026EC00B8F000008A6A00005FEC91F0100E816E69
:1026FC00080E816E6FECB0F000004CECB0F08A4626
:10270C0000008A4251ECB0F08A6AB2ECB0F08A88D0
:10271C000000000000000000100E816EF6EC7CF052
:10272C008A428DECB0F000000000100E816E93EC2C
:10273C007CF08A8800000000000000008A6AB2EC7D
:10274C00B0F08A8651ECB0F08A4600008A4245EC23
:10275C00B0F06FECB0F00000100E816E100E816EB8
:10276C0009EC91F0000000008A6A4CECB0F000001B
:10277C0000008A6AC7ECB8F000008A6A00005FECBF
:10278C0091F0100E816E080E816E6FECB0F00000AF
:10279C004CECB0F08A4600008A4251ECB0F00000DC
:1027AC0000008A6AB2ECB0F08A8800000000100EBB
:1027BC00816EF6EC7CF08A428DECB0F000000000EB
:1027CC00100E816E93EC7CF08A88000000008A6AFF
:1027DC00B2ECB0F08A8651ECB0F0000000008A46F2
:1027EC0000008A4245ECB0F06FECB0F00000100E27
:1027FC00816E100E816E09EC91F0000000008A6A67
:10280C004CECB0F0000000008A6AC7ECB8F0000095
:10281C008A6A00005FEC91F0100E816E080E816EDA
:10282C006FECB0F000004CECB0F08A4600008A422D
:10283C0056ECB0F000008A6AB2ECB0F08A88100E48
:10284C00816E7EECB0F000008A428DECB0F000009E
:10285C000000100E816E7EECB0F000008A888A6A4F
:10286C00B2ECB0F08A8656ECB0F000008A4600005C
:10287C008A4245ECB0F06FECB0F00000100E816EA7
:10288C00100E816E09EC91F0000000008A6A4CEC8D
:10289C00B0F0000000008A6AC7ECB8F000008A6A49
:1028AC004CECB0F000000000100E816E97ECB0F014
:1028BC000000000000008DECB0F0100E816E6FEC8B
:1028CC00B0F000004CECB0F00000000000005BEC3D
:1028DC00B0F08A6AB2ECB0F08A88BEECB0F08A42F2
:1028EC00CDECB0F00000000000008A46BEECB0F069
:1028FC008A6AB2ECB0F08A885BECB0F000000000A1
:10290C00000045ECB0F06FECB0F00000100E816EE2
:10291C0097ECB0F00000000000008DECB0F000006F
:10292C00000000008A6A4CECB0F0000000008A6ADB
:10293C00C7ECB8F000008A6A000085EC91F0100E2C
:10294C00816E080E816E6FECB0F000004CECB0F0B4
:10295C008A4600008A425BECB0F0000000008A6AF4
:10296C00BEECB0F08A88BEECB0F08A4297ECB0F0C6
:10297C0000000000000092ECB0F000008A46BEECB3
:10298C00B0F08A6ABEECB0F08A865BECB0F0000066
:10299C0000008A4600008A4245ECB0F06FECB0F0C3
:1029AC000000100E816E080E816E27EC91F0000075
:1029BC0000008A6A4CECB0F0000000008A6AC7EC98
:1029CC00B8F000008A6A000085EC91F0100E816E60
:1029DC00080E816E6FECB0F000004CECB0F08A4643
:1029EC0000008A4265ECB0F000008A6ABEECB0F0E0
:1029FC008A88BEECB0F08A4297ECB0F00000000080
:102A0C0000008DECB0F08A46BEECB0F08A6ABEECE9
:102A1C00B0F08A8665ECB0F000008A4600008A426D
:102A2C0045ECB0F06FECB0F00000100E816E080EAB
:102A3C00816E27EC91F0000000008A6A4CECB0F03B
:102A4C00000000008A6AC7ECB8F000008A6A000037
:102A5C0085EC91F0100E816E080E816E6FECB0F06B
:102A6C0000004CECB0F08A4600008A426AECB0F0F0
:102A7C008A6AC2ECB0F08A88C2ECB0F08A4297EC59
:102A8C00B0F000000000000079ECB0F000008A46C5
:102A9C00C2ECB0F08A6AC2ECB0F08A866AECB0F094
:102AAC008A4600008A4245ECB0F06FECB0F00000B2
:102ABC00100E816E080E816E27EC91F00000000064
:102ACC008A6A4CECB0F0000000008A6AC7ECB8F0DF
:102ADC0000008A6A000085EC91F0100E816E080EE1
:102AEC00816E6FECB0F000004CECB0F08A46000048
:102AFC008A426FECB0F08A6AC2ECB0F08A88C2EC01
:102B0C00B0F08A4297ECB0F00000000000006AECD4
:102B1C00B0F000008A46C2ECB0F08A6AC2ECB0F0A9
:102B2C008A866FECB0F08A4600008A4245ECB0F021
:102B3C006FECB0F00000100E816E080E816E27EC69
:102B4C0091F0000000008A6A4CECB0F0000000002C
:102B5C008A6AC7ECB8F000008A6A000085EC91F034
:102B6C00100E816E080E816E6FECB0F000004CEC14
:102B7C00B0F08A4600008A4279ECB0F08A6AC2EC66
:102B8C00B0F08A88C7ECB0F08A4297ECB0F0000045
:102B9C000000000056ECB0F0000000008A46C7ECC4
:102BAC00B0F08A6AC2ECB0F08A8679ECB0F08A4652
:102BBC0000008A4245ECB0F06FECB0F00000100E53
:102BCC00816E080E816E27EC91F0000000008A6A7D
:102BDC004CECB0F0000000008A6AC7ECB8F0100EA4
:102BEC00816E000085EC91F0100E816E080E816EE6
:102BFC006FECB0F000004CECB0F08A4600008A425A
:102C0C0079ECB0F0000000008A6AC7ECB0F08A885A
:102C1C004CECB0F08A4297ECB0F0000000000000E1
:102C2C00C7ECB0F08A464CECB0F08A6AC7ECB0F056
:102C3C008A8679ECB0F0000000008A4600008A42D7
:102C4C0045ECB0F06FECB0F00000100E816E080E89
:102C5C00816E27EC91F00000100E816E4CECB0F000
:102C6C00000000008A6AC7ECB8F0100E816E0000FC
:102C7C0085EC91F0100E816E080E816E6FECB0F049
:102C8C0000004CECB0F08A4600008A4283ECB0F0B5
:102C9C008A6AC7ECB0F08A884CECB0F000000000F7
:102CAC008A4297ECB0F08A464CECB0F00000000081
:102CBC008A6AC7ECB0F08A8683ECB0F08A460000D2
:102CCC008A4245ECB0F06FECB0F00000100E816E53
:102CDC00080E816E27EC91F00000100E816E4CEC0A
:102CEC00B0F0000000008A6AC7ECB8F0100E816EDC
:102CFC0076EC91F0100E816E080E816E51ECB0F0F6
:102D0C000000100E816E00000000080E816E56EC63
:102D1C00B0F000000000100E816E080E816E6FEC9A
:102D2C00B0F000004CECB0F08A4600008A428DEC0A
:102D3C00B0F08A6A4CECB0F08A8851ECB0F000002C
:102D4C0000008A426FECB0F0000000008A4651ECA3
:102D5C00B0F0000000008A6A4CECB0F08A868DEC72
:102D6C00B0F08A4600008A4245ECB0F06FECB0F04F
:102D7C000000100E816E080E816E5BECB0F000004E
:102D8C00100E816E00000000080E816E4CECB0F04D
:102D9C0000000000100E816E080E816E18EC91F090
:102DAC0000008A6AC7ECB8F0100E816E76EC91F0D8
:102DBC00100E816E080E816E4CECB0F0000000001D
:102DCC00100E816E7CECBAF0080E816E56ECB0F0F1
:102DDC00100E816E080E816E6FECB0F000004CECA2
:102DEC00B0F08A4600008A428DECB0F08A460000B2
:102DFC008A4200008A6A4CECB0F0000000008A881D
:102E0C0097ECB0F000000000000000000000000093
:102E1C008A6A4CECB0F0000000008A8600008A46FA
:102E2C0000008A428DECB0F08A4600008A4245ECE4
:102E3C00B0F06FECB0F00000100E816E080E816ED9
:102E4C0056ECB0F000000000100E816E5EECBBF092
:102E5C00080E816E4CECB0F0100E816E080E816E77
:102E6C0018EC91F000008A6AC7ECB8F0100E816E75
:102E7C0076EC91F0100E816E080E816E4CECB0F079
:102E8C00100E816E75ECBAF0080E816E51ECB0F03C
:102E9C000000100E816E080E816E6FECB0F0000019
:102EAC004CECB0F08A4600008A428DECB0F08A46B9
:102EBC0000008A42A1ECB0F08A6A51ECB0F000003C
:102ECC008A888DECB0F08A6A51ECB0F000008A86EA
:102EDC00A1ECB0F08A4600008A428DECB0F08A4634
:102EEC0000008A4245ECB0F06FECB0F00000100E20
:102EFC00816E080E816E56ECB0F0100E816E57ECA0
:102F0C00BBF0080E816EC7ECB0F0100E816E080E8F
:102F1C00816E18EC91F000008A6AC7ECB8F0100EC4
:102F2C00816E76EC91F0100E816E080E816EC7ECFE
:102F3C00B0F0100E816E70ECBAF0080E816E4CEC95
:102F4C00B0F000000000100E816E080E816E6FEC68
:102F5C00B0F000004CECB0F08A4600008A428DECD8
:102F6C00B0F08A4600008A424CECB0F000008A6A4D
:102F7C005BECB0F0000000008A860000000000004E
:102F8C008A46A1ECB0F08A420000000000008A6A78
:102F9C005BECB0F0000000008A864CECB0F0000056
:102FAC008A4600008A428DECB0F08A4600008A42C4
:102FBC0045ECB0F06FECB0F00000100E816E080E16
:102FCC00816E51ECB0F00000100E816E52ECBBF033
:102FDC00080E816EBEECB0F0100E816E080E816E84
:102FEC0018EC91F000008A6AC7ECB8F0100E816EF4
:102FFC0076EC91F0100E816E080E816EBEECB0F086
:10300C00100E816E67ECBAF0080E816E4CECB0F0CD
:10301C00100E816E080E816E6FECB0F000004CEC5F
:10302C00B0F08A4600008A428DECB0F08A4600006F
:10303C008A4256ECB0F000008A6A97ECB0F08A86AF
:10304C0056ECB0F000008A4600008A428DECB0F0DD
:10305C008A4600008A4245ECB0F06FECB0F00000FC
:10306C00100E816E080E816E4CECB0F0000000006A
:10307C00100E816E49ECBBF0080E816EA1ECB0F025
:10308C00100E816E080E816E18EC91F000008A6AA9
:10309C00C7ECB8F0100E816E76EC91F0100E816ECC
:1030AC00080E816EA1ECB0F0100E816E5AECBAF0E5
:1030BC00080E816EC7ECB0F0100E816E080E816E9A
:1030CC006FECB0F000004CECB0F08A4600008A4285
:1030DC008DECB0F08A4600008A4265ECB0F000003E
:1030EC0000008A6A79ECB0F000008A8665ECB0F0DA
:1030FC00000000008A4600008A428DECB0F08A463F
:10310C0000008A4245ECB0F06FECB0F00000100EFD
:10311C00816E080E816E4CECB0F0100E816E3CECA2
:10312C00BBF0080E816E000000000000100E816ED6
:10313C00080E816E18EC91F000008A6AC7ECB8F0AA
:10314C00100E816E76EC91F0100E816E080E816E71
:10315C00000000000000100E816E55ECBAF0080E55
:10316C00816EBEECB0F0100E816E080E816E01EC1B
:10317C007EF0100E816E080E816EC7ECB0F0100E52
:10318C00816E37ECBBF0080E816E0000100E816E64
:10319C00080E816E18EC91F000008A6AC7ECB8F04A
:1031AC00100E816E76EC91F0100E816E080E816E11
:1031BC000000100E816E4CECBAF0080E816EA1EC82
:1031CC00B0F0100E816E080E816E01EC7EF0100EC8
:1031DC00816E080E816EBEECB0F0100E816E2EEC7E
:1031EC00BBF00000100E816E080E816E18EC91F091
:1031FC0000008A6AC7ECB8F0100E816E76EC91F084
:10320C00100E816E0000100E816E3FECBAF0080EAD
:10321C00816E000000000000100E816E080E816EA1
:10322C0001EC7EF0100E816E080E816EA1ECB0F0F8
:10323C00100E816E21ECBBF00000080E816E18ECB4
:10324C0091F000008A6AC7ECB8F0100E816E76EC33
:10325C0091F000008A46000034ECBAF0080E816E42
:10326C000000100E816E080E816E01EC7EF0100EC7
:10327C00816E080E816E000000000000100E816E41
:10328C0016ECBBF0080E816E83ECB0F00000100E53
:10329C00816E080E816E000000000000100E816E21
:1032AC004CECB0F0000000008A6AEAEC98F087EF72
:1032BC0032F0E8EC9FF000008A6AC7ECB8F0100E10
:1032CC00816E76EC91F000008A46000034ECBAF086
:1032DC00080E816E0000100E816E080E816E01ECDE
:1032EC007EF0100E816E080E816E00000000000052
:1032FC00100E816E16ECBBF0080E816E83ECB0F0F4
:10330C000000100E816E080E816E0000000000009F
:10331C00100E816EB2ECB0F082A08BEF32F082A274
:10332C00C4EF79F000008A6AC7ECB8F0100E816E19
:10333C0076EC91F0100E816E0000100E816E3FEC59
:10334C00BAF0080E816E000000000000100E816EB5
:10335C00080E816E01EC7EF0100E816E080E816EEF
:10336C00A1ECB0F0100E816E21ECBBF00000080E49
:10337C00816E18EC91F000008A6AC7ECB8F0100E60
:10338C00816E76EC91F0100E816E080E816E00004D
:10339C00100E816E4CECBAF0080E816EA1ECB0F000
:1033AC00100E816E080E816E01EC7EF0100E816E97
:1033BC00080E816EBEECB0F0100E816E2EECBBF0E0
:1033CC000000100E816E080E816E18EC91F000005A
:1033DC008A6AC7ECB8F0100E816E76EC91F0100E84
:1033EC00816E080E816E000000000000100E816ED0
:1033FC0055ECBAF0080E816EBEECB0F0100E816E7A
:10340C00080E816E01EC7EF0100E816E080E816E3E
:10341C00C7ECB0F0100E816E37ECBBF0080E816E6D
:10342C000000100E816E080E816E18EC91F00000F9
:10343C008A6AC7ECB8F0100E816E76EC91F0100E23
:10344C00816E080E816EA1ECB0F0100E816E5AECFC
:10345C00BAF0080E816EC7ECB0F0100E816E080E3B
:10346C00816E6FECB0F000004CECB0F08A460000BE
:10347C008A428DECB0F08A4600008A4265ECB0F0CE
:10348C00000000008A6A79ECB0F000008A8665ECD6
:10349C00B0F0000000008A4600008A428DECB0F0CB
:1034AC008A4600008A4245ECB0F06FECB0F00000A8
:1034BC00100E816E080E816E4CECB0F0100E816E09
:1034CC003CECBBF0080E816E000000000000100EFA
:1034DC00816E080E816E18EC91F000008A6AC7ECC0
:1034EC00B8F0100E816E76EC91F0100E816E080E15
:1034FC00816EBEECB0F0100E816E67ECBAF0080E67
:10350C00816E4CECB0F0100E816E080E816E6FEC7B
:10351C00B0F000004CECB0F08A4600008A428DEC12
:10352C00B0F08A4600008A4256ECB0F000008A6A7D
:10353C0097ECB0F08A8656ECB0F000008A4600009A
:10354C008A428DECB0F08A4600008A4245ECB0F01D
:10355C006FECB0F00000100E816E080E816E4CEC1A
:10356C00B0F000000000100E816E49ECBBF0080EAC
:10357C00816EA1ECB0F0100E816E080E816E18EC0D
:10358C0091F000008A6AC7ECB8F0100E816E76ECF0
:10359C0091F0100E816E080E816EC7ECB0F0100E1B
:1035AC00816E70ECBAF0080E816E4CECB0F000003D
:1035BC000000100E816E080E816E6FECB0F00000F2
:1035CC004CECB0F08A4600008A428DECB0F08A4692
:1035DC0000008A424CECB0F000008A6A5BECB0F060
:1035EC00000000008A860000000000008A46A1EC62
:1035FC00B0F08A420000000000008A6A5BECB0F078
:10360C00000000008A864CECB0F000008A460000F6
:10361C008A428DECB0F08A4600008A4245ECB0F04C
:10362C006FECB0F00000100E816E080E816E51EC44
:10363C00B0F00000100E816E52ECBBF0080E816EE3
:10364C00BEECB0F0100E816E080E816E18EC91F08D
:10365C0000008A6AC7ECB8F0100E816E76EC91F01F
:10366C00100E816E080E816E4CECB0F0100E816E57
:10367C0075ECBAF0080E816E51ECB0F00000100E33
:10368C00816E080E816E6FECB0F000004CECB0F067
:10369C008A4600008A428DECB0F08A4600008A42CD
:1036AC00A1ECB0F08A6A51ECB0F000008A888DEC85
:1036BC00B0F08A6A51ECB0F000008A86A1ECB0F050
:1036CC008A4600008A428DECB0F08A4600008A429D
:1036DC0045ECB0F06FECB0F00000100E816E080EEF
:1036EC00816E56ECB0F0100E816E57ECBBF0080EEC
:1036FC00816EC7ECB0F0100E816E080E816E18EC66
:10370C0091F000008A6AC7ECB8F0100E816E76EC6E
:10371C0091F0100E816E080E816E4CECB0F0000032
:10372C000000100E816E7CECBAF0080E816E56EC27
:10373C00B0F0100E816E080E816E6FECB0F00000D0
:10374C004CECB0F08A4600008A428DECB0F08A4610
:10375C0000008A4200008A6A4CECB0F000000000C5
:10376C008A8897ECB0F00000000000000000000018
:10377C0000008A6A4CECB0F0000000008A86000061
:10378C008A4600008A428DECB0F08A4600008A42DC
:10379C0045ECB0F06FECB0F00000100E816E080E2E
:1037AC00816E56ECB0F000000000100E816E5EECE5
:1037BC00BBF0080E816E4CECB0F0100E816E080E52
:1037CC00816E18EC91F000008A6AC7ECB8F0100E0C
:1037DC00816E76EC91F0100E816E080E816E51ECBC
:1037EC00B0F00000100E816E00000000080E816E1B
:1037FC0056ECB0F000000000100E816E080E816EC9
:10380C006FECB0F000004CECB0F08A4600008A423D
:10381C008DECB0F08A6A4CECB0F08A8851ECB0F0C8
:10382C00000000008A426FECB0F0000000008A46F5
:10383C0051ECB0F0000000008A6A4CECB0F08A86C3
:10384C008DECB0F08A4600008A4245ECB0F06FEC8B
:10385C00B0F00000100E816E080E816E5BECB0F0C3
:10386C000000100E816E00000000080E816E4CEC02
:10387C00B0F000000000100E816E080E816E18EC86
:10388C0091F000008A6AC7ECB8F0100E816E76ECED
:10389C0091F0100E816E080E816E83ECB0F000007A
:1038AC000000100E816E080E816E6FECB0F00000FF
:1038BC004CECB0F08A4600008A4283ECB0F08A6A85
:1038CC00C7ECB0F08A884CECB0F0000000008A42E3
:1038DC0097ECB0F08A464CECB0F0000000008A6A1D
:1038EC00C7ECB0F08A8683ECB0F08A4600008A42BE
:1038FC0045ECB0F06FECB0F00000100E816E080ECD
:10390C00816E83ECB0F000000000100E816E080E8A
:10391C00816E18EC91F000008A6AC7ECB8F0100EBA
:10392C00816E76EC91F0100E816E080E816E83EC38
:10393C00B0F000000000100E816E080E816E6FEC6E
:10394C00B0F000004CECB0F08A4600008A4279ECF2
:10395C00B0F0000000008A6AC7ECB0F08A884CEC2A
:10396C00B0F08A4297ECB0F0000000000000C7EC09
:10397C00B0F08A464CECB0F08A6AC7ECB0F08A869C
:10398C0079ECB0F0000000008A4600008A4245EC59
:10399C00B0F06FECB0F00000100E816E080E816E6E
:1039AC0083ECB0F000000000100E816E080E816EEA
:1039BC0083ECB0F000000000100E816E080E816EDA
:1039CC00000000000000100E816E4CECB0F0000006
:1039DC0000008A6AC7ECB8F000008A6A000085EC27
:1039EC0091F0100E816E080E816E6FECB0F000003D
:1039FC004CECB0F08A4600008A4279ECB0F08A6A4E
:103A0C00C2ECB0F08A88C7ECB0F08A4297ECB0F008
:103A1C0000000000000056ECB0F0000000008A46E8
:103A2C00C7ECB0F08A6AC2ECB0F08A8679ECB0F0E0
:103A3C008A4600008A4245ECB0F06FECB0F0000012
:103A4C00100E816E080E816E27EC91F000000000C4
:103A5C008A6A4CECB0F0000000008A6AC7ECB8F03F
:103A6C0000008A6A000085EC91F0100E816E080E41
:103A7C00816E6FECB0F000004CECB0F08A460000A8
:103A8C008A426FECB0F08A6AC2ECB0F08A88C2EC61
:103A9C00B0F08A4297ECB0F00000000000006AEC35
:103AAC00B0F000008A46C2ECB0F08A6AC2ECB0F00A
:103ABC008A866FECB0F08A4600008A4245ECB0F082
:103ACC006FECB0F00000100E816E080E816E27ECCA
:103ADC0091F0000000008A6A4CECB0F0000000008D
:103AEC008A6AC7ECB8F000008A6A000085EC91F095
:103AFC00100E816E080E816E6FECB0F000004CEC75
:103B0C00B0F08A4600008A426AECB0F08A6AC2ECD5
:103B1C00B0F08A88C2ECB0F08A4297ECB0F00000AA
:103B2C000000000079ECB0F000008A46C2ECB0F066
:103B3C008A6AC2ECB0F08A866AECB0F08A46000061
:103B4C008A4245ECB0F06FECB0F00000100E816EC4
:103B5C00080E816E27EC91F0000000008A6A4CEC94
:103B6C00B0F0000000008A6AC7ECB8F000008A6A66
:103B7C00000085EC91F0100E816E080E816E6FECDA
:103B8C00B0F000004CECB0F08A4600008A4265ECC4
:103B9C00B0F000008A6ABEECB0F08A88BEECB0F0DF
:103BAC008A4297ECB0F00000000000008DECB0F001
:103BBC008A46BEECB0F08A6ABEECB0F08A8665EC40
:103BCC00B0F000008A4600008A4245ECB0F06FEC81
:103BDC00B0F00000100E816E080E816E27EC91F093
:103BEC00000000008A6A4CECB0F0000000008A6A09
:103BFC00C7ECB8F000008A6A000085EC91F0100E5A
:103C0C00816E080E816E6FECB0F000004CECB0F0E1
:103C1C008A4600008A425BECB0F0000000008A6A21
:103C2C00BEECB0F08A88BEECB0F08A4297ECB0F0F3
:103C3C0000000000000092ECB0F000008A46BEECE0
:103C4C00B0F08A6ABEECB0F08A865BECB0F0000093
:103C5C0000008A4600008A4245ECB0F06FECB0F0F0
:103C6C000000100E816E080E816E27EC91F00000A2
:103C7C0000008A6A4CECB0F0000000008A6AC7ECC5
:103C8C00B8F000008A6A000085EC91F0100E816E8D
:103C9C00080E816E6FECB0F000004CECB0F08A4670
:103CAC0000008A425BECB0F08A6AA1ECB0F08A6A40
:103CBC0000008A88000079ECB0F0000000008A4215
:103CCC006AECB0F00000000051ECB0F00000100EF7
:103CDC00816E79ECB0F0000000008A6A00008A6AFC
:103CEC00A1ECB0F08A865BECB0F08A4600008A4208
:103CFC0045ECB0F06FECB0F00000100E816E080EC9
:103D0C00816E27EC91F0000000008A6A4CECB0F058
:103D1C00000000008A6AC7ECB8F000008A6A4CEC1C
:103D2C00B0F000000000100E816ECDECB0F0000081
:103D3C00000065ECB0F051ECB0F051ECB0F00000CC
:103D4C0000008A4200008A6AB2ECB0F08A88100E39
:103D5C00816E93EC7CF08A426AECB0F000000000BB
:103D6C0051ECB0F00000100E816EF6EC7CF08A88FD
:103D7C008A6AB2ECB0F08A8600008A4651ECB0F048
:103D8C00000000004CECB0F000000000CDECB0F0F6
:103D9C000000000065ECB0F00000000000008A6A32
:103DAC004CECB0F0000000008A6AC7ECB8F00000E0
:103DBC008A6A00005FEC91F0100E816E080E816E25
:103DCC006FECB0F000004CECB0F08A4600008A4278
:103DDC0051ECB0F0000000008A6AB2ECB0F08A88B6
:103DEC0000000000100E816E93EC7CF08A426AECAD
:103DFC00B0F00000000051ECB0F00000100E816E2D
:103E0C00F6EC7CF08A88000000008A6AB2ECB0F014
:103E1C008A8651ECB0F0000000008A4600008A420D
:103E2C0045ECB0F06FECB0F00000100E816E100E8F
:103E3C00816E09EC91F0000000008A6A4CECB0F045
:103E4C00000000008A6AC7ECB8F000008A6A000023
:103E5C005FEC91F0100E816E080E816E6FECB0F07D
:103E6C0000004CECB0F08A4600008A4251ECB0F0F5
:103E7C008A6AB2ECB0F08A880000000000000000F2
:103E8C00100E816E93EC7CF08A426AECB0F000006C
:103E9C00000051ECB0F00000100E816EF6EC7CF0DE
:103EAC008A8800000000000000008A6AB2ECB0F0C2
:103EBC008A8651ECB0F08A4600008A4245ECB0F09C
:103ECC006FECB0F00000100E816E100E816E09ECDC
:103EDC0091F0000000008A6A4CECB0F00000000089
:103EEC008A6AC7ECB8F000008A6A00005FEC91F0B7
:103EFC00100E816E080E816E6FECB0F000004CEC71
:103F0C00B0F08A4600008A424CECB0F00000000091
:103F1C008A6AA1ECB0F08A88B2ECB0F0100E816E17
:103F2C0093EC7CF08A426AECB0F00000000051EC9B
:103F3C00B0F00000100E816EF6EC7CF08A88B2ECCA
:103F4C00B0F08A6AA1ECB0F08A864CECB0F00000BC
:103F5C0000008A4600008A4245ECB0F06FECB0F0ED
:103F6C000000100E816E100E816E09EC91F00000B5
:103F7C0000008A6A4CECB0F0000000008A6AC7ECC2
:103F8C00B8F000008A6A00005FEC91F0100E816EB0
:103F9C00080E816E6FECB0F000004CECB0F08A466D
:103FAC0000008A424CECB0F08A6AB2ECB0F08A881D
:103FBC00A1ECB0F08A420000100E816E93EC7CF004
:103FCC008A426AECB0F00000000051ECB0F0000046
:103FDC00100E816EF6EC7CF08A4200008A46A1EC51
:103FEC00B0F08A6AB2ECB0F08A864CECB0F08A463B
:103FFC0000008A4245ECB0F06FECB0F00000100EFF
:10400C00816E100E816E09EC91F0000000008A6A3E
:10401C004CECB0F0000000008A6AC7ECB8F000006D
:10402C008A6A00005FEC91F0100E816E080E816EB2
:10403C006FECB0F000004CECB0F08A4600008A4205
:10404C0045ECB0F08A6AA1ECB0F08A88A1ECB0F033
:10405C008A42000000000000100E816E93EC7CF090
:10406C008A426AECB0F00000000051ECB0F00000A5
:10407C00100E816EF6EC7CF08A420000000000000D
:10408C008A46A1ECB0F08A6AA1ECB0F08A8645ECC5
:10409C00B0F08A4600008A4245ECB0F06FECB0F00C
:1040AC000000100E816E100E816E09EC91F0000074
:1040BC0000008A6A4CECB0F0000000008A6AC7EC81
:1040CC00B8F0100E816E00005FEC91F0100E816E56
:1040DC00080E816E6FECB0F000004CECB0F08A462C
:1040EC0000008A42C2ECB0F08A6AA1ECB0F08A8877
:1040FC00B2ECB0F08A420000000000000000100E8C
:10410C00816E93EC7CF08A42BEECB0F08A466AEC8D
:10411C00B0F000008A42BEECB0F0100E816EF6ECEE
:10412C007CF08A4200000000000000008A46B2ECDD
:10413C00B0F08A6AA1ECB0F08A86C2ECB0F08A4684
:10414C0000008A4245ECB0F06FECB0F00000100EAD
:10415C00816E100E816E09EC91F00000100E816ED4
:10416C004CECB0F0000000008A6AC7ECB8F0100EFE
:10417C00816E00005FEC91F0100E816E080E816E66
:10418C006FECB0F000004CECB0F08A4600008A42B4
:10419C00BEECB0F08A6AA1ECB0F08A88A1ECB0F069
:1041AC008A42B2ECB0F0100E816E93EC7CF08A4235
:1041BC00BEECB0F08A466AECB0F000008A42BEEC6D
:1041CC00B0F0100E816EF6EC7CF08A42B2ECB0F0DE
:1041DC008A46A1ECB0F08A6AA1ECB0F08A86BEECFB
:1041EC00B0F08A4600008A4245ECB0F06FECB0F0BB
:1041FC000000100E816E100E816E09EC91F0000023
:10420C00100E816E4CECB0F0000000008A6AC7EC16
:10421C00B8F0100E816E00005FEC91F0100E816E04
:10422C00080E816E6FECB0F000004CECB0F08A46DA
:10423C0000008A42B2ECB0F08A6AA1ECB0F08A8835
:10424C00A1ECB0F08A42BEECB0F0100E816E93EC93
:10425C007CF08A42BEECB0F08A466AECB0F000000A
:10426C008A42BEECB0F0100E816EF6EC7CF08A4205
:10427C00BEECB0F08A46A1ECB0F08A6AA1ECB0F0CA
:10428C008A86B2ECB0F08A4600008A4245ECB0F067
:10429C006FECB0F00000100E816E100E816E09EC08
:1042AC0091F00000100E816E4CECB0F0000000009C
:1042BC008A6AC7ECB8F0100E816E00005FEC91F0CA
:1042CC00100E816E080E816E6FECB0F000004CEC9D
:1042DC00B0F08A4600008A42000000000000000096
:1042EC008A6AA1ECB0F08A88A1ECB0F08A42C7ECE3
:1042FC00B0F0100E816E93EC7CF08A42BEECB0F004
:10430C008A466AECB0F000008A42BEECB0F0100EA7
:10431C00816EF6EC7CF08A42C7ECB0F08A46A1ECD8
:10432C00B0F08A6AA1ECB0F08A86000000000000B0
:10433C0000008A4600008A4245ECB0F06FECB0F009
:10434C000000100E816E100E816E09EC91F00000D1
:10435C00100E816E4CECB0F0000000008A6AC7ECC5
:10436C00B8F0100E816E00005FEC91F0100E816EB3
:10437C00080E816E6FECB0F000004CECB0F08A4689
:10438C0000008A420000000000008A6AA1ECB0F034
:10439C008A88A1ECB0F08A4245ECB0F0100E816E28
:1043AC0093EC7CF08A42BEECB0F08A466AECB0F03A
:1043BC0000008A42BEECB0F0100E816EF6EC7CF080
:1043CC008A4245ECB0F08A46A1ECB0F08A6AA1ECC6
:1043DC00B0F08A860000000000008A4600008A4285
:1043EC0045ECB0F06FECB0F00000100E816E100ECA
:1043FC00816E09EC91F00000100E816E4CECB0F067
:10440C00000000008A6AC7ECB8F0100E816E000044
:10441C005FEC91F0100E816E080E816E6FECB0F0B7
:10442C0000004CECB0F08A468A420000000000000C
:10443C008A6AA1ECB0F08A88A1ECB0F08A424CEC0C
:10444C00B0F0100E816E93EC7CF08A42BEECB0F0B2
:10445C008A466AECB0F000008A42BEECB0F0100E56
:10446C00816EF6EC7CF08A424CECB0F08A46A1EC02
:10447C00B0F08A6AA1ECB0F08A860000000000005F
:10448C008A468A4245ECB0F06FECB0F00000100E9A
:10449C00816E100E816E09EC91F00000100E816E91
:1044AC004CECB0F0000000008A6AC7ECB8F0100EBB
:1044BC00816E9CEC91F0100E816E080E816E6FEC8B
:1044CC00B0F0000051ECB0F000008A6AA1ECB0F042
:1044DC008A8800000000000000008A424CECB0F01A
:1044EC0000000000100E816E93EC7CF08A42BEEC52
:1044FC00B0F08A466AECB0F000008A42BEECB0F034
:10450C00100E816EF6EC7CF08A424CECB0F00000A0
:10451C0000008A4600000000000000008A6AA1EC3E
:10452C00B0F08A8651ECB0F06FECB0F00000100ED9
:10453C00816E100E816E36EC91F0100E816E4CEC8B
:10454C00B0F0000000008A6AC7ECB8F0100E816E63
:10455C009CEC91F0100E816E080E816E6FECB0F039
:10456C00000051ECB0F08A6AA1ECB0F08A8800002F
:10457C000000000000008A4251ECB0F0100E816E79
:10458C0093EC7CF08A42BEECB0F08A466AECB0F058
:10459C0000008A42BEECB0F0100E816EF6EC7CF09E
:1045AC008A4251ECB0F08A46000000000000000086
:1045BC008A6AA1ECB0F08A864CECB0F000000000E6
:1045CC006FECB0F00000100E816E100E816E36ECA8
:1045DC0091F0100E816E4CECB0F0000000008A6A75
:1045EC00C7ECB8F0100E816E9CEC91F0100E816E41
:1045FC00080E816E6FECB0F000004CECB0F00000D7
:10460C0000008A6AA1ECB0F08A880000000000006B
:10461C0000008A4251ECB0F00000100E816E93EC59
:10462C007CF08A42BEECB0F08A466AECB0F0000036
:10463C008A42BEECB0F0100E816EF6EC7CF08A4231
:10464C0051ECB0F000008A460000000000000000B1
:10465C008A6AA1ECB0F08A864CECB0F000006FECEA
:10466C00B0F00000100E816E100E816E36EC91F0E1
:10467C00100E816E4CECB0F0000000008A6AC7ECA2
:10468C00B8F0100E816E9CEC91F0100E816E080E3D
:10469C00816E6FECB0F000004CECB0F000008A6A58
:1046AC00A1ECB0F08A8800000000000000008A42F3
:1046BC0051ECB0F000000000100E816E93EC7CF019
:1046CC008A42BEECB0F08A466AECB0F000008A4236
:1046DC00BEECB0F0100E816EF6EC7CF08A4251EC20
:1046EC00B0F0000000008A4600000000000000004E
:1046FC008A6AA1ECB0F08A864CECB0F06FECB0F0AA
:10470C000000100E816E100E816E36EC91F0100EC2
:10471C00816E4CECB0F0000000008A6AC7ECB8F077
:10472C00100E816E9CEC91F0100E816E080E816E55
:10473C006FECB0F000004CECB0F08A6AA1ECB0F079
:10474C008A8800000000000000008A4256ECB0F09D
:10475C00100E816E93EC7CF08A42BEECB0F08A466F
:10476C006AECB0F000008A42BEECB0F0100E816E24
:10477C00F6EC7CF08A4256ECB0F08A460000000061
:10478C00000000008A6AA1ECB0F08A8645ECB0F01B
:10479C006FECB0F00000100E816E100E816E36ECD6
:1047AC0091F0100E816E4CECB0F0000000008A6AA3
:1047BC00C7ECB8F0100E816E9CEC91F0100E816E6F
:1047CC00080E816E6FECB0F000004CECB0F08A6A11
:1047DC0000000000000000008A88000000000000BB
:1047EC0000008A4256ECB0F00000100E816E7EEC98
:1047FC00B0F000008A42BEECB0F08A466AECB0F031
:10480C0000008A42BEECB0F0100E816E7EECB0F06F
:10481C0000008A4256ECB0F000008A46000000000E
:10482C00000000008A6A00000000000000008A8678
:10483C0045ECB0F06FECB0F00000100E816E100E75
:10484C00816E36EC91F0100E816E4CECB0F00000E5
:10485C0000008A6AC7ECB8F000008A6A9CEC91F000
:10486C00100E816E080E816EBBEC7FF0100E816E07
:10487C00100E816E36EC91F000008A6A4CECB0F0B0
:10488C00000000008A6AC7ECB8F000008A6A9CEC51
:10489C0091F0100E816E080E816E95EC80F0100E6A
:1048AC00816E100E816E36EC91F000008A6A4CEC31
:1048BC00B0F0000000008A6AC7ECB8F000008A6A09
:1048CC009CEC91F0100E816E080E816E4BEC81F019
:1048DC00100E816E100E816E36EC91F000008A6A1B
:1048EC004CECB0F0000000008A6AC7ECB8F0000095
:1048FC008A6A9CEC91F0100E816E080E816E3DEC74
:10490C0082F0100E816E100E816E36EC91F000006C
:10491C008A6A4CECB0F0000000008A6AC7ECB8F070
:10492C0000008A6A9CEC91F0100E816E080E816E6C
:10493C002EEC83F0100E816E100E816E36EC91F021
:10494C0000008A6A4CECB0F0000000008A6AC7ECE8
:10495C00B8F000008A6A9CEC91F0100E816E080E83
:10496C00816E2AEC84F0100E816E100E816E36EC86
:10497C0091F000008A6A4CECB0F0000000008A6AEA
:10498C00C7ECB8F000008A6A4CECB0F000000000F4
:10499C00100E816E97ECB0F000008A6A56ECB0F005
:1049AC000000100E816E00008A6A56ECB0F0000018
:1049BC00100E816E100E816EE4EC84F0100E816E80
:1049CC00100E816E56ECB0F0000000008A6A100EDA
:1049DC00816E56ECB0F00000100E816E97ECB0F0CA
:1049EC000000000000008A6A4CECB0F000000000EF
:1049FC008A6AC7ECB8F000008A6A9CEC91F0100E41
:104A0C00816E080E816E4EEC86F0100E816E100ECB
:104A1C00816E36EC91F000008A6A4CECB0F000002C
:104A2C0000008A6AC7ECB8F000008A6A9CEC91F02E
:104A3C00100E816E080E816E4EEC86F0100E816E9B
:104A4C00100E816E36EC91F000008A6A4CECB0F0DE
:104A5C00000000008A6AC7ECB8F000008A6A9CEC7F
:104A6C0091F0100E816E080E816E2DEC7EF0100E02
:104A7C00816E100E816E36EC91F000008A6A4CEC5F
:104A8C00B0F0000000008A6AC7ECB8F000008A6A37
:104A9C009CEC91F0100E816E080E816E46EC7FF04E
:104AAC00100E816E100E816E36EC91F000008A6A49
:104ABC004CECB0F0000000008A6AC7ECB8F00000C3
:104ACC008A6A9CEC91F0100E816E080E816E46EC99
:104ADC007FF0100E816E100E816E36EC91F000009E
:104AEC008A6A4CECB0F0000000008A6AC7ECB8F09F
:104AFC00100E816E9CEC91F0100E816E080E816E82
:104B0C0025EC88F0100E816E100E816E36EC91F053
:104B1C00100E816E4CECB0F0000000008A6AC7ECFD
:104B2C00B8F0100E816E9CEC91F0100E816E080E98
:104B3C00816E09EC89F0100E816E100E816E36ECD0
:104B4C0091F0100E816E4CECB0F0000000008A6AFF
:104B5C00C7ECB8F0100E816E9CEC91F0100E816ECB
:104B6C00080E816E22EC8BF0100E816E100E816E91
:104B7C0036EC91F0100E816E4CECB0F000000000A1
:104B8C008A6AC7ECB8F0100E816E9CEC91F0100E96
:104B9C00816E080E816E22EC8BF0100E816E100E61
:104BAC00816E36EC91F0100E816E4CECB0F0000082
:104BBC0000008A6AC7ECB8F0100E816E9CEC91F084
:104BCC00100E816E080E816E22EC8BF0100E816E31
:104BDC00100E816E36EC91F0100E816E4CECB0F034
:104BEC00000000008A6AC7ECB8F0100E816E9CECD5
:104BFC0091F0100E816E080E816EBAEC89F0100ED9
:104C0C00816E100E816E36EC91F0100E816E4CECB4
:104C1C00B0F0000000008A6AC7ECB8F0100E816E8C
:104C2C009CEC91F0100E816E080E816EE3EC8AF014
:104C3C00100E816E100E816E36EC91F0100E816E9E
:104C4C004CECB0F0000000008A6AC7ECB8F0100E13
:104C5C00816E9CEC91F0100E816E080E816EE3EC6F
:104C6C008AF0100E816E100E816E36EC91F0100EE3
:104C7C00816E4CECB0F0000000008A6AC7ECB8F012
:104C8C00100E816E9CEC91F0100E816E080E816EF0
:104C9C00E3EC8AF0100E816E100E816E36EC91F002
:104CAC00100E816E4CECB0F0000000008A6AC7EC6C
:104CBC00B8F0100E816E9CEC91F0100E816E080E07
:104CCC00816EE3EC8AF0100E816E100E816E36EC64
:104CDC0091F0100E816E4CECB0F0000000008A6A6E
:104CEC00C7ECB8F0100E816E9CEC91F0100E816E3A
:104CFC00080E816E35EC87F0100E816E100E816EF1
:104D0C0036EC91F0100E816E4CECB0F0000000000F
:104D1C008A6AC7ECB8F0100E816E9CEC91F0100E04
:104D2C00816E080E816EE9EC87F0100E816E100E0C
:104D3C00816E36EC91F0100E816E4CECB0F00000F0
:104D4C0000008A6AC7ECB8F000008A6A9CEC91F00B
:104D5C00100E816E080E816E04EC8DF0100E816EBB
:104D6C00100E816E36EC91F000008A6A4CECB0F0BB
:104D7C00000000008A6AC7ECB8F000008A6A9CEC5C
:104D8C0091F0100E816E080E816E04EC8DF0100EF9
:104D9C00816E100E816E36EC91F000008A6A4CEC3C
:104DAC00B0F0000000008A6AC7ECB8F000008A6A14
:104DBC009CEC91F0100E816E080E816EB2EC8DF0B1
:104DCC00100E816E100E816E36EC91F000008A6A26
:104DDC004CECB0F0000000008A6AC7ECB8F00000A0
:104DEC008A6A9CEC91F0100E816E080E816E27EC95
:104DFC008EF0100E816E100E816E36EC91F000006C
:104E0C008A6A4CECB0F0000000008A6AC7ECB8F07B
:104E1C0000008A6A9CEC91F0100E816E080E816E77
:104E2C0096EC8EF0100E816E100E816E36EC91F0B9
:104E3C0000008A6A4CECB0F0000000008A6AC7ECF3
:104E4C00B8F000008A6A9CEC91F0100E816E080E8E
:104E5C00816E11EC8FF0100E816E100E816E36EC9F
:104E6C0091F000008A6A4CECB0F0000000008A6AF5
:104E7C00C7ECB8F000008A6A4CECB0F000000000FF
:104E8C00100E816E97ECB0F000008A6A56ECB0F010
:104E9C000000100E816E00008A6A56ECB0F0000023
:104EAC00100E816E100E816E8AEC8FF0100E816EDA
:104EBC00100E816E56ECB0F0000000008A6A100EE5
:104ECC00816E56ECB0F00000100E816E97ECB0F0D5
:104EDC000000000000008A6A4CECB0F000000000FA
:104EEC008A6AC7ECB8F000008A6A9CEC91F0100E4C
:104EFC00816E080E816E12EC90F0100E816E100E09
:104F0C00816E36EC91F000008A6A4CECB0F0000037
:104F1C0000008A6AC7ECB8F000008A6A9CEC91F039
:104F2C00100E816E080E816E8FEC90F0100E816E5B
:104F3C00100E816E36EC91F000008A6A4CECB0F0E9
:104F4C00000000008A6AC7ECB8F000008A6A9CEC8A
:104F5C0091F0100E816E080E816EA0EC8BF0100E8D
:104F6C00816E100E816E36EC91F000008A6A4CEC6A
:104F7C00B0F0000000008A6AC7ECB8F000008A6A42
:104F8C009CEC91F0100E816E080E816E52EC8CF040
:104F9C00100E816E100E816E36EC91F000008A6A54
:104FAC004CECB0F0000000008A6AC7ECB8F00000CE
:104FBC008A6A9CEC91F0100E816E080E816E90EC5A
:104FCC008CF0100E816E100E816E36EC91F000009C
:104FDC008A6A4CECB0F0000000008A6AC7ECB8F0AA
:104FEC00100E816E9CEC91F0100E816E080E816E8D
:104FFC006FECB0F000004CECB0F08A6A00000000DE
:10500C00000000008A88A1ECB0F08A4256ECB0F0A7
:10501C00100E816EF6EC7CF08A42BEECB0F08A6A1F
:10502C006AECB0F000008A86BEECB0F0100E816E17
:10503C0093EC7CF08A4256ECB0F08A46A1ECB0F0CE
:10504C008A6A00000000000000008A8645ECB0F07F
:10505C006FECB0F00000100E816E100E816E36EC0D
:10506C0091F0100E816E4CECB0F0000000008A6ADA
:10507C00C7ECB8F0100E816E9CEC91F0100E816EA6
:10508C00080E816E6FECB0F000004CECB0F000003C
:10509C008A6A00000000000000008A88A1ECB0F0D1
:1050AC008A4251ECB0F000000000100E816EF6EC5C
:1050BC007CF08A42BEECB0F08A6A6AECB0F0000078
:1050CC008A86BEECB0F0100E816E93EC7CF08A42B6
:1050DC0051ECB0F0000000008A46A1ECB0F08A6AF6
:1050EC0000000000000000008A864CECB0F06FEC71
:1050FC00B0F00000100E816E100E816E36EC91F047
:10510C00100E816E4CECB0F0000000008A6AC7EC07
:10511C00B8F0100E816E9CEC91F0100E816E080EA2
:10512C00816E6FECB0F000004CECB0F000000000B1
:10513C008A6A00000000000000008A88A1ECB0F030
:10514C008A4251ECB0F00000100E816EF6EC7CF04F
:10515C008A42BEECB0F08A6A6AECB0F000008A8633
:10516C00BEECB0F0100E816E93EC7CF08A4251ECE8
:10517C00B0F000008A46A1ECB0F08A6A0000000092
:10518C00000000008A864CECB0F000006FECB0F030
:10519C000000100E816E100E816E36EC91F0100E28
:1051AC00816E4CECB0F0000000008A6AC7ECB8F0DD
:1051BC00100E816E9CEC91F0100E816E080E816EBB
:1051CC006FECB0F0000051ECB0F08A6A0000000007
:1051DC00000000008A88A1ECB0F08A4251ECB0F0DB
:1051EC00100E816EF6EC7CF08A42BEECB0F08A6A4E
:1051FC006AECB0F000008A86BEECB0F0100E816E46
:10520C0093EC7CF08A4251ECB0F08A46A1ECB0F001
:10521C008A6A00000000000000008A864CECB0F0A6
:10522C00000000006FECB0F00000100E816E100E4C
:10523C00816E36EC91F0100E816E4CECB0F00000EB
:10524C0000008A6AC7ECB8F0100E816E9CEC91F0ED
:10525C00100E816E080E816E6FECB0F0000051ECF8
:10526C00B0F000008A6A00000000000000008A888C
:10527C00A1ECB0F08A424CECB0F000000000100E33
:10528C00816EF6EC7CF08A42BEECB0F08A6A6AEC75
:10529C00B0F000008A86BEECB0F0100E816E93EC7C
:1052AC007CF08A424CECB0F0000000008A46A1EC85
:1052BC00B0F08A6A00000000000000008A8651EC01
:1052CC00B0F06FECB0F00000100E816E100E816E1D
:1052DC0036EC91F0100E816E4CECB0F0000000003A
:1052EC008A6AC7ECB8F0100E816E9CEC91F0100E2F
:1052FC00816E080E816E6FECB0F000004CECB0F0DB
:10530C008A4600008A42000000008A6A0000000001
:10531C00000000008A88A1ECB0F08A424CECB0F09E
:10532C000000100E816EF6EC7CF08A42BEECB0F000
:10533C008A6A6AECB0F000008A86BEECB0F0100EFF
:10534C00816E93EC7CF08A424CECB0F000008A4603
:10535C00A1ECB0F08A6A00000000000000008A8610
:10536C00000000008A4600008A4245ECB0F06FEC69
:10537C00B0F00000100E816E100E816E36EC91F0C4
:10538C00100E816E4CECB0F0000000008A6AC7EC85
:10539C00B8F0100E816EB9EC91F0100E816E080E03
:1053AC00816E6FECB0F000004CECB0F08A4600005F
:1053BC008A420000000000008A6A00000000000021
:1053CC0000008A88A1ECB0F08A424CECB0F0100ED0
:1053DC00816EF6EC7CF08A42BEECB0F08A6A6AEC24
:1053EC00B0F000008A86BEECB0F0100E816E93EC2B
:1053FC007CF08A424CECB0F08A46A1ECB0F08A6AA0
:10540C0000000000000000008A8600000000000080
:10541C008A4600008A4245ECB0F06FECB0F0000018
:10542C00100E816E100E816E4FEC91F0100E816E8D
:10543C004CECB0F0000000008A6AC7ECB8F0100E1B
:10544C00816EB9EC91F0100E816E080E816E6FECCE
:10545C00B0F000004CECB0F08A4600008A4200002C
:10546C000000000000008A6AA1ECB0F08A88A1EC70
:10547C00B0F08A42C7ECB0F0100E816EF6EC7CF006
:10548C008A42BEECB0F08A6A6AECB0F000008A8600
:10549C00BEECB0F0100E816E93EC7CF08A42C7EC3F
:1054AC00B0F08A46A1ECB0F08A6AA1ECB0F08A8622
:1054BC0000000000000000008A4600008A4245EC13
:1054CC00B0F06FECB0F00000100E816E100E816E1B
:1054DC004FEC91F0100E816E4CECB0F0000000001F
:1054EC008A6AC7ECB8F0100E816EB9EC91F0100E10
:1054FC00816E080E816E6FECB0F000004CECB0F0D9
:10550C008A4600008A42A1ECB0F08A6AA1ECB0F0A5
:10551C008A88A1ECB0F08A42C2ECB0F0100E816E19
:10552C00F6EC7CF08A42BEECB0F08A6A6AECB0F021
:10553C0000008A86BEECB0F0100E816E93EC7CF00D
:10554C008A42C2ECB0F08A46A1ECB0F08A6AA1ECB7
:10555C00B0F08A86A1ECB0F08A4600008A4245EC95
:10556C00B0F06FECB0F00000100E816E100E816E7A
:10557C004FEC91F0100E816E4CECB0F0000000007E
:10558C008A6AC7ECB8F0100E816EB9EC91F0100E6F
:10559C00816E080E816E6FECB0F000004CECB0F038
:1055AC008A4600008A42B2ECB0F08A6AA1ECB0F0F4
:1055BC008A88A1ECB0F08A42BEECB0F0100E816E7D
:1055CC00F6EC7CF08A42BEECB0F08A6A6AECB0F081
:1055DC0000008A86BEECB0F0100E816E93EC7CF06D
:1055EC008A42BEECB0F08A46A1ECB0F08A6AA1EC1B
:1055FC00B0F08A86B2ECB0F08A4600008A4245ECE4
:10560C00B0F06FECB0F00000100E816E100E816ED9
:10561C004FEC91F0100E816E4CECB0F000000000DD
:10562C008A6AC7ECB8F0100E816EB9EC91F0100ECE
:10563C00816E080E816E6FECB0F000004CECB0F097
:10564C008A4600008A42BEECB0F08A6AB2ECB0F036
:10565C008A88A1ECB0F08A42A1ECB0F0100E816EF9
:10566C00F6EC7CF08A42BEECB0F08A6A6AECB0F0E0
:10567C0000008A86BEECB0F0100E816E93EC7CF0CC
:10568C008A42A1ECB0F08A46A1ECB0F08A6AB2EC86
:10569C00B0F08A86BEECB0F08A4600008A4245EC37
:1056AC00B0F06FECB0F00000100E816E100E816E39
:1056BC004FEC91F0100E816E4CECB0F0000000003D
:1056CC008A6AC7ECB8F0100E816EB9EC91F0100E2E
:1056DC00816E080E816E6FECB0F000004CECB0F0F7
:1056EC008A4600008A42C7ECB0F08A6AA1ECB0F09E
:1056FC008A88A1ECB0F08A42000000000000000093
:10570C00100E816EF6EC7CF08A42BEECB0F08A6A28
:10571C006AECB0F000008A86BEECB0F0100E816E20
:10572C0093EC7CF08A4200000000000000008A46E6
:10573C00A1ECB0F08A6AA1ECB0F08A86C7ECB0F0AC
:10574C008A4600008A4245ECB0F06FECB0F00000E5
:10575C00100E816E100E816E4FEC91F0100E816E5A
:10576C004CECB0F0000000008A6AC7ECB8F0000006
:10577C008A6A00005FEC91F0100E816E080E816E4B
:10578C006FECB0F000004CECB0F08A4600008A429E
:10579C0045ECB0F08A6AB2ECB0F08A88A1ECB0F0BB
:1057AC008A4200000000100E816EF6EC7CF08A42FA
:1057BC008DECB0F000000000100E816E93EC7CF0CC
:1057CC008A42000000008A46A1ECB0F08A6AB2EC72
:1057DC00B0F08A8645ECB0F08A4600008A4245EC6F
:1057EC00B0F06FECB0F00000100E816E100E816EF8
:1057FC0009EC91F0000000008A6A4CECB0F000005B
:10580C0000008A6AC7ECB8F000008A6A00005FECFE
:10581C0091F0100E816E080E816E6FECB0F00000EE
:10582C004CECB0F08A4600008A424CECB0F0000020
:10583C008A6AA1ECB0F08A88B2ECB0F08A42100E01
:10584C00816EF6EC7CF08A428DECB0F0000000002A
:10585C00100E816E93EC7CF08A428A46B2ECB0F06A
:10586C008A6AA1ECB0F08A864CECB0F000008A4653
:10587C0000008A4245ECB0F06FECB0F00000100E66
:10588C00816E100E816E09EC91F0000000008A6AA6
:10589C004CECB0F0000000008A6AC7ECB8F00000D5
:1058AC008A6A00005FEC91F0100E816E080E816E1A
:1058BC006FECB0F000004CECB0F08A4600008A426D
:1058CC004CECB0F0000000008A6AB2ECB0F08A88B0
:1058DC00A1ECB0F0100E816EF6EC7CF08A428DECEF
:1058EC00B0F000000000100E816E93EC7CF08A8802
:1058FC00A1ECB0F08A6AB2ECB0F08A864CECB0F055
:10590C00000000008A4600008A4245ECB0F06FECC3
:10591C00B0F00000100E816E100E816E09EC91F04B
:10592C00000000008A6A4CECB0F0000000008A6AAB
:10593C00C7ECB8F000008A6A00005FEC91F0100E22
:10594C00816E080E816E6FECB0F000004CECB0F084
:10595C008A4600008A4251ECB0F000008A6AB2EC30
:10596C00B0F08A88000000000000100E816EF6EC8A
:10597C007CF08A428DECB0F000000000100E816EBD
:10598C0093EC7CF08A880000000000008A6AB2EC7C
:10599C00B0F08A8651ECB0F000008A4600008A42D2
:1059AC0045ECB0F06FECB0F00000100E816E100EF4
:1059BC00816E09EC91F0000000008A6A4CECB0F0AA
:1059CC00000000008A6AC7ECB8F000008A6A000088
:1059DC005FEC91F0100E816E080E816E6FECB0F0E2
:1059EC0000004CECB0F08A4600008A4256ECB0F055
:1059FC008A6AB2ECB0F08A880000100E816EF6EC68
:105A0C007CF08A428DECB0F000000000100E816E2C
:105A1C0093EC7CF08A8800008A6AB2ECB0F08A863B
:105A2C0056ECB0F08A4600008A4245ECB0F06FECC0
:105A3C00B0F00000100E816E100E816E09EC91F02A
:105A4C00000000008A6A4CECB0F0000000008A6A8A
:105A5C00C7ECB8F000008A6A00005FEC91F0100E01
:105A6C00816E080E816E6FECB0F000004CECB0F063
:105A7C008A4600008A4256ECB0F0000000008A6AA8
:105A8C00B2ECB0F0100E816E7EECB0F000008A42E9
:105A9C008DECB0F000000000100E816E7EECB0F0CA
:105AAC0000008A6AB2ECB0F08A8656ECB0F00000C6
:105ABC0000008A4600008A4245ECB0F06FECB0F072
:105ACC000000100E816E100E816E09EC91F000003A
:105ADC0000008A6A4CECB0F0000000008A6AC7EC47
:105AEC00B8F000008A6A4CECB0F000000000100E18
:105AFC00816E97ECB0F00000000000008DECB0F06F
:105B0C00100E816E6FECB0F000007EECB0F08A6A83
:105B1C00B2ECB0F08A88BEECB0F08A4297ECB0F0F0
:105B2C0000000000000097ECB0F0000000008A4676
:105B3C00BEECB0F08A6AB2ECB0F08A885BECB0F0E4
:105B4C0051ECB0F06FECB0F00000100E816E97ECE1
:105B5C00B0F00000000000008DECB0F00000000080
:105B6C0000008A6A4CECB0F0000000008A6AC7ECB6
:105B7C00B8F000008A6A000085EC91F0100E816E7E
:105B8C00080E816E6FECB0F000004CECB0F08A4661
:105B9C0000008A4265ECB0F08A6ABEECB0F08A88EC
:105BAC00BEECB0F08A4297ECB0F0000000000000B0
:105BBC008DECB0F0000000008A46BEECB0F08A6AB2
:105BCC00BEECB0F08A8665ECB0F08A4600008A42E2
:105BDC0045ECB0F06FECB0F00000100E816E080ECA
:105BEC00816E27EC91F0000000008A6A4CECB0F05A
:105BFC00000000008A6AC7ECB8F000008A6A000056
:105C0C0085EC91F0100E816E080E816E6FECB0F089
:105C1C0000004CECB0F08A4600008A4265ECB0F013
:105C2C00000000008A6ABEECB0F08A88C2ECB0F0CA
:105C3C008A4297ECB0F00000000000007EECB0F05F
:105C4C00000000008A46C2ECB0F08A6ABEECB0F0EC
:105C5C008A8665ECB0F0000000008A4600008A429B
:105C6C0045ECB0F06FECB0F00000100E816E080E39
:105C7C00816E27EC91F0000000008A6A4CECB0F0C9
:105C8C00000000008A6AC7ECB8F000008A6A0000C5
:105C9C0085EC91F0100E816E080E816E6FECB0F0F9
:105CAC0000004CECB0F08A4600008A426AECB0F07E
:105CBC0000008A6AC2ECB0F08A88C2ECB0F08A426A
:105CCC0097ECB0F00000000000006FECB0F00000AA
:105CDC0000008A46C2ECB0F08A6AC2ECB0F08A8648
:105CEC006AECB0F000008A4600008A4245ECB0F045
:105CFC006FECB0F00000100E816E080E816E27EC78
:105D0C0091F0000000008A6A4CECB0F0000000003A
:105D1C008A6AC7ECB8F000008A6A000085EC91F042
:105D2C00100E816E080E816E6FECB0F000004CEC22
:105D3C00B0F08A4600008A426FECB0F000008A6A2C
:105D4C00C2ECB0F08A88C7ECB0F08A4297ECB0F0A5
:105D5C0000000000000065ECB0F08A46C7ECB0F023
:105D6C008A6AC2ECB0F08A866FECB0F000008A460A
:105D7C0000008A4245ECB0F06FECB0F00000100E61
:105D8C00816E080E816E27EC91F0000000008A6A8B
:105D9C004CECB0F0000000008A6AC7ECB8F00000D0
:105DAC008A6A000085EC91F0100E816E080E816EEF
:105DBC006FECB0F000004CECB0F08A4600008A4268
:105DCC0079ECB0F000008A6AC2ECB0F08A8845EC3D
:105DDC00B0F08A4297ECB0F000000000000051ECEB
:105DEC00B0F000008A4645ECB0F08A6AC2ECB0F024
:105DFC008A8679ECB0F000008A4600008A4245ECB5
:105E0C00B0F06FECB0F00000100E816E080E816ED9
:105E1C0027EC91F0000000008A6A4CECB0F0000016
:105E2C0000008A6AC7ECB8F0100E816E000085EC99
:105E3C0091F0100E816E080E816E6FECB0F00000C8
:105E4C004CECB0F08A4600008A427EECB0F00000C8
:105E5C008A6AC7ECB0F08A884CECB0F000008A4239
:105E6C0097ECB0F000000000000000000000000003
:105E7C008A464CECB0F000008A6AC7ECB0F08A8617
:105E8C007EECB0F000008A4600008A4245ECB0F08F
:105E9C006FECB0F00000100E816E080E816E27ECD6
:105EAC0091F00000100E816E4CECB0F00000000080
:105EBC008A6AC7ECB8F0100E816E000085EC91F088
:105ECC00100E816E080E816E6FECB0F000004CEC81
:105EDC00B0F08A4600008A4283ECB0F000008A6A77
:105EEC0045ECB0F08A8851ECB0F08A428DECB0F001
:105EFC008A4651ECB0F08A6A45ECB0F08A8683ECA5
:105F0C00B0F000008A4600008A4245ECB0F06FEC1D
:105F1C00B0F00000100E816E080E816E27EC91F02F
:105F2C000000100E816E4CECB0F0000000008A6A8C
:105F3C00C7ECB8F0100E816E76EC91F0100E816EFD
:105F4C00080E816E51ECB0F00000100E816E000056
:105F5C000000080E816E56ECB0F000000000100E30
:105F6C00816E080E816E6FECB0F000004CECB0F05E
:105F7C008A4600008A428DECB0F0000000008A6A6C
:105F8C004CECB0F08A885BECB0F08A4256ECB0F086
:105F9C00000000008A465BECB0F08A6A4CECB0F072
:105FAC008A868DECB0F0000000008A4600008A4220
:105FBC0045ECB0F06FECB0F00000100E816E080EE6
:105FCC00816E5BECB0F00000100E816E00000000E2
:105FDC00080E816E4CECB0F000000000100E816ECB
:105FEC00080E816E18EC91F000008A6AC7ECB8F0CC
:105FFC00100E816E76EC91F0100E816E080E816E93
:10600C004CECB0F00000100E816E7CECBAF0100E6F
:10601C00816E080E816E51ECB0F000000000100E85
:10602C00816E080E816E6FECB0F000004CECB0F09D
:10603C008A4600008A428DECB0F08A4600008A4203
:10604C000000000000008A6A51ECB0F08A8897ECDE
:10605C00B0F08A6A51ECB0F08A86000000000000B3
:10606C008A4600008A428DECB0F08A4600008A42D3
:10607C0045ECB0F06FECB0F00000100E816E080E25
:10608C00816E56ECB0F0000000008A46100E816E56
:10609C005EECBBF0080E816E45ECB0F0100E816E1C
:1060AC00080E816E18EC91F000008A6AC7ECB8F00B
:1060BC00100E816E76EC91F0100E816E080E816ED2
:1060CC0045ECB0F0100E816E75ECBAF0100E816ECE
:1060DC00080E816E51ECB0F0100E816E080E816EC0
:1060EC006FECB0F000004CECB0F08A4600008A4235
:1060FC008DECB0F08A4600008A42C2ECB0F08A6A9D
:10610C0056ECB0F08A886FECB0F0000000008A6AA0
:10611C0056ECB0F08A86C2ECB0F08A4600008A4297
:10612C008DECB0F08A4600008A4245ECB0F06FEC82
:10613C00B0F00000100E816E080E816E56ECB0F0BF
:10614C008A46100E816E57ECBBF0080E816EC2ECC5
:10615C00B0F0100E816E080E816E18EC91F00000FC
:10616C008A6AC7ECB8F0100E816E76EC91F0100EC6
:10617C00816E080E816EC2ECB0F0100E816E70EC68
:10618C00BAF0100E816E080E816E4CECB0F000006F
:10619C00100E816E080E816E6FECB0F000004CECAE
:1061AC00B0F08A4600008A428DECB0F08A460000BE
:1061BC008A424CECB0F0000000008A6A97ECB0F018
:1061CC00000000000000BEECB0F08A864CECB0F091
:1061DC00000000008A4600008A428DECB0F08A462E
:1061EC0000008A4245ECB0F06FECB0F00000100EED
:1061FC00816E080E816E51ECB0F000008A46100ED4
:10620C00816E52ECBBF0080E816EB2ECB0F0100E49
:10621C00816E080E816E18EC91F000008A6AC7EC52
:10622C00B8F0100E816E76EC91F0100E816E080EA7
:10623C00816EB2ECB0F0100E816E67ECBAF0100EFD
:10624C00816E080E816E45ECB0F0100E816E080E5A
:10625C00816E6FECB0F000004CECB0F08A460000A0
:10626C008A428DECB0F08A4600008A425BECB0F0BA
:10627C008A6A8DECB0F0000000008A865BECB0F00E
:10628C008A4600008A428DECB0F08A4600008A42B1
:10629C0045ECB0F06FECB0F00000100E816E080E03
:1062AC00816E4CECB0F0000000008A46100E816E3E
:1062BC0049ECBBF0080E816E0000000000000000ED
:1062CC00100E816E080E816E18EC91F000008A6A37
:1062DC00C7ECB8F0100E816E76EC91F0100E816E5A
:1062EC00080E816E0000000000000000100E816E90
:1062FC005AECBAF0100E816E080E816EC2ECB0F042
:10630C00100E816E080E816E6FECB0F000004CEC3C
:10631C00B0F08A4600008A428DECB0F08A4600004C
:10632C008A426FECB0F0000000008A6A5BECB0F0BF
:10633C0000008A866FECB0F0000000008A46000076
:10634C008A428DECB0F08A4600008A4245ECB0F0EF
:10635C006FECB0F00000100E816E080E816E4CECEC
:10636C00B0F08A46100E816E3CECBBF0080E816ECC
:10637C0000000000100E816E080E816E18EC91F07A
:10638C0000008A6AC7ECB8F0100E816E76EC91F0C2
:10639C00100E816E080E816E00000000100E816ED2
:1063AC0055ECBAF0100E816E080E816EB2ECB0F0A6
:1063BC00100E816E080E816E01EC7EF0100E816E57
:1063CC00080E816EC7ECB0F08A46100E816E37EC69
:1063DC00BBF0080E816E100E816E080E816E18ECEB
:1063EC0091F000008A6AC7ECB8F0100E816E76EC62
:1063FC0091F0100E816E080E816E100E816E4CECB9
:10640C00BAF0100E816E080E816E000000000000C4
:10641C000000100E816E080E816E01EC7EF0100EE5
:10642C00816E080E816EBEECB0F08A46100E816E45
:10643C002EECBBF0100E816E080E816E18EC91F0F4
:10644C0000008A6AC7ECB8F0100E816E76EC91F001
:10645C00100E816E100E816E3FECBAF0100E816E34
:10646C00080E816E00000000100E816E080E816E09
:10647C0001EC7EF0100E816E080E816EA1ECB0F076
:10648C008A46100E816E21ECBBF0080E816E18EC62
:10649C0091F000008A6AC7ECB8F0100E816E76ECB1
:1064AC0091F0100E816E34ECBAF0100E816E080E65
:1064BC00816E100E816E080E816E01EC7EF0100E56
:1064CC00816E080E816E0000000000008A46100EDE
:1064DC00816E16ECBBF0080E816E83ECB0F0100EE2
:1064EC00816E080E816E000000000000100E816E9F
:1064FC004CECB0F0000000008A6AE6EC91F0000071
:10650C00000075ECB5F030EF00F048ECAEF00E5337
:10651C00D8A438EF4BF00000E0ECA6F000008A6A3B
:10652C00C7ECB8F0100E816E76EC91F0100E816E07
:10653C0034ECBAF0100E816E080E816E100E816E66
:10654C00080E816E01EC7EF0100E816E080E816ECD
:10655C000000000000008A46100E816E16ECBBF0A5
:10656C00080E816E83ECB0F0100E816E080E816EF9
:10657C00000000000000100E816E4CECB0F000002A
:10658C0000008A6AC7ECB8F0100E816E76EC91F0C0
:10659C00100E816E100E816E3FECBAF0100E816EF3
:1065AC00080E816E00000000100E816E080E816EC8
:1065BC0001EC7EF0100E816E080E816EA1ECB0F035
:1065CC008A46100E816E21ECBBF0080E816E18EC21
:1065DC0091F000008A6AC7ECB8F0100E816E76EC70
:1065EC0091F0100E816E080E816E100E816E4CECC7
:1065FC00BAF0100E816E080E816E000000000000D3
:10660C000000100E816E080E816E01EC7EF0100EF3
:10661C00816E080E816EBEECB0F08A46100E816E53
:10662C002EECBBF0100E816E080E816E18EC91F002
:10663C0000008A6AC7ECB8F0100E816E76EC91F00F
:10664C00100E816E080E816E00000000100E816E1F
:10665C0055ECBAF0100E816E080E816EB2ECB0F0F3
:10666C00100E816E080E816E01EC7EF0100E816EA4
:10667C00080E816EC7ECB0F08A46100E816E37ECB6
:10668C00BBF0080E816E100E816E080E816E18EC38
:10669C0091F000008A6AC7ECB8F0100E816E76ECAF
:1066AC0091F0100E816E080E816E0000000000004B
:1066BC000000100E816E5AECBAF0100E816E080EAE
:1066CC00816EC2ECB0F0100E816E080E816E83EC00
:1066DC00B0F000000000100E816E080E816E83EC8D
:1066EC00B0F000000000100E816E080E816E92EC6E
:1066FC00B0F083ECB0F000000000100E816E080EBC
:10670C00816E83ECB0F000000000100E816E080E5C
:10671C00816E83ECB0F000000000100E816E080E4C
:10672C00816E4CECB0F08A46100E816E3CECBBF0E6
:10673C00080E816E00000000100E816E080E816E36
:10674C0018EC91F000008A6AC7ECB8F0100E816E5C
:10675C0076EC91F0100E816E080E816EB2ECB0F0FA
:10676C00100E816E67ECBAF0100E816E080E816E01
:10677C0045ECB0F0100E816E080E816E6FECB0F02F
:10678C0000004CECB0F08A4600008A428DECB0F070
:10679C008A4600008A426FECB0F0000000008A6A62
:1067AC005BECB0F000008A866FECB0F000000000EB
:1067BC008A4600008A428DECB0F08A4600008A427C
:1067CC0045ECB0F06FECB0F00000100E816E080ECE
:1067DC00816E4CECB0F0000000008A46100E816E09
:1067EC0049ECBBF0080E816E0000000000000000B8
:1067FC00100E816E080E816E18EC91F000008A6A02
:10680C00C7ECB8F0100E816E76EC91F0100E816E24
:10681C00080E816EC2ECB0F0100E816E70ECBAF006
:10682C00100E816E080E816E4CECB0F00000100E54
:10683C00816E080E816E6FECB0F000004CECB0F085
:10684C008A4600008A428DECB0F08A4600008A42EB
:10685C0056ECB0F0000000008A6A92ECB0F0000038
:10686C008A8656ECB0F0000000008A4600008A428E
:10687C008DECB0F08A4600008A4245ECB0F06FEC2B
:10688C00B0F00000100E816E080E816E51ECB0F06D
:10689C0000008A46100E816E52ECBBF0080E816E21
:1068AC00B2ECB0F0100E816E080E816E18EC91F007
:1068BC0000008A6AC7ECB8F0100E816E76EC91F08D
:1068CC00100E816E080E816E45ECB0F0100E816ECC
:1068DC0075ECBAF0100E816E080E816E51ECB0F0B2
:1068EC00100E816E080E816E6FECB0F000004CEC57
:1068FC00B0F08A4600008A428DECB0F08A46000067
:10690C008A424CECB0F08A6A97ECB0F000000000C0
:10691C0000004CECB0F08A864CECB0F08A460000DB
:10692C008A428DECB0F08A4600008A4245ECB0F009
:10693C006FECB0F00000100E816E080E816E56ECFC
:10694C00B0F08A46100E816E57ECBBF0080E816ECB
:10695C00C2ECB0F0100E816E080E816E18EC91F046
:10696C0000008A6AC7ECB8F0100E816E76EC91F0DC
:10697C00100E816E080E816E4CECB0F00000100E03
:10698C00816E7CECBAF0100E816E080E816E51ECAB
:10699C00B0F000000000100E816E080E816E6FECDE
:1069AC00B0F000004CECB0F08A4600008A4297EC44
:1069BC00B0F00000000000008A6A56ECB0F08A8843
:1069CC007EECB0F08A6A56ECB0F08A8697ECB0F0A8
:1069DC000000000000008A4600008A4245ECB0F03E
:1069EC006FECB0F00000100E816E080E816E56EC4C
:1069FC00B0F0000000008A46100E816E5EECBBF019
:106A0C00080E816E45ECB0F0100E816E080E816E92
:106A1C0018EC91F000008A6AC7ECB8F0100E816E89
:106A2C0076EC91F0100E816E080E816E51ECB0F088
:106A3C000000100E816E00000000080E816E56ECF6
:106A4C00B0F000000000100E816E080E816E6FEC2D
:106A5C00B0F000004CECB0F08A4600008A4292EC98
:106A6C00B0F000008A6A4CECB0F0000000008A889C
:106A7C00000097ECB0F000000000000000000000E7
:106A8C008A6A4CECB0F0000000008A8692ECB0F000
:106A9C0000008A4600008A4245ECB0F06FECB0F082
:106AAC000000100E816E080E816E5BECB0F00000E1
:106ABC00100E816E00000000080E816E4CECB0F0E0
:106ACC0000000000100E816E080E816E18EC91F023
:106ADC0000008A6AC7ECB8F0100E816E76EC91F06B
:106AEC00100E816E080E816E83ECB0F00000000079
:106AFC00100E816E080E816E6FECB0F000004CEC45
:106B0C00B0F08A4600008A428DECB0F08A6A4CECF8
:106B1C00B0F000008A885BECB0F0000000008A4204
:106B2C0056ECB0F08A465BECB0F0000000008A6ACC
:106B3C004CECB0F000008A868DECB0F08A46000078
:106B4C008A4245ECB0F06FECB0F00000100E816E94
:106B5C00080E816E83ECB0F000000000100E816E08
:106B6C00080E816E18EC91F000008A6AC7ECB8F040
:106B7C00100E816E76EC91F0100E816E080E816E07
:106B8C0083ECB0F000000000100E816E080E816ED8
:106B9C006FECB0F000004CECB0F08A4600008A427A
:106BAC007EECB0F0000000008A6A45ECB0F08A88F8
:106BBC0051ECB0F0000000008A428DECB0F08A4637
:106BCC0051ECB0F0000000008A6A45ECB0F08A8607
:106BDC007EECB0F0000000008A4600008A4245ECD2
:106BEC00B0F06FECB0F00000100E816E080E816EEC
:106BFC0083ECB0F000000000100E816E080E816E68
:106C0C0083ECB0F000000000100E816E080E816E57
:106C1C00000000000000100E816E4CECB0F0000083
:106C2C0000008A6AC7ECB8F000008A6A000085ECA4
:106C3C0091F0100E816E080E816E6FECB0F00000BA
:106C4C004CECB0F08A4600008A4279ECB0F00000BF
:106C5C008A6A45ECB0F08A884CECB0F00000000079
:106C6C008A4297ECB0F0000000000000A1ECB0F0FC
:106C7C008A464CECB0F0000000008A6A45ECB0F09B
:106C8C008A8679ECB0F000008A4600008A4245EC16
:106C9C00B0F06FECB0F00000100E816E080E816E3B
:106CAC0027EC91F0000000008A6A4CECB0F0000078
:106CBC0000008A6AC7ECB8F000008A6A000085EC14
:106CCC0091F0100E816E080E816E6FECB0F000002A
:106CDC004CECB0F08A4600008A426FECB0F0000039
:106CEC008A6AC7ECB0F08A884CECB0F08A4297EC18
:106CFC00B0F000000000000056ECB0F08A464CECFE
:106D0C00B0F08A6AC7ECB0F08A866FECB0F0000085
:106D1C008A4600008A4245ECB0F06FECB0F00000FF
:106D2C00100E816E080E816E27EC91F000000000B1
:106D3C008A6A4CECB0F0000000008A6AC7ECB8F02C
:106D4C0000008A6A000085EC91F0100E816E080E2E
:106D5C00816E6FECB0F000004CECB0F08A46000095
:106D6C008A426AECB0F000008A6AC2ECB0F08A8801
:106D7C0045ECB0F08A4297ECB0F000000000000047
:106D8C006AECB0F000008A4645ECB0F08A6AC2ECBE
:106D9C00B0F08A866AECB0F000008A4600008A42A5
:106DAC0045ECB0F06FECB0F00000100E816E080EE8
:106DBC00816E27EC91F0000000008A6A4CECB0F078
:106DCC00000000008A6AC7ECB8F000008A6A000074
:106DDC0085EC91F0100E816E080E816E6FECB0F0A8
:106DEC0000004CECB0F08A4600008A4265ECB0F032
:106DFC00000000008A6ABEECB0F08A8845ECB0F066
:106E0C008A4297ECB0F000000000000079ECB0F082
:106E1C0000008A4645ECB0F08A6ABEECB0F08A8677
:106E2C0065ECB0F0000000008A4600008A4245EC98
:106E3C00B0F06FECB0F00000100E816E080E816E99
:106E4C0027EC91F0000000008A6A4CECB0F00000D6
:106E5C0000008A6AC7ECB8F000008A6A000085EC72
:106E6C0091F0100E816E080E816E6FECB0F0000088
:106E7C004CECB0F08A4600008A425BECB0F00000AB
:106E8C0000008A6AC2ECB0F08A88C2ECB0F08A4288
:106E9C0097ECB0F00000000000008DECB0F08A46DA
:106EAC00C2ECB0F08A6AC2ECB0F08A865BECB0F04F
:106EBC00000000008A4600008A4245ECB0F06FECFE
:106ECC00B0F00000100E816E080E816E27EC91F070
:106EDC00000000008A6A4CECB0F0000000008A6AE6
:106EEC00C7ECB8F000008A6A000085EC91F0100E37
:106EFC00816E080E816E6FECB0F000004CECB0F0BF
:106F0C008A4600008A425BECB0F08A6AA1ECB0F0D1
:106F1C008A6A00008A88000079ECB0F0000000005A
:106F2C008A426AECB0F00000000051ECB0F00000B6
:106F3C00100E816E79ECB0F0000000008A6A00003F
:106F4C008A6AA1ECB0F08A865BECB0F08A4600004D
:106F5C008A4245ECB0F06FECB0F00000100E816E80
:106F6C00080E816E27EC91F0000000008A6A4CEC50
:106F7C00B0F0000000008A6AC7ECB8F000008A6A22
:106F8C004CECB0F000000000100E816ECDECB0F0B7
:106F9C000000000065ECB0F056ECB0F04CECB0F03A
:106FAC0000008A42000000008A6AB2ECB0F08A88C5
:106FBC00100E816E93EC7CF08A426AECB0F000000B
:106FCC00000051ECB0F00000100E816EF6EC7CF07D
:106FDC008A888A6AB2ECB0F08A86000000008A4681
:106FEC004CECB0F0000051ECB0F000000000CDEC27
:106FFC00B0F00000000065ECB0F0000000000000F4
:10700C008A6A4CECB0F0000000008A6AC7ECB8F059
:10701C0000008A6A00005FEC91F0100E816E080E81
:10702C00816E6FECB0F000004CECB0F08A460000C2
:10703C008A4251ECB0F000008A6ABEECB0F08A884B
:10704C0000000000100E816E93EC7CF08A426AEC1A
:10705C00B0F00000000051ECB0F00000100E816E9A
:10706C00F6EC7CF08A88000000008A6ABEECB0F076
:10707C008A8651ECB0F000008A4600008A4245EC4A
:10708C00B0F06FECB0F00000100E816E100E816E3F
:10709C0009EC91F0000000008A6A4CECB0F00000A2
:1070AC0000008A6AC7ECB8F000008A6A00005FEC46
:1070BC0091F0100E816E080E816E6FECB0F0000036
:1070CC004CECB0F08A4600008A424CECB0F0000068
:1070DC0000008A6ABEECB0F08A8800000000000054
:1070EC000000100E816E93EC7CF08A426AECB0F0DA
:1070FC000000000051ECB0F00000100E816EF6ECB8
:10710C007CF08A8800000000000000008A6ABEEC57
:10711C00B0F08A864CECB0F0000000008A4600000B
:10712C008A4245ECB0F06FECB0F00000100E816EAE
:10713C00100E816E09EC91F0000000008A6A4CEC94
:10714C00B0F0000000008A6AC7ECB8F000008A6A50
:10715C0000005FEC91F0100E816E080E816E6FECEA
:10716C00B0F000004CECB0F08A4600008A424CECC7
:10717C00B0F000008A6AB2ECB0F08A88B2ECB0F0E1
:10718C00100E816E93EC7CF08A426AECB0F0000039
:10719C00000051ECB0F00000100E816EF6EC7CF0AB
:1071AC008A88B2ECB0F08A6AB2ECB0F08A864CEC09
:1071BC00B0F000008A4600008A4245ECB0F06FEC5B
:1071CC00B0F00000100E816E100E816E09EC91F083
:1071DC00000000008A6A4CECB0F0000000008A6AE3
:1071EC00C7ECB8F000008A6A00005FEC91F0100E5A
:1071FC00816E080E816E6FECB0F000004CECB0F0BC
:10720C008A4600008A4245ECB0F08A6AB2ECB0F0D3
:10721C008A88B2ECB0F08A420000100E816E93ECBA
:10722C007CF08A426AECB0F00000000051ECB0F047
:10723C000000100E816EF6EC7CF08A4200008A464B
:10724C00B2ECB0F08A6AB2ECB0F08A8645ECB0F0E1
:10725C008A4600008A4245ECB0F06FECB0F00000BA
:10726C00100E816E100E816E09EC91F00000000082
:10727C008A6A4CECB0F0000000008A6AC7ECB8F0E7
:10728C0000008A6A00005FEC91F0100E816E080E0F
:10729C00816E6FECB0F000004CECB0F08A46000050
:1072AC008A42C2ECB0F08A6AB2ECB0F08A88B2ECD6
:1072BC00B0F08A42000000000000100E816E93ECCA
:1072CC007CF08A426AECB0F00000000051ECB0F0A7
:1072DC000000100E816EF6EC7CF08A42000000007B
:1072EC0000008A46B2ECB0F08A6AB2ECB0F08A8642
:1072FC00C2ECB0F08A4600008A4245ECB0F06FEC6C
:10730C00B0F00000100E816E100E816E09EC91F041
:10731C00000000008A6A4CECB0F0000000008A6AA1
:10732C00C7ECB8F0100E816E00005FEC91F0100EFF
:10733C00816E080E816E6FECB0F000004CECB0F07A
:10734C008A4600008A42B2ECB0F08A6AB2ECB0F025
:10735C008A88B2ECB0F08A42A1ECB0F0100E816ECB
:10736C0093EC7CF08A42BEECB0F08A466AECB0F04A
:10737C0000008A42BEECB0F0100E816EF6EC7CF090
:10738C008A42A1ECB0F08A46B2ECB0F08A6AB2EC58
:10739C00B0F08A86B2ECB0F08A4600008A4245EC26
:1073AC00B0F06FECB0F00000100E816E100E816E1C
:1073BC0009EC91F00000100E816E4CECB0F0000066
:1073CC0000008A6AC7ECB8F0100E816E00005FEC0A
:1073DC0091F0100E816E080E816E6FECB0F0000013
:1073EC004CECB0F08A4600008A42A1ECB0F08A6AFC
:1073FC00A1ECB0F08A88B2ECB0F08A42BEECB0F0EE
:10740C00100E816E93EC7CF08A42BEECB0F08A4692
:10741C006AECB0F000008A42BEECB0F0100E816E47
:10742C00F6EC7CF08A42BEECB0F08A46B2ECB0F0DE
:10743C008A6AA1ECB0F08A86A1ECB0F08A46000012
:10744C008A4245ECB0F06FECB0F00000100E816E8B
:10745C00100E816E09EC91F00000100E816E4CEC58
:10746C00B0F0000000008A6AC7ECB8F0100E816E14
:10747C0000005FEC91F0100E816E080E816E6FECC7
:10748C00B0F000004CECB0F08A4600008A420000DC
:10749C000000000000008A6AA1ECB0F08A88A1EC20
:1074AC00B0F08A42C7ECB0F0100E816E93EC7CF019
:1074BC008A42BEECB0F08A466AECB0F000008A4218
:1074CC00BEECB0F0100E816EF6EC7CF08A42C7EC8C
:1074DC00B0F08A46A1ECB0F08A6AA1ECB0F08A86D2
:1074EC0000000000000000008A4600008A4245ECC3
:1074FC00B0F06FECB0F00000100E816E100E816ECB
:10750C0009EC91F00000100E816E4CECB0F0000014
:10751C0000008A6AC7ECB8F0100E816E00005FECB8
:10752C0091F0100E816E080E816E6FECB0F00000C1
:10753C004CECB0F08A4600008A42000000008A6AD7
:10754C00A1ECB0F08A88B2ECB0F08A4245ECB0F015
:10755C00100E816E93EC7CF08A42BEECB0F08A4641
:10756C006AECB0F000008A42BEECB0F0100E816EF6
:10757C00F6EC7CF08A4245ECB0F08A46B2ECB0F006
:10758C008A6AA1ECB0F08A86000000008A460000EE
:10759C008A4245ECB0F06FECB0F00000100E816E3A
:1075AC00100E816E09EC91F00000100E816E4CEC07
:1075BC00B0F0000000008A6AC7ECB8F0100E816EC3
:1075CC0000005FEC91F0100E816E080E816E6FEC76
:1075DC00B0F0000051ECB0F000008A6AA1ECB0F001
:1075EC008A88A1ECB0F08A424CECB0F00000100E8E
:1075FC00816E93EC7CF08A42BEECB0F08A466AEC69
:10760C00B0F000008A42BEECB0F0100E816EF6ECC9
:10761C007CF08A424CECB0F000008A46A1ECB0F051
:10762C008A6AA1ECB0F08A8651ECB0F06FECB0F045
:10763C000000100E816E100E816E09EC91F00000AE
:10764C00100E816E4CECB0F0000000008A6AC7ECA2
:10765C00B8F0100E816E00005FEC91F0100E816E90
:10766C00080E816E6FECB0F0000051ECB0F08A6A3D
:10767C00A1ECB0F08A88A1ECB0F08A424CECB0F0EE
:10768C0000000000100E816E93EC7CF08A42BEEC80
:10769C00B0F08A466AECB0F000008A42BEECB0F062
:1076AC00100E816EF6EC7CF08A424CECB0F00000CF
:1076BC0000008A46A1ECB0F08A6AA1ECB0F08A8690
:1076CC004CECB0F0000000006FECB0F00000100EBD
:1076DC00816E100E816E09EC91F00000100E816E1F
:1076EC004CECB0F0000000008A6AC7ECB8F0100E49
:1076FC00816E9CEC91F0100E816E080E816E6FEC19
:10770C00B0F000004CECB0F0000000008A6A000001
:10771C000000000000008A88A1ECB0F08A4251EC15
:10772C00B0F00000100E816E93EC7CF08A42BEEC3F
:10773C00B0F08A466AECB0F000008A42BEECB0F0C1
:10774C00100E816EF6EC7CF08A4251ECB0F0000029
:10775C008A46A1ECB0F08A6A00000000000000002C
:10776C008A864CECB0F000006FECB0F00000100E0C
:10777C00816E100E816E36EC91F0100E816E4CEC19
:10778C00B0F0000000008A6AC7ECB8F0100E816EF1
:10779C009CEC91F0100E816E080E816E6FECB0F0C7
:1077AC0000004CECB0F000008A6A00000000000001
:1077BC0000008A88A1ECB0F08A4251ECB0F00000D5
:1077CC000000100E816E93EC7CF08A42BEECB0F09F
:1077DC008A466AECB0F000008A42BEECB0F0100EA3
:1077EC00816EF6EC7CF08A4251ECB0F000000000A7
:1077FC008A46A1ECB0F08A6A00000000000000008C
:10780C008A864CECB0F06FECB0F00000100E816E7C
:10781C00100E816E36EC91F0100E816E4CECB0F0C7
:10782C00000000008A6AC7ECB8F0100E816E9CEC68
:10783C0091F0100E816E080E816E6FECB0F00000AE
:10784C0045ECB0F08A6AA1ECB0F08A88A1ECB0F0FB
:10785C008A4256ECB0F0100E816E93EC7CF08A42AA
:10786C00BEECB0F08A466AECB0F000008A42BEEC86
:10787C00B0F0100E816EF6EC7CF08A4256ECB0F053
:10788C008A46A1ECB0F08A6AA1ECB0F08A86C7EC0B
:10789C00B0F06FECB0F00000100E816E100E816E27
:1078AC0036EC91F0100E816E4CECB0F00000000044
:1078BC008A6AC7ECB8F0100E816E9CEC91F0100E39
:1078CC00816E080E816E6FECB0F0000045ECB0F0EC
:1078DC008A6A00000000000000008A88A1ECB0F069
:1078EC008A4256ECB0F00000100E816E93EC7CF0E6
:1078FC008A42BEECB0F08A466AECB0F000008A42D4
:10790C00BEECB0F0100E816EF6EC7CF08A4256ECB8
:10791C00B0F000008A46A1ECB0F08A6A00000000CA
:10792C00000000008A86C7ECB0F06FECB0F00000ED
:10793C00100E816E100E816E36EC91F0100E816E71
:10794C004CECB0F0000000008A6AC7ECB8F0100EE6
:10795C00816E9CEC91F0100E816E080E816E6FECB6
:10796C00B0F00000C7ECB0F08A6A00000000000024
:10797C0000008A88A1ECB0F08A4256ECB0F000000E
:10798C000000100E816E93EC7CF08A42BEECB0F0DD
:10799C008A466AECB0F000008A42BEECB0F0100EE1
:1079AC00816EF6EC7CF08A4256ECB0F000000000E0
:1079BC008A46A1ECB0F08A6A0000000000000000CA
:1079CC008A86C2ECB0F06FECB0F00000100E816E45
:1079DC00100E816E36EC91F0100E816E4CECB0F006
:1079EC00000000008A6AC7ECB8F0100E816E9CECA7
:1079FC0091F0100E816E080E816E6FECB0F00000ED
:107A0C00C2ECB0F08A6A00000000000000008A8816
:107A1C00A1ECB0F08A425BECB0F0100E816E7EEC03
:107A2C00B0F000008A42BEECB0F08A466AECB0F0CE
:107A3C0000008A42BEECB0F0100E816E7EECB0F00D
:107A4C0000008A425BECB0F08A46A1ECB0F08A6A86
:107A5C0000000000000000008A86BEECB0F06FEC65
:107A6C00B0F00000100E816E100E816E36EC91F0AD
:107A7C00100E816E4CECB0F0000000008A6AC7EC6E
:107A8C00B8F000008A6A9CEC91F0100E816E080E22
:107A9C00816E5FEC80F0100E816E100E816E36ECF4
:107AAC0091F000008A6A4CECB0F0000000008A6A89
:107ABC00C7ECB8F000008A6A9CEC91F0100E816E55
:107ACC00080E816EF1EC7FF0100E816E100E816E3F
:107ADC0036EC91F000008A6A4CECB0F0000000002B
:107AEC008A6AC7ECB8F000008A6A9CEC91F0100E20
:107AFC00816E080E816EFFEC81F0100E816E100EFF
:107B0C00816E36EC91F000008A6A4CECB0F000000B
:107B1C0000008A6AC7ECB8F000008A6A9CEC91F00D
:107B2C00100E816E080E816EF0EC82F0100E816EDC
:107B3C00100E816E36EC91F000008A6A4CECB0F0BD
:107B4C00000000008A6AC7ECB8F000008A6A9CEC5E
:107B5C0091F0100E816E080E816EE9EC83F0100E20
:107B6C00816E100E816E36EC91F000008A6A4CEC3E
:107B7C00B0F0000000008A6AC7ECB8F000008A6A16
:107B8C009CEC91F0100E816E080E816EA3EC84F0CB
:107B9C00100E816E100E816E36EC91F000008A6A28
:107BAC004CECB0F0000000008A6AC7ECB8F00000A2
:107BBC008A6A4CECB0F000000000100E816E97EC5D
:107BCC00B0F000008A6A56ECB0F00000100E816E26
:107BDC0000008A6A56ECB0F00000100E816E100E98
:107BEC00816E63EC85F0100E816E100E816E56EC7A
:107BFC00B0F0000000008A6A100E816E56ECB0F0F6
:107C0C000000100E816E97ECB0F000000000000038
:107C1C008A6A4CECB0F0000000008A6AC7ECB8F03D
:107C2C0000008A6A9CEC91F0100E816E080E816E39
:107C3C0013EC86F0100E816E100E816E36EC91F006
:107C4C0000008A6A4CECB0F0000000008A6AC7ECB5
:107C5C00B8F000008A6A9CEC91F0100E816E080E50
:107C6C00816E9EEC85F0100E816E100E816E36ECDE
:107C7C0091F000008A6A4CECB0F0000000008A6AB7
:107C8C00C7ECB8F000008A6A9CEC91F0100E816E83
:107C9C00080E816EDAEC7EF0100E816E100E816E85
:107CAC0036EC91F000008A6A4CECB0F00000000059
:107CBC008A6AC7ECB8F000008A6A9CEC91F0100E4E
:107CCC00816E080E816E13EC7FF0100E816E100E1B
:107CDC00816E36EC91F000008A6A4CECB0F000003A
:107CEC0000008A6AC7ECB8F000008A6A9CEC91F03C
:107CFC00100E816E080E816E82EC7FF0100E816E7C
:107D0C00100E816E36EC91F000008A6A4CECB0F0EB
:107D1C00000000008A6AC7ECB8F0100E816E9CEC73
:107D2C0091F0100E816E080E816E61EC88F0100ED1
:107D3C00816E100E816E36EC91F0100E816E4CEC53
:107D4C00B0F0000000008A6AC7ECB8F0100E816E2B
:107D5C009CEC91F0100E816E080E816ED6EC88F0C2
:107D6C00100E816E100E816E36EC91F0100E816E3D
:107D7C004CECB0F0000000008A6AC7ECB8F0100EB2
:107D8C00816E9CEC91F0100E816E080E816ED6EC1B
:107D9C0088F0100E816E100E816E36EC91F0100E84
:107DAC00816E4CECB0F0000000008A6A020E0F6F7E
:107DBC000000000000008B9E97ECB0F0000000006B
:107DCC00000000008B8E97ECB0F00000000000006B
:107DDC00000003D08A6AC7ECB8F0100E816E9CECE0
:107DEC0091F0100E816E080E816E87EC89F0100EEA
:107DFC00816E100E816E36EC91F0100E816E45EC9A
:107E0C00B0F00F2FE7D700008A6AC7ECB8F0100E5D
:107E1C00816E9CEC91F0100E816E080E816EFBEC65
:107E2C0089F0100E816E100E816E36EC91F0100EF2
:107E3C00816E4CECB0F00000030E8A6A0F6F0000EC
:107E4C000000000000008B9E97ECB0F000000000DA
:107E5C00000000008B8E97ECB0F0000000000000DA
:107E6C00000003D08A6AC7ECB8F0100E816E9CEC4F
:107E7C0091F0100E816E080E816E71EC8AF0100E6E
:107E8C00816E100E816E36EC91F0100E816E45EC09
:107E9C00B0F00F2FE7D700008A6AC7ECB8F0100ECD
:107EAC00816E9CEC91F0100E816E080E816EC3EC0D
:107EBC0086F0100E816E100E816E36EC91F0100E65
:107ECC00816E4CECB0F0000000008A6AC7ECB8F090
:107EDC00100E816E9CEC91F0100E816E080E816E6E
:107EEC00C3EC86F0100E816E100E816E36EC91F0A4
:107EFC00100E816E4CECB0F0000000008A6AC7ECEA
:107F0C00B8F0100E816E9CEC91F0100E816E080E84
:107F1C00816EB0EC87F0100E816E100E816E36EC17
:107F2C0091F0100E816E4CECB0F0000000008A6AEB
:107F3C00C7ECB8F000008A6A9CEC91F0100E816ED0
:107F4C00080E816E42EC8DF0100E816E100E816E5B
:107F5C0036EC91F000008A6A4CECB0F000000000A6
:107F6C008A6AC7ECB8F000008A6A9CEC91F0100E9B
:107F7C00816E080E816E7DEC8DF0100E816E100EF0
:107F8C00816E36EC91F000008A6A4CECB0F0000087
:107F9C0000008A6AC7ECB8F000008A6A9CEC91F089
:107FAC00100E816E080E816EECEC8DF0100E816E51
:107FBC00100E816E36EC91F000008A6A4CECB0F039
:107FCC00000000008A6AC7ECB8F000008A6A9CECDA
:107FDC0091F0100E816E080E816E61EC8EF0100E19
:107FEC00816E100E816E36EC91F000008A6A4CECBA
:107FFC00B0F0000000008A6AC7ECB8F000008A6A92
:10800C009CEC91F0100E816E080E816ED6EC8EF009
:10801C00100E816E100E816E36EC91F000008A6AA3
:10802C004CECB0F0000000008A6AC7ECB8F000001D
:10803C008A6A9CEC91F0100E816E080E816E4FECEA
:10804C008FF0100E816E100E816E36EC91F00000E8
:10805C008A6A4CECB0F0000000008A6AC7ECB8F0F9
:10806C0000008A6A4CECB0F000000000100E816E2B
:10807C0097ECB0F000008A6A56ECB0F00000100EDD
:10808C00816E00008A6A56ECB0F00000100E816E12
:10809C00100E816ED1EC8FF0100E816E100E816E71
:1080AC0056ECB0F0000000008A6A100E816E56EC9F
:1080BC00B0F00000100E816E97ECB0F000000000E4
:1080CC0000008A6A4CECB0F0000000008A6AC7EC31
:1080DC00B8F000008A6A9CEC91F0100E816E080ECC
:1080EC00816E4EEC90F0100E816E100E816E36EC9F
:1080FC0091F000008A6A4CECB0F0000000008A6A33
:10810C00C7ECB8F000008A6A9CEC91F0100E816EFE
:10811C00080E816ECBEC90F0100E816E100E816EFD
:10812C0036EC91F000008A6A4CECB0F000000000D4
:10813C008A6AC7ECB8F000008A6A9CEC91F0100EC9
:10814C00816E080E816EDAEC8BF0100E816E100EC3
:10815C00816E36EC91F000008A6A4CECB0F00000B5
:10816C0000008A6AC7ECB8F000008A6A9CEC91F0B7
:10817C00100E816E080E816E18EC8CF0100E816E54
:10818C00100E816E36EC91F000008A6A4CECB0F067
:10819C00000000008A6AC7ECB8F000008A6A9CEC08
:1081AC0091F0100E816E080E816ECAEC8CF0100EE0
:1081BC00816E100E816E36EC91F000008A6A4CECE8
:1081CC00B0F0000000008A6AC7ECB8F0100E816EA7
:1081DC009CEC91F0100E816E080E816E6FECB0F07D
:1081EC000000BEECB0F08A6AA1ECB0F08A88000006
:1081FC000000000000008A425BECB0F00000100EA2
:10820C00816EF6EC7CF08A42BEECB0F08A6A6AECC5
:10821C00B0F000008A86BEECB0F0100E816E93ECCC
:10822C007CF08A425BECB0F000008A460000000053
:10823C00000000008A6AA1ECB0F08A86B2ECB0F0C3
:10824C006FECB0F00000100E816E100E816E36ECEB
:10825C0091F0100E816E4CECB0F0000000008A6AB8
:10826C00C7ECB8F0100E816E9CEC91F0100E816E84
:10827C00080E816E6FECB0F00000C2ECB0F08A6AB0
:10828C00A1ECB0F08A8800000000000000008A42D7
:10829C005BECB0F0100E816EF6EC7CF08A42BEEC1A
:1082AC00B0F08A6A6AECB0F000008A86BEECB0F0DE
:1082BC00100E816E93EC7CF08A425BECB0F08A4637
:1082CC0000000000000000008A6AA1ECB0F08A8671
:1082DC00BEECB0F06FECB0F00000100E816E100E22
:1082EC00816E36EC91F0100E816E4CECB0F000000B
:1082FC0000008A6AC7ECB8F0100E816E9CEC91F00D
:10830C00100E816E080E816E6FECB0F00000C7ECA1
:10831C00B0F08A6AA1ECB0F08A880000000000007E
:10832C0000008A4256ECB0F000000000100E816E86
:10833C00F6EC7CF08A42BEECB0F08A6A6AECB0F0E3
:10834C0000008A86BEECB0F0100E816E93EC7CF0CF
:10835C008A4256ECB0F0000000008A460000000093
:10836C00000000008A6AA1ECB0F08A86C2ECB0F082
:10837C006FECB0F00000100E816E100E816E36ECBA
:10838C0091F0100E816E4CECB0F0000000008A6A87
:10839C00C7ECB8F0100E816E9CEC91F0100E816E53
:1083AC00080E816E6FECB0F0000045ECB0F08A6AFC
:1083BC00A1ECB0F08A8800000000000000008A42A6
:1083CC0056ECB0F00000100E816EF6EC7CF08A4298
:1083DC00BEECB0F08A6A6AECB0F000008A86BEECA3
:1083EC00B0F0100E816E93EC7CF08A4256ECB0F03B
:1083FC0000008A4600000000000000008A6AA1EC20
:10840C00B0F08A86C7ECB0F06FECB0F00000100E44
:10841C00816E100E816E36EC91F0100E816E4CEC6C
:10842C00B0F0000000008A6AC7ECB8F0100E816E44
:10843C009CEC91F0100E816E080E816E6FECB0F01A
:10844C0000004CECB0F08A6AA1ECB0F08A88A1EC88
:10845C00B0F08A4251ECB0F000000000100E816EBA
:10846C00F6EC7CF08A42BEECB0F08A6A6AECB0F0B2
:10847C0000008A86BEECB0F0100E816E93EC7CF09E
:10848C008A4251ECB0F0000000008A46A1ECB0F03A
:10849C008A6AA1ECB0F08A8645ECB0F06FECB0F0D3
:1084AC000000100E816E100E816E36EC91F0100EE5
:1084BC00816E4CECB0F0000000008A6AC7ECB8F09A
:1084CC00100E816E9CEC91F0100E816E080E816E78
:1084DC006FECB0F000004CECB0F000008A6AA1EC3C
:1084EC00B0F08A88A1ECB0F08A4251ECB0F00000F8
:1084FC00100E816EF6EC7CF08A42BEECB0F08A6A0B
:10850C006AECB0F000008A86BEECB0F0100E816E02
:10851C0093EC7CF08A4251ECB0F000008A46A1EC5E
:10852C00B0F08A6AA1ECB0F08A864CECB0F06FEC3B
:10853C00B0F00000100E816E100E816E36EC91F0D2
:10854C00100E816E4CECB0F0000000008A6AC7EC93
:10855C00B8F0100E816EB9EC91F0100E816E080E11
:10856C00816E6FECB0F000004CECB0F0000000003D
:10857C008A6AA1ECB0F08A88A1ECB0F08A4251EC86
:10858C00B0F0100E816EF6EC7CF08A42BEECB0F0CE
:10859C008A6A6AECB0F000008A86BEECB0F0100E6D
:1085AC00816E93EC7CF08A4251ECB0F08A46A1ECDF
:1085BC00B0F08A6AA1ECB0F08A864CECB0F0000006
:1085CC006FECB0F00000100E816E100E816E4FEC4F
:1085DC0091F0100E816E4CECB0F0000000008A6A35
:1085EC00C7ECB8F0100E816EB9EC91F0100E816EE4
:1085FC00080E816E6FECB0F0000051ECB0F08A6A9E
:10860C00A1ECB0F08A88B2ECB0F08A424CECB0F03D
:10861C000000100E816EF6EC7CF08A42BEECB0F0DD
:10862C008A6A6AECB0F000008A86BEECB0F0100EDC
:10863C00816E93EC7CF08A424CECB0F000008A46E0
:10864C00B2ECB0F08A6AA1ECB0F08A864CECB0F0D7
:10865C00000000006FECB0F00000100E816E100EE8
:10866C00816E4FEC91F0100E816E4CECB0F000006E
:10867C0000008A6AC7ECB8F0100E816EB9EC91F06C
:10868C00100E816E080E816E6FECB0F000004CEC99
:10869C00B0F08A4600008A42000000008A6AA1EC11
:1086AC00B0F08A88A1ECB0F08A424CECB0F0100E1D
:1086BC00816EF6EC7CF08A42BEECB0F08A6A6AEC11
:1086CC00B0F000008A86BEECB0F0100E816E93EC18
:1086DC007CF08A424CECB0F08A46A1ECB0F08A6A8D
:1086EC00A1ECB0F08A86000000008A4600008A42A5
:1086FC0045ECB0F06FECB0F00000100E816E100E77
:10870C00816E4FEC91F0100E816E4CECB0F00000CD
:10871C0000008A6AC7ECB8F0100E816EB9EC91F0CB
:10872C00100E816E080E816E6FECB0F000004CECF8
:10873C00B0F08A4600008A420000000000008A6AFD
:10874C00A1ECB0F08A88B2ECB0F08A42C7ECB0F081
:10875C00100E816EF6EC7CF08A42BEECB0F08A6AA8
:10876C006AECB0F000008A86BEECB0F0100E816EA0
:10877C0093EC7CF08A42C7ECB0F08A46B2ECB0F0D5
:10878C008A6AA1ECB0F08A860000000000008A46DC
:10879C0000008A4245ECB0F06FECB0F00000100E17
:1087AC00816E100E816E4FEC91F0100E816E4CECC0
:1087BC00B0F0000000008A6AC7ECB8F0100E816EB1
:1087CC00B9EC91F0100E816E080E816E6FECB0F06A
:1087DC0000004CECB0F08A4600008A420000000019
:1087EC00000000008A6AB2ECB0F08A88A1ECB0F00C
:1087FC008A42C2ECB0F0100E816EF6EC7CF08A422C
:10880C00BEECB0F08A6A6AECB0F000008A86BEEC6E
:10881C00B0F0100E816E93EC7CF08A42C2ECB0F09A
:10882C008A46A1ECB0F08A6AB2ECB0F08A860000FD
:10883C000000000000008A4600008A4245ECB0F0BF
:10884C006FECB0F00000100E816E100E816E4FECCC
:10885C0091F0100E816E4CECB0F0000000008A6AB2
:10886C00C7ECB8F0100E816EB9EC91F0100E816E61
:10887C00080E816E6FECB0F000004CECB0F08A4644
:10888C0000008A42B2ECB0F08A6AA1ECB0F08A889F
:10889C00B2ECB0F08A42B2ECB0F0100E816EF6EC95
:1088AC007CF08A42BEECB0F08A6A6AECB0F0000050
:1088BC008A86BEECB0F0100E816E93EC7CF08A428E
:1088CC00B2ECB0F08A46B2ECB0F08A6AA1ECB0F02F
:1088DC008A86B2ECB0F08A4600008A4245ECB0F0D1
:1088EC006FECB0F00000100E816E100E816E4FEC2C
:1088FC0091F0100E816E4CECB0F0000000008A6A12
:10890C00C7ECB8F000008A6A00005FEC91F0100E22
:10891C00816E080E816E6FECB0F000004CECB0F084
:10892C008A4600008A42BEECB0F08A6AB2ECB0F023
:10893C008A88B2ECB0F08A4200000000000000000F
:10894C00100E816EF6EC7CF08A428DECB0F00000DB
:10895C000000100E816E93EC7CF08A420000000047
:10896C00000000008A46B2ECB0F08A6AB2ECB0F0BB
:10897C008A86BEECB0F08A4600008A4245ECB0F024
:10898C006FECB0F00000100E816E100E816E09ECD1
:10899C0091F0000000008A6A4CECB0F0000000007E
:1089AC008A6AC7ECB8F000008A6A00005FEC91F0AC
:1089BC00100E816E080E816E6FECB0F000004CEC66
:1089CC00B0F08A4600008A42C7ECB0F08A6AB2EC7A
:1089DC00B0F08A88B2ECB0F08A4200000000100EB1
:1089EC00816EF6EC7CF08A428DECB0F00000000059
:1089FC00100E816E93EC7CF08A42000000008A46D7
:108A0C00B2ECB0F08A6AB2ECB0F08A86C7ECB0F087
:108A1C008A4600008A4245ECB0F06FECB0F00000E2
:108A2C00100E816E100E816E09EC91F000000000AA
:108A3C008A6A4CECB0F0000000008A6AC7ECB8F00F
:108A4C0000008A6A00005FEC91F0100E816E080E37
:108A5C00816E6FECB0F000004CECB0F08A46000078
:108A6C008A424CECB0F08A6AB2ECB0F08A88B2EC74
:108A7C00B0F08A42100E816EF6EC7CF08A428DECDE
:108A8C00B0F000000000100E816E93EC7CF08A4276
:108A9C008A46B2ECB0F08A6AB2ECB0F08A864CEC42
:108AAC00B0F08A4600008A4245ECB0F06FECB0F0B2
:108ABC000000100E816E100E816E09EC91F000001A
:108ACC0000008A6A4CECB0F0000000008A6AC7EC27
:108ADC00B8F000008A6A00005FEC91F0100E816E15
:108AEC00080E816E6FECB0F000004CECB0F08A46D2
:108AFC0000008A424CECB0F0000000008A6AB2EC34
:108B0C00B0F08A88A1ECB0F0100E816EF6EC7CF01F
:108B1C008A428DECB0F000000000100E816E93ECD8
:108B2C007CF08A88A1ECB0F08A6AB2ECB0F08A864C
:108B3C004CECB0F0000000008A4600008A4245EC84
:108B4C00B0F06FECB0F00000100E816E100E816E64
:108B5C0009EC91F0000000008A6A4CECB0F00000C7
:108B6C0000008A6AC7ECB8F000008A6A00005FEC6B
:108B7C0091F0100E816E080E816E6FECB0F000005B
:108B8C004CECB0F08A4600008A4251ECB0F08A6A94
:108B9C00BEECB0F08A88000000000000100E816E60
:108BAC00F6EC7CF08A428DECB0F000000000100E68
:108BBC00816E93EC7CF08A880000000000008A6AC9
:108BCC00BEECB0F08A8651ECB0F08A4600008A42C6
:108BDC0045ECB0F06FECB0F00000100E816E100E92
:108BEC00816E09EC91F0000000008A6A4CECB0F048
:108BFC00000000008A6AC7ECB8F000008A6A000026
:108C0C005FEC91F0100E816E080E816E6FECB0F07F
:108C1C0000004CECB0F08A4600008A4251ECB0F0F7
:108C2C00000000008A6ABEECB0F08A880000100ECA
:108C3C00816E7EECB0F000008A428DECB0F000004A
:108C4C000000100E816E7EECB0F000008A880000EF
:108C5C008A6ABEECB0F08A8651ECB0F000000000DD
:108C6C008A4600008A4245ECB0F06FECB0F0000090
:108C7C00100E816E100E816E09EC91F00000000058
:108C8C008A6A4CECB0F0000000008A6AC7ECB8F0BD
:108C9C0000008A6A4CECB0F000000000100E816EEF
:108CAC0097ECB0F00000000000008DECB0F0100E5E
:108CBC00816E6FECB0F000006FECB0F000008A42F7
:108CCC00000000008A6AB2ECB0F08A88C2ECB0F006
:108CDC008A42CDECB0F00000000000008A46C2ECE5
:108CEC00B0F08A6AB2ECB0F08A86000000008A46C6
:108CFC006FECB0F06FECB0F00000100E816E97ECE2
:108D0C00B0F00000000000008DECB0F0000000009E
:108D1C0000008A6A4CECB0F0000000008A6AC7ECD4
:108D2C00B8F000008A6A000085EC91F0100E816E9C
:108D3C00080E816E6FECB0F000004CECB0F08A467F
:108D4C0000008A425BECB0F000008A6ABEECB0F026
:108D5C008A88C2ECB0F08A4297ECB0F000000000B8
:108D6C00000092ECB0F000008A46C2ECB0F08A6AC7
:108D7C00BEECB0F08A865BECB0F000008A460000D6
:108D8C008A4245ECB0F06FECB0F00000100E816E32
:108D9C00080E816E27EC91F0000000008A6A4CEC02
:108DAC00B0F0000000008A6AC7ECB8F000008A6AD4
:108DBC00000085EC91F0100E816E080E816E6FEC48
:108DCC00B0F000004CECB0F08A4600008A4265EC32
:108DDC00B0F08A6AC2ECB0F08A88C7ECB0F08A4274
:108DEC0097ECB0F00000000000007EECB0F000004A
:108DFC0000008A46C7ECB0F08A6AC2ECB0F08A86F2
:108E0C0065ECB0F08A4600008A4245ECB0F06FEC9D
:108E1C00B0F00000100E816E080E816E27EC91F000
:108E2C00000000008A6A4CECB0F0000000008A6A76
:108E3C00C7ECB8F000008A6A000085EC91F0100EC7
:108E4C00816E080E816E6FECB0F000004CECB0F04F
:108E5C008A4600008A426AECB0F08A6AC2ECB0F032
:108E6C008A8845ECB0F08A4297ECB0F00000000024
:108E7C0000006FECB0F08A4645ECB0F08A6AC2ECA8
:108E8C00B0F08A866AECB0F08A4600008A4245EC63
:108E9C00B0F06FECB0F00000100E816E080E816E19
:108EAC0027EC91F0000000008A6A4CECB0F0000056
:108EBC0000008A6AC7ECB8F000008A6A000085ECF2
:108ECC0091F0100E816E080E816E6FECB0F0000008
:108EDC004CECB0F08A4600008A426FECB0F08A6A23
:108EEC00C2ECB0F08A884CECB0F08A4297ECB0F04F
:108EFC000000000000005BECB0F000008A464CEC77
:108F0C00B0F08A6AC2ECB0F08A866FECB0F08A4698
:108F1C0000008A4245ECB0F06FECB0F00000100E8F
:108F2C00816E080E816E27EC91F0000000008A6AB9
:108F3C004CECB0F0000000008A6AC7ECB8F00000FE
:108F4C008A6A000085EC91F0100E816E080E816E1D
:108F5C006FECB0F000004CECB0F08A4600008A4296
:108F6C0079ECB0F08A6AC7ECB0F08A884CECB0F0BF
:108F7C0000008A4297ECB0F00000000000004CECBE
:108F8C00B0F08A464CECB0F000008A6AC7ECB0F046
:108F9C008A8679ECB0F08A4600008A4245ECB0F043
:108FAC006FECB0F00000100E816E080E816E27EC95
:108FBC0091F0000000008A6A4CECB0F00000000058
:108FCC008A6AC7ECB8F0100E816E000085EC91F047
:108FDC00100E816E080E816E6FECB0F000004CEC40
:108FEC00B0F08A4600008A427EECB0F08A6A45EC0A
:108FFC00B0F08A884CECB0F0000000008A4297EC8C
:10900C00B0F000000000000000008A464CECB0F00C
:10901C00000000008A6A45ECB0F08A867EECB0F065
:10902C008A4600008A4245ECB0F06FECB0F00000CC
:10903C00100E816E080E816E27EC91F00000100E60
:10904C00816E4CECB0F0000000008A6AC7ECB8F0FE
:10905C00100E816E000085EC91F0100E816E080EE2
:10906C00816E6FECB0F000004CECB0F08A46000062
:10907C008A4283ECB0F000008A6A4CECB0F08A882B
:10908C0056ECB0F000008A426FECB0F0000000002B
:10909C008A4656ECB0F000008A6A4CECB0F08A8636
:1090AC0083ECB0F000008A4600008A4245ECB0F038
:1090BC006FECB0F00000100E816E080E816E27EC84
:1090CC0091F00000100E816E4CECB0F0000000002E
:1090DC008A6AC7ECB8F0100E816E76EC91F0100E27
:1090EC00816E080E816E51ECB0F00000100E816E96
:1090FC0000000000080E816E56ECB0F0000000007D
:10910C00100E816E080E816E6FECB0F000004CEC0E
:10911C00B0F08A4600008A428DECB0F000000000EE
:10912C008A6A4CECB0F000008A88ADECB0F08A6A28
:10913C004CECB0F000008A868DECB0F00000000022
:10914C008A4600008A4245ECB0F06FECB0F00000AB
:10915C00100E816E080E816E5BECB0F00000100EEC
:10916C00816E00000000080E816E4CECB0F0000027
:10917C000000100E816E080E816E18EC91F000004C
:10918C008A6AC7ECB8F0100E816E76EC91F0100E76
:10919C00816E080E816E4CECB0F000000000100ED9
:1091AC00816E7CECBAF0080E816E56ECB0F0100EAD
:1091BC00816E080E816E6FECB0F000004CECB0F0DC
:1091CC008A4600008A4297ECB0F08A6A51ECB0F003
:1091DC00000000008A888DECB0F0000000008A6A64
:1091EC0051ECB0F0000000008A8697ECB0F08A4693
:1091FC0000008A4245ECB0F06FECB0F00000100EAD
:10920C00816E080E816E56ECB0F000000000100E5E
:10921C00816E5EECBBF0080E816E4CECB0F0100E63
:10922C00816E080E816E18EC91F000008A6AC7EC12
:10923C00B8F0100E816E76EC91F0100E816E080E67
:10924C00816E4CECB0F0100E816E75ECBAF0080E1D
:10925C00816E51ECB0F00000100E816E080E816E24
:10926C006FECB0F000004CECB0F08A4600008A4283
:10927C008DECB0F08A4600008A42C2ECB0F08A6AEB
:10928C005BECB0F0000000008A885BECB0F00000F2
:10929C008A6A5BECB0F0000000008A86C2ECB0F089
:1092AC008A4600008A428DECB0F08A4600008A4261
:1092BC0045ECB0F06FECB0F00000100E816E080EB3
:1092CC00816E56ECB0F0100E816E57ECBBF0080EB0
:1092DC00816EC7ECB0F0100E816E080E816E18EC2A
:1092EC0091F000008A6AC7ECB8F0100E816E76EC33
:1092FC0091F0100E816E080E816EC7ECB0F0100E5E
:10930C00816E70ECBAF0080E816E4CECB0F000007F
:10931C000000100E816E080E816E6FECB0F0000034
:10932C004CECB0F08A4600008A428DECB0F08A46D4
:10933C0000008A4251ECB0F000008A6A97ECB0F061
:10934C000000000000000000000000008A8651ECC4
:10935C00B0F000008A4600008A428DECB0F08A46DC
:10936C0000008A4245ECB0F06FECB0F00000100E3B
:10937C00816E080E816E51ECB0F00000100E816E03
:10938C0052ECBBF0080E816EBEECB0F0100E816E8C
:10939C00080E816E18EC91F000008A6AC7ECB8F0E8
:1093AC00100E816E76EC91F0100E816E080E816EAF
:1093BC00BEECB0F0100E816E67ECBAF0080E816E48
:1093CC004CECB0F0100E816E080E816E6FECB0F0AC
:1093DC0000004CECB0F08A4600008A428DECB0F0F4
:1093EC008A4600008A4265ECB0F000008A6A7EEC86
:1093FC00B0F08A8665ECB0F000008A4600008A4224
:10940C008DECB0F08A4600008A4245ECB0F06FEC6F
:10941C00B0F00000100E816E080E816E4CECB0F0B6
:10942C0000000000100E816E49ECBBF0080E816E3E
:10943C00A1ECB0F0100E816E080E816E18EC91F05C
:10944C0000008A6AC7ECB8F0100E816E76EC91F0D1
:10945C00100E816E080E816EA1ECB0F0100E816EB4
:10946C005AECBAF0080E816EC7ECB0F0100E816E9B
:10947C00080E816E83ECB0F000000000100E816EBF
:10948C00080E816E83ECB0F000000000100E816EAF
:10949C00080E816E92ECB0F083ECB0F0000000008E
:1094AC00100E816E080E816E83ECB0F0000000008F
:1094BC00100E816E080E816E83ECB0F0000000007F
:1094CC00100E816E080E816E4CECB0F0100E816E99
:1094DC003CECBBF0080E816E000000000000100E8A
:1094EC00816E080E816E18EC91F000008A6AC7EC50
:1094FC00B8F0100E816E76EC91F0100E816E080EA5
:10950C00816E000000000000100E816E55ECBAF068
:10951C00080E816EBEECB0F0100E816E080E816EDE
:10952C0001EC7EF0100E816E080E816EC7ECB0F06F
:10953C00100E816E37ECBBF0080E816E0000100E21
:10954C00816E080E816E18EC91F000008A6AC7ECEF
:10955C00B8F0100E816E76EC91F0100E816E080E44
:10956C00816E0000100E816E4CECBAF0080E816E0C
:10957C00A1ECB0F0100E816E080E816E01EC7EF045
:10958C00100E816E080E816EBEECB0F0100E816E66
:10959C002EECBBF00000100E816E080E816E18ECE4
:1095AC0091F000008A6AC7ECB8F0100E816E76EC70
:1095BC0091F0100E816E0000100E816E3FECBAF02F
:1095CC00080E816E000000000000100E816E080E67
:1095DC00816E01EC7EF0100E816E080E816EA1EC96
:1095EC00B0F0100E816E21ECBBF00000080E816E05
:1095FC0018EC91F000008A6AC7ECB8F0100E816E7E
:10960C0076EC91F000008A46000034ECBAF0080EBB
:10961C00816E0000100E816E080E816E01EC7EF0E2
:10962C00100E816E080E816E000000000000100EFE
:10963C00816E16ECBBF0080E816E83ECB0F000006E
:10964C00100E816E080E816E000000000000100EDE
:10965C00816E4CECB0F0000000008A6AEAEC98F0E5
:10966C00E4EF63F0E8EC9FF000008A6AC7ECB8F016
:10967C00100E816E76EC91F000008A46000034ECFE
:10968C00BAF0080E816E0000100E816E080E816E0D
:10969C0001EC7EF0100E816E080E816E0000000051
:1096AC000000100E816E16ECBBF0080E816E83EC80
:1096BC00B0F00000100E816E080E816E00000000EC
:1096CC000000100E816EB2ECB0F082A0B7EF65F026
:1096DC0082A22EEF00F000008A6AC7ECB8F0100EE0
:1096EC00816E76EC91F0100E816E0000100E816E82
:1096FC003FECBAF0080E816E000000000000100E66
:10970C00816E080E816E01EC7EF0100E816E080EDB
:10971C00816EA1ECB0F0100E816E21ECBBF000005C
:10972C00080E816E18EC91F000008A6AC7ECB8F054
:10973C00100E816E76EC91F0100E816E080E816E1B
:10974C000000100E816E4CECBAF0080E816EA1EC8C
:10975C00B0F0100E816E080E816E01EC7EF0100ED2
:10976C00816E080E816EBEECB0F0100E816E2EEC88
:10977C00BBF00000100E816E080E816E18EC91F09B
:10978C0000008A6AC7ECB8F0100E816E76EC91F08E
:10979C00100E816E080E816E000000000000100E8D
:1097AC00816E55ECBAF0080E816EBEECB0F0100E66
:1097BC00816E080E816E01EC7EF0100E816E080E2B
:1097CC00816EC7ECB0F0100E816E37ECBBF0080E5A
:1097DC00816E0000100E816E080E816E18EC91F0F7
:1097EC0000008A6AC7ECB8F0100E816E76EC91F02E
:1097FC00100E816E080E816EA1ECB0F0100E816E11
:10980C005AECBAF0080E816EC7ECB0F0100E816EF7
:10981C00080E816E83ECB0F000000000100E816E1B
:10982C00080E816E83ECB0F000000000100E816E0B
:10983C00080E816E92ECB0F083ECB0F000000000EA
:10984C00100E816E080E816E83ECB0F000000000EB
:10985C00100E816E080E816E83ECB0F000000000DB
:10986C00100E816E080E816E4CECB0F0100E816EF5
:10987C003CECBBF0080E816E000000000000100EE6
:10988C00816E080E816E18EC91F000008A6AC7ECAC
:10989C00B8F0100E816E76EC91F0100E816E080E01
:1098AC00816EBEECB0F0100E816E67ECBAF0080E53
:1098BC00816E4CECB0F0100E816E080E816E6FEC68
:1098CC00B0F000004CECB0F08A4600008A428DECFF
:1098DC00B0F08A4600008A4265ECB0F000008A6A5B
:1098EC007EECB0F08A8665ECB0F000008A46000091
:1098FC008A428DECB0F08A4600008A4245ECB0F00A
:10990C006FECB0F00000100E816E080E816E4CEC06
:10991C00B0F000000000100E816E49ECBBF0080E98
:10992C00816EA1ECB0F0100E816E080E816E18ECF9
:10993C0091F000008A6AC7ECB8F0100E816E76ECDC
:10994C0091F0100E816E080E816EC7ECB0F0100E07
:10995C00816E70ECBAF0080E816E4CECB0F0000029
:10996C000000100E816E080E816E6FECB0F00000DE
:10997C004CECB0F08A4600008A428DECB0F08A467E
:10998C0000008A4251ECB0F000008A6A97ECB0F00B
:10999C000000000000000000000000008A8651EC6E
:1099AC00B0F000008A4600008A428DECB0F08A4686
:1099BC0000008A4245ECB0F06FECB0F00000100EE5
:1099CC00816E080E816E51ECB0F00000100E816EAD
:1099DC0052ECBBF0080E816EBEECB0F0100E816E36
:1099EC00080E816E18EC91F000008A6AC7ECB8F092
:1099FC00100E816E76EC91F0100E816E080E816E59
:109A0C004CECB0F0100E816E75ECBAF0080E816E55
:109A1C0051ECB0F00000100E816E080E816E6FECF0
:109A2C00B0F000004CECB0F08A4600008A428DEC9D
:109A3C00B0F08A4600008A42C2ECB0F08A6A5BEC55
:109A4C00B0F0000000008A885BECB0F000008A6A7D
:109A5C005BECB0F0000000008A86C2ECB0F08A46E5
:109A6C0000008A428DECB0F08A4600008A4245EC38
:109A7C00B0F06FECB0F00000100E816E080E816E2D
:109A8C0056ECB0F0100E816E57ECBBF0080E816EE8
:109A9C00C7ECB0F0100E816E080E816E18EC91F0D0
:109AAC0000008A6AC7ECB8F0100E816E76EC91F06B
:109ABC00100E816E080E816E4CECB0F000000000B0
:109ACC00100E816E7CECBAF0080E816E56ECB0F084
:109ADC00100E816E080E816E6FECB0F000004CEC35
:109AEC00B0F08A4600008A4297ECB0F08A6A51ECDA
:109AFC00B0F0000000008A888DECB0F0000000008F
:109B0C008A6A51ECB0F0000000008A8697ECB0F045
:109B1C008A4600008A4245ECB0F06FECB0F00000D1
:109B2C00100E816E080E816E56ECB0F00000000035
:109B3C00100E816E5EECBBF0080E816E4CECB0F03A
:109B4C00100E816E080E816E18EC91F000008A6A7E
:109B5C00C7ECB8F0100E816E76EC91F0100E816EA1
:109B6C00080E816E51ECB0F00000100E816E0000FA
:109B7C000000080E816E56ECB0F000000000100ED4
:109B8C00816E080E816E6FECB0F000004CECB0F002
:109B9C008A4600008A428DECB0F0000000008A6A10
:109BAC004CECB0F000008A88ADECB0F08A6A4CEC5A
:109BBC00B0F000008A868DECB0F0000000008A4600
:109BCC0000008A4245ECB0F06FECB0F00000100ED3
:109BDC00816E080E816E5BECB0F00000100E816E91
:109BEC0000000000080E816E4CECB0F0000000008C
:109BFC00100E816E080E816E18EC91F000008A6ACE
:109C0C00C7ECB8F0100E816E76EC91F0100E816EF0
:109C1C00080E816E83ECB0F000000000100E816E17
:109C2C00080E816E6FECB0F000004CECB0F08A4680
:109C3C0000008A4283ECB0F000008A6A4CECB0F071
:109C4C008A8856ECB0F000008A426FECB0F000004D
:109C5C0000008A4656ECB0F000008A6A4CECB0F07A
:109C6C008A8683ECB0F000008A4600008A4245ECFC
:109C7C00B0F06FECB0F00000100E816E080E816E2B
:109C8C0083ECB0F000000000100E816E080E816EA7
:109C9C0018EC91F000008A6AC7ECB8F0100E816ED7
:109CAC0076EC91F0100E816E080E816E83ECB0F0A4
:109CBC0000000000100E816E080E816E6FECB0F08B
:109CCC0000004CECB0F08A4600008A427EECB0F00A
:109CDC008A6A45ECB0F08A884CECB0F000000000C9
:109CEC008A4297ECB0F000000000000000008A46A9
:109CFC004CECB0F0000000008A6A45ECB0F08A86AB
:109D0C007EECB0F08A4600008A4245ECB0F06FEC75
:109D1C00B0F00000100E816E080E816E83ECB0F076
:109D2C0000000000100E816E080E816E83ECB0F006
:109D3C0000000000100E816E080E816E0000000005
:109D4C000000100E816E4CECB0F0000000008A6A2E
:109D5C00C7ECB8F000008A6A000085EC91F0100E98
:109D6C00816E080E816E6FECB0F000004CECB0F020
:109D7C008A4600008A4279ECB0F08A6AC7ECB0F0EF
:109D8C008A884CECB0F000008A4297ECB0F00000EE
:109D9C00000000004CECB0F08A464CECB0F0000037
:109DAC008A6AC7ECB0F08A8679ECB0F08A4600007B
:109DBC008A4245ECB0F06FECB0F00000100E816EF2
:109DCC00080E816E27EC91F0000000008A6A4CECC2
:109DDC00B0F0000000008A6AC7ECB8F000008A6A94
:109DEC00000085EC91F0100E816E080E816E6FEC08
:109DFC00B0F000004CECB0F08A4600008A426FECE8
:109E0C00B0F08A6AC2ECB0F08A884CECB0F08A42AE
:109E1C0097ECB0F00000000000005BECB0F000002C
:109E2C008A464CECB0F08A6AC2ECB0F08A866FECD1
:109E3C00B0F08A4600008A4245ECB0F06FECB0F00E
:109E4C000000100E816E080E816E27EC91F0000060
:109E5C0000008A6A4CECB0F0000000008A6AC7EC83
:109E6C00B8F000008A6A000085EC91F0100E816E4B
:109E7C00080E816E6FECB0F000004CECB0F08A462E
:109E8C0000008A426AECB0F08A6AC2ECB0F08A88B0
:109E9C0045ECB0F08A4297ECB0F0000000000000F6
:109EAC006FECB0F08A4645ECB0F08A6AC2ECB0F0C8
:109EBC008A866AECB0F08A4600008A4245ECB0F023
:109ECC006FECB0F00000100E816E080E816E27EC66
:109EDC0091F0000000008A6A4CECB0F00000000029
:109EEC008A6AC7ECB8F000008A6A000085EC91F031
:109EFC00100E816E080E816E6FECB0F000004CEC11
:109F0C00B0F08A4600008A4265ECB0F08A6AC2EC76
:109F1C00B0F08A88C7ECB0F08A4297ECB0F0000041
:109F2C00000000007EECB0F0000000008A46C7EC98
:109F3C00B0F08A6AC2ECB0F08A8665ECB0F08A4662
:109F4C0000008A4245ECB0F06FECB0F00000100E4F
:109F5C00816E080E816E27EC91F0000000008A6A79
:109F6C004CECB0F0000000008A6AC7ECB8F00000BE
:109F7C008A6A000085EC91F0100E816E080E816EDD
:109F8C006FECB0F000004CECB0F08A4600008A4256
:109F9C005BECB0F000008A6ABEECB0F08A88C2ECD0
:109FAC00B0F08A4297ECB0F000000000000092EC98
:109FBC00B0F000008A46C2ECB0F08A6ABEECB0F099
:109FCC008A865BECB0F000008A4600008A4245ECC1
:109FDC00B0F06FECB0F00000100E816E080E816EC8
:109FEC0027EC91F0000000008A6A4CECB0F0000005
:109FFC0000008A6AC7ECB8F000008A6A000085ECA1
:10A00C0091F0100E816E080E816E6FECB0F00000B6
:10A01C004CECB0F0000000008A4600008A4256EC7E
:10A02C00B0F08A6AB2ECB0F08A8800007EECB0F036
:10A03C0000008A426AECB0F00000000051ECB0F075
:10A04C000000100E816E7EECB0F000008A6AB2EC5B
:10A05C00B0F08A8656ECB0F08A4600008A424CEC8E
:10A06C00B0F000006FECB0F00000100E816E080E26
:10A07C00816E27EC91F0000000008A6A4CECB0F085
:10A08C00000000008A6AC7ECB8F000008A6A4CEC49
:10A09C00B0F000000000100E816ECDECB0F00000AE
:10A0AC00000065ECB0F051ECB0F000004CECB0F0FE
:10A0BC0000008A42000000008A6ABEECB0F08A8878
:10A0CC000000100E816E93EC7CF08A426AECB0F0CA
:10A0DC000000000051ECB0F00000100E816EF6ECA8
:10A0EC007CF08A8800008A6ABEECB0F08A86000098
:10A0FC0000008A4651ECB0F000004CECB0F0CDEC16
:10A10C00B0F00000000065ECB0F0000000000000B2
:10A11C008A6A4CECB0F0000000008A6AC7ECB8F018
:10A12C0000008A6A00005FEC91F0100E816E080E40
:10A13C00816E6FECB0F000004CECB0F08A46000081
:10A14C008A4251ECB0F08A6ABEECB0F08A8800000A
:10A15C0000000000100E816E93EC7CF08A426AECD9
:10A16C00B0F00000000051ECB0F00000100E816E59
:10A17C00F6EC7CF08A880000000000008A6ABEECD5
:10A18C00B0F08A8651ECB0F08A4600008A4245EC69
:10A19C00B0F06FECB0F00000100E816E100E816EFE
:10A1AC0009EC91F0000000008A6A4CECB0F0000061
:10A1BC0000008A6AC7ECB8F000008A6A00005FEC05
:10A1CC0091F0100E816E080E816E6FECB0F00000F5
:10A1DC004CECB0F08A4600008A424CECB0F0000027
:10A1EC0000008A6AB2ECB0F08A88A1ECB0F0100ED4
:10A1FC00816E93EC7CF08A426AECB0F000000000B7
:10A20C0051ECB0F00000100E816EF6EC7CF08A88F8
:10A21C00A1ECB0F08A6AB2ECB0F08A864CECB0F0EB
:10A22C00000000008A4600008A4245ECB0F06FEC5A
:10A23C00B0F00000100E816E100E816E09EC91F0E2
:10A24C00000000008A6A4CECB0F0000000008A6A42
:10A25C00C7ECB8F000008A6A00005FEC91F0100EB9
:10A26C00816E080E816E6FECB0F000004CECB0F01B
:10A27C008A4600008A424CECB0F08A6AB2ECB0F02C
:10A28C008A88B2ECB0F08A42100E816E93EC7CF0AE
:10A29C008A426AECB0F00000000051ECB0F0000013
:10A2AC00100E816EF6EC7CF08A428A46B2ECB0F06D
:10A2BC008A6AB2ECB0F08A864CECB0F08A460000A8
:10A2CC008A4245ECB0F06FECB0F00000100E816EDD
:10A2DC00100E816E09EC91F0000000008A6A4CECC3
:10A2EC00B0F0000000008A6AC7ECB8F000008A6A7F
:10A2FC0000005FEC91F0100E816E080E816E6FEC19
:10A30C00B0F000004CECB0F08A4600008A42C7EC7A
:10A31C00B0F08A6AB2ECB0F08A88B2ECB0F08A4243
:10A32C0000000000100E816E93EC7CF08A426AEC07
:10A33C00B0F00000000051ECB0F00000100E816E87
:10A34C00F6EC7CF08A42000000008A46B2ECB0F0D9
:10A35C008A6AB2ECB0F08A86C7ECB0F08A4600008C
:10A36C008A4245ECB0F06FECB0F00000100E816E3C
:10A37C00100E816E09EC91F0000000008A6A4CEC22
:10A38C00B0F0000000008A6AC7ECB8F000008A6ADE
:10A39C0000005FEC91F0100E816E080E816E6FEC78
:10A3AC00B0F000004CECB0F08A4600008A42BEECE3
:10A3BC00B0F08A6AB2ECB0F08A88B2ECB0F08A42A3
:10A3CC000000000000000000100E816E93EC7CF089
:10A3DC008A426AECB0F00000000051ECB0F00000D2
:10A3EC00100E816EF6EC7CF08A420000000000003A
:10A3FC0000008A46B2ECB0F08A6AB2ECB0F08A8601
:10A40C00BEECB0F08A4600008A4245ECB0F06FEC2E
:10A41C00B0F00000100E816E100E816E09EC91F000
:10A42C00000000008A6A4CECB0F0000000008A6A60
:10A43C00C7ECB8F0100E816E00005FEC91F0100EBE
:10A44C00816E080E816E6FECB0F000004CECB0F039
:10A45C008A4600008A42B2ECB0F08A6AA1ECB0F0F5
:10A46C008A88B2ECB0F08A42B2ECB0F0100E816E79
:10A47C0093EC7CF08A42BEECB0F08A466AECB0F009
:10A48C0000008A42BEECB0F0100E816EF6EC7CF04F
:10A49C008A42B2ECB0F08A46B2ECB0F08A6AA1EC17
:10A4AC00B0F08A86B2ECB0F08A4600008A4245ECE5
:10A4BC00B0F06FECB0F00000100E816E100E816EDB
:10A4CC0009EC91F00000100E816E4CECB0F0000025
:10A4DC0000008A6AC7ECB8F0100E816E00005FECC9
:10A4EC0091F0100E816E080E816E6FECB0F00000D2
:10A4FC004CECB0F08A4600008A42000000000000DC
:10A50C0000008A6AB2ECB0F08A88A1ECB0F08A4202
:10A51C00C2ECB0F0100E816E93EC7CF08A42BEEC73
:10A52C00B0F08A466AECB0F000008A42BEECB0F0A3
:10A53C00100E816EF6EC7CF08A42C2ECB0F08A46CA
:10A54C00A1ECB0F08A6AB2ECB0F08A860000000090
:10A55C00000000008A4600008A4245ECB0F06FEC27
:10A56C00B0F00000100E816E100E816E09EC91F0AF
:10A57C000000100E816E4CECB0F0000000008A6AF6
:10A58C00C7ECB8F0100E816E00005FEC91F0100E6D
:10A59C00816E080E816E6FECB0F000004CECB0F0E8
:10A5AC008A4600008A420000000000008A6AA1EC82
:10A5BC00B0F08A88B2ECB0F08A42C7ECB0F0100E62
:10A5CC00816E93EC7CF08A42BEECB0F08A466AEC69
:10A5DC00B0F000008A42BEECB0F0100E816EF6ECCA
:10A5EC007CF08A42C7ECB0F08A46B2ECB0F08A6AD2
:10A5FC00A1ECB0F08A860000000000008A46000042
:10A60C008A4245ECB0F06FECB0F00000100E816E99
:10A61C00100E816E09EC91F00000100E816E4CEC66
:10A62C00B0F0000000008A6AC7ECB8F0100E816E22
:10A63C0000005FEC91F0100E816E080E816E6FECD5
:10A64C00B0F000004CECB0F08A4600008A420000EA
:10A65C0000008A6AA1ECB0F08A88A1ECB0F08A42C2
:10A66C004CECB0F0100E816E93EC7CF08A42BEEC98
:10A67C00B0F08A466AECB0F000008A42BEECB0F052
:10A68C00100E816EF6EC7CF08A424CECB0F08A46EF
:10A69C00A1ECB0F08A6AA1ECB0F08A860000000050
:10A6AC008A4600008A4245ECB0F06FECB0F0000036
:10A6BC00100E816E100E816E09EC91F00000100EE0
:10A6CC00816E4CECB0F0000000008A6AC7ECB8F068
:10A6DC00100E816E00005FEC91F0100E816E080E72
:10A6EC00816E6FECB0F0000051ECB0F08A6AA1EC16
:10A6FC00B0F08A88B2ECB0F08A424CECB0F00000BA
:10A70C00100E816E93EC7CF08A42BEECB0F08A465F
:10A71C006AECB0F000008A42BEECB0F0100E816E14
:10A72C00F6EC7CF08A424CECB0F000008A46B2ECBD
:10A73C00B0F08A6AA1ECB0F08A864CECB0F0000064
:10A74C0000006FECB0F00000100E816E100E816EE8
:10A75C0009EC91F00000100E816E4CECB0F0000092
:10A76C0000008A6AC7ECB8F0100E816E00005FEC36
:10A77C0091F0100E816E080E816E6FECB0F000003F
:10A78C004CECB0F0000000008A6AA1ECB0F08A88B2
:10A79C00A1ECB0F08A4251ECB0F0100E816E93EC4B
:10A7AC007CF08A42BEECB0F08A466AECB0F0000055
:10A7BC008A42BEECB0F0100E816EF6EC7CF08A4250
:10A7CC0051ECB0F08A46A1ECB0F08A6AA1ECB0F082
:10A7DC008A864CECB0F000006FECB0F00000100E6C
:10A7EC00816E100E816E09EC91F00000100E816EDE
:10A7FC004CECB0F0000000008A6AC7ECB8F0100E08
:10A80C00816E9CEC91F0100E816E080E816E6FECD7
:10A81C00B0F000004CECB0F000008A6AA1ECB0F093
:10A82C008A88A1ECB0F08A4251ECB0F00000100E16
:10A83C00816E93EC7CF08A42BEECB0F08A466AECF6
:10A84C00B0F000008A42BEECB0F0100E816EF6EC57
:10A85C007CF08A4251ECB0F000008A46A1ECB0F0DA
:10A86C008A6AA1ECB0F08A864CECB0F06FECB0F0D8
:10A87C000000100E816E100E816E36EC91F0100EF1
:10A88C00816E4CECB0F0000000008A6AC7ECB8F0A6
:10A89C00100E816E9CEC91F0100E816E080E816E84
:10A8AC006FECB0F000004CECB0F08A6AA1ECB0F0A8
:10A8BC008A88A1ECB0F08A4251ECB0F000000000A4
:10A8CC00100E816E93EC7CF08A42BEECB0F08A469E
:10A8DC006AECB0F000008A42BEECB0F0100E816E53
:10A8EC00F6EC7CF08A4251ECB0F0000000008A4695
:10A8FC00A1ECB0F08A6AA1ECB0F08A8645ECB0F01D
:10A90C006FECB0F00000100E816E100E816E36EC04
:10A91C0091F0100E816E4CECB0F0000000008A6AD1
:10A92C00C7ECB8F0100E816E9CEC91F0100E816E9D
:10A93C00080E816E6FECB0F0000045ECB0F08A6A46
:10A94C00A1ECB0F08A8800000000000000008A42F0
:10A95C0056ECB0F00000100E816E93EC7CF08A4245
:10A96C00BEECB0F08A466AECB0F000008A42BEEC55
:10A97C00B0F0100E816EF6EC7CF08A4256ECB0F022
:10A98C0000008A4600000000000000008A6AA1EC6A
:10A99C00B0F08A86C7ECB0F06FECB0F00000100E8F
:10A9AC00816E100E816E36EC91F0100E816E4CECB7
:10A9BC00B0F0000000008A6AC7ECB8F0100E816E8F
:10A9CC009CEC91F0100E816E080E816E6FECB0F065
:10A9DC000000C7ECB0F08A6AA1ECB0F08A880000E5
:10A9EC000000000000008A4256ECB0F000000000AD
:10A9FC00100E816E93EC7CF08A42BEECB0F08A466D
:10AA0C006AECB0F000008A42BEECB0F0100E816E21
:10AA1C00F6EC7CF08A4256ECB0F0000000008A465E
:10AA2C0000000000000000008A6AA1ECB0F08A86E9
:10AA3C00C2ECB0F06FECB0F00000100E816E100E96
:10AA4C00816E36EC91F0100E816E4CECB0F0000083
:10AA5C0000008A6AC7ECB8F0100E816E9CEC91F085
:10AA6C00100E816E080E816E6FECB0F00000C2EC1F
:10AA7C00B0F08A6AA1ECB0F08A88000000000000F7
:10AA8C0000008A425BECB0F0100E816E93EC7CF00F
:10AA9C008A42BEECB0F08A466AECB0F000008A4202
:10AAAC00BEECB0F0100E816EF6EC7CF08A425BECE2
:10AABC00B0F08A4600000000000000008A6AA1EC99
:10AACC00B0F08A86BEECB0F06FECB0F00000100E67
:10AADC00816E100E816E36EC91F0100E816E4CEC86
:10AAEC00B0F0000000008A6AC7ECB8F0100E816E5E
:10AAFC009CEC91F0100E816E080E816E6FECB0F034
:10AB0C000000BEECB0F08A6AA1ECB0F08A880000BC
:10AB1C000000000000008A425BECB0F00000100E58
:10AB2C00816E7EECB0F000008A42BEECB0F08A463A
:10AB3C006AECB0F000008A42BEECB0F0100E816EF0
:10AB4C007EECB0F000008A425BECB0F000008A466C
:10AB5C0000000000000000008A6AA1ECB0F08A86B8
:10AB6C00B2ECB0F06FECB0F00000100E816E100E75
:10AB7C00816E36EC91F0100E816E4CECB0F0000052
:10AB8C0000008A6AC7ECB8F000008A6A9CEC91F06D
:10AB9C00100E816E080E816EF1EC7FF0100E816E3E
:10ABAC00100E816E36EC91F000008A6A4CECB0F01D
:10ABBC00000000008A6AC7ECB8F000008A6A9CECBE
:10ABCC0091F0100E816E080E816ED3EC80F0100E99
:10ABDC00816E100E816E36EC91F000008A6A4CEC9E
:10ABEC00B0F0000000008A6AC7ECB8F000008A6A76
:10ABFC009CEC91F0100E816E080E816E87EC81F04A
:10AC0C00100E816E100E816E36EC91F000008A6A87
:10AC1C004CECB0F0000000008A6AC7ECB8F0000001
:10AC2C008A6A9CEC91F0100E816E080E816E79ECA4
:10AC3C0082F0100E816E100E816E36EC91F00000D9
:10AC4C008A6A4CECB0F0000000008A6AC7ECB8F0DD
:10AC5C0000008A6A9CEC91F0100E816E080E816ED9
:10AC6C006CEC83F0100E816E100E816E36EC91F050
:10AC7C0000008A6A4CECB0F0000000008A6AC7EC55
:10AC8C00B8F000008A6A9CEC91F0100E816E080EF0
:10AC9C00816E68EC84F0100E816E100E816E36ECB5
:10ACAC0091F000008A6A4CECB0F0000000008A6A57
:10ACBC00C7ECB8F000008A6A4CECB0F00000000061
:10ACCC00100E816E97ECB0F000008A6A56ECB0F072
:10ACDC000000100E816E00008A6A56ECB0F0000085
:10ACEC00100E816E100E816E28EC85F0100E816EA8
:10ACFC00100E816E56ECB0F0000000008A6A100E47
:10AD0C00816E56ECB0F00000100E816E97ECB0F036
:10AD1C000000000000008A6A4CECB0F0000000005B
:10AD2C008A6AC7ECB8F000008A6A9CEC91F0100EAD
:10AD3C00816E080E816E9EEC85F0100E816E100EE9
:10AD4C00816E36EC91F000008A6A4CECB0F0000099
:10AD5C0000008A6AC7ECB8F000008A6A9CEC91F09B
:10AD6C00100E816E080E816E88EC86F0100E816ECE
:10AD7C00100E816E36EC91F000008A6A4CECB0F04B
:10AD8C00000000008A6AC7ECB8F000008A6A9CECEC
:10AD9C0091F0100E816E080E816E69EC7EF0100E33
:10ADAC00816E100E816E36EC91F000008A6A4CECCC
:10ADBC00B0F0000000008A6AC7ECB8F000008A6AA4
:10ADCC009CEC91F0100E816E080E816E13EC7FF0EE
:10ADDC00100E816E100E816E36EC91F000008A6AB6
:10ADEC004CECB0F0000000008A6AC7ECB8F0000030
:10ADFC008A6A9CEC91F0100E816E080E816E82ECCA
:10AE0C007FF0100E816E100E816E36EC91F000000A
:10AE1C008A6A4CECB0F0000000008A6AC7ECB8F00B
:10AE2C00100E816E9CEC91F0100E816E080E816EEE
:10AE3C0061EC88F0100E816E100E816E36EC91F084
:10AE4C00100E816E4CECB0F0000000008A6AC7EC6A
:10AE5C00B8F0100E816E9CEC91F0100E816E080E05
:10AE6C00816ED6EC88F0100E816E100E816E36EC71
:10AE7C0091F0100E816E4CECB0F0000000008A6A6C
:10AE8C00C7ECB8F0100E816E9CEC91F0100E816E38
:10AE9C00080E816ED6EC88F0100E816E100E816E4D
:10AEAC0036EC91F0100E816E4CECB0F0000000000E
:10AEBC008A6A020E0F6F0000000000008B9E97EC58
:10AECC00B0F000000000000000008B8E97ECB0F09A
:10AEDC00000000000000000003D08A6AC7ECB8F044
:10AEEC00100E816E9CEC91F0100E816E080E816E2E
:10AEFC0087EC89F0100E816E100E816E36EC91F09D
:10AF0C00100E816E45ECB0F00F2FE7D700008A6A67
:10AF1C00C7ECB8F0100E816E9CEC91F0100E816EA7
:10AF2C00080E816EFBEC89F0100E816E100E816E96
:10AF3C0036EC91F0100E816E4CECB0F00000030E6C
:10AF4C008A6A0F6F00000000000000008B9E97ECD7
:10AF5C00B0F000000000000000008B8E97ECB0F009
:10AF6C00000000000000000003D08A6AC7ECB8F0B3
:10AF7C00100E816E9CEC91F0100E816E080E816E9D
:10AF8C0071EC8AF0100E816E100E816E36EC91F021
:10AF9C00100E816E45ECB0F00F2FE7D700008A6AD7
:10AFAC00C7ECB8F0100E816E9CEC91F0100E816E17
:10AFBC00080E816EC3EC86F0100E816E100E816E41
:10AFCC0036EC91F0100E816E4CECB0F000000000ED
:10AFDC008A6AC7ECB8F0100E816E9CEC91F0100EE2
:10AFEC00816E080E816EC3EC86F0100E816E100E11
:10AFFC00816E36EC91F0100E816E4CECB0F00000CE
:10B00C0000008A6AC7ECB8F0100E816E9CEC91F0CF
:10B01C00100E816E080E816EB0EC87F0100E816EF2
:10B02C00100E816E36EC91F0100E816E4CECB0F07F
:10B03C00000000008A6AC7ECB8F000008A6A9CEC39
:10B04C0091F0100E816E080E816E42EC8DF0100E98
:10B05C00816E100E816E36EC91F000008A6A4CEC19
:10B06C00B0F0000000008A6AC7ECB8F000008A6AF1
:10B07C009CEC91F0100E816E080E816E7DEC8DF0C3
:10B08C00100E816E100E816E36EC91F000008A6A03
:10B09C004CECB0F0000000008A6AC7ECB8F000007D
:10B0AC008A6A9CEC91F0100E816E080E816EECECAD
:10B0BC008DF0100E816E100E816E36EC91F000004A
:10B0CC008A6A4CECB0F0000000008A6AC7ECB8F059
:10B0DC0000008A6A9CEC91F0100E816E080E816E55
:10B0EC0061EC8EF0100E816E100E816E36EC91F0CC
:10B0FC0000008A6A4CECB0F0000000008A6AC7ECD1
:10B10C00B8F000008A6A9CEC91F0100E816E080E6B
:10B11C00816ED6EC8EF0100E816E100E816E36ECB8
:10B12C0091F000008A6A4CECB0F0000000008A6AD2
:10B13C00C7ECB8F000008A6A9CEC91F0100E816E9E
:10B14C00080E816E4FEC8FF0100E816E100E816E1A
:10B15C0036EC91F000008A6A4CECB0F00000000074
:10B16C008A6AC7ECB8F000008A6A4CECB0F00000B8
:10B17C000000100E816E97ECB0F000008A6A56EC5D
:10B18C00B0F00000100E816E00008A6A56ECB0F030
:10B19C000000100E816E100E816ED1EC8FF0100E2F
:10B1AC00816E100E816E56ECB0F0000000008A6AC1
:10B1BC00100E816E56ECB0F00000100E816E97EC04
:10B1CC00B0F00000000000008A6A4CECB0F0000007
:10B1DC0000008A6AC7ECB8F000008A6A9CEC91F017
:10B1EC00100E816E080E816E4EEC90F0100E816E7A
:10B1FC00100E816E36EC91F000008A6A4CECB0F0C7
:10B20C00000000008A6AC7ECB8F000008A6A9CEC67
:10B21C0091F0100E816E080E816ECBEC90F0100E3A
:10B22C00816E100E816E36EC91F000008A6A4CEC47
:10B23C00B0F0000000008A6AC7ECB8F000008A6A1F
:10B24C009CEC91F0100E816E080E816EDAEC8BF096
:10B25C00100E816E100E816E36EC91F000008A6A31
:10B26C004CECB0F0000000008A6AC7ECB8F00000AB
:10B27C008A6A9CEC91F0100E816E080E816E18ECAF
:10B28C008CF0100E816E100E816E36EC91F0000079
:10B29C008A6A4CECB0F0000000008A6AC7ECB8F087
:10B2AC0000008A6A9CEC91F0100E816E080E816E83
:10B2BC00CAEC8CF0100E816E100E816E36EC91F093
:10B2CC0000008A6A4CECB0F0000000008A6AC7ECFF
:10B2DC00B8F0100E816E9CEC91F0100E816E080E81
:10B2EC00816E6FECB0F00000C2ECB0F08A6A000026
:10B2FC000000000000008A88A1ECB0F08A425BECF0
:10B30C00B0F0100E816EF6EC7CF08A42BEECB0F020
:10B31C008A6A6AECB0F000008A86BEECB0F0100EBF
:10B32C00816E93EC7CF08A425BECB0F08A46A1EC27
:10B33C00B0F08A6A00000000000000008A86BEECB3
:10B34C00B0F06FECB0F00000100E816E100E816E3C
:10B35C0036EC91F0100E816E4CECB0F00000000059
:10B36C008A6AC7ECB8F0100E816E9CEC91F0100E4E
:10B37C00816E080E816E6FECB0F00000C7ECB0F07F
:10B38C008A6A00000000000000008A88A1ECB0F07E
:10B39C008A4256ECB0F000000000100E816EF6EC04
:10B3AC007CF08A42BEECB0F08A6A6AECB0F0000025
:10B3BC008A86BEECB0F0100E816E93EC7CF08A4263
:10B3CC0056ECB0F0000000008A46A1ECB0F08A6A9E
:10B3DC0000000000000000008A86C2ECB0F06FECA8
:10B3EC00B0F00000100E816E100E816E36EC91F0F4
:10B3FC00100E816E4CECB0F0000000008A6AC7ECB5
:10B40C00B8F0100E816E9CEC91F0100E816E080E4F
:10B41C00816E6FECB0F0000045ECB0F08A6A000071
:10B42C000000000000008A88A1ECB0F08A4256ECC3
:10B43C00B0F00000100E816EF6EC7CF08A42BEEC8F
:10B44C00B0F08A6A6AECB0F000008A86BEECB0F00C
:10B45C00100E816E93EC7CF08A4256ECB0F000003A
:10B46C008A46A1ECB0F08A6A0000000000000000DF
:10B47C008A86C7ECB0F06FECB0F00000100E816E55
:10B48C00100E816E36EC91F0100E816E4CECB0F01B
:10B49C00000000008A6AC7ECB8F0100E816E9CECBC
:10B4AC0091F0100E816E080E816E6FECB0F0000002
:10B4BC0045ECB0F08A6AA1ECB0F08A88A1ECB0F04F
:10B4CC008A4256ECB0F0100E816EF6EC7CF08A429B
:10B4DC00BEECB0F08A6A6AECB0F000008A86BEEC72
:10B4EC00B0F0100E816E93EC7CF08A4256ECB0F00A
:10B4FC008A46A1ECB0F08A6AA1ECB0F08A86C7EC5F
:10B50C00B0F06FECB0F00000100E816E100E816E7A
:10B51C0036EC91F0100E816E4CECB0F00000000097
:10B52C008A6AC7ECB8F0100E816E9CEC91F0100E8C
:10B53C00816E080E816E6FECB0F000004CECB0F038
:10B54C0000008A6A00000000000000008A88A1EC5C
:10B55C00B0F08A4251ECB0F000000000100E816E89
:10B56C00F6EC7CF08A42BEECB0F08A6A6AECB0F081
:10B57C0000008A86BEECB0F0100E816E93EC7CF06D
:10B58C008A4251ECB0F0000000008A46A1ECB0F009
:10B59C008A6A00000000000000008A864CECB0F0C3
:10B5AC006FECB0F00000100E816E100E816E36EC58
:10B5BC0091F0100E816E4CECB0F0000000008A6A25
:10B5CC00C7ECB8F0100E816E9CEC91F0100E816EF1
:10B5DC00080E816E6FECB0F000004CECB0F0000087
:10B5EC0000008A6A00000000000000008A88A1ECBC
:10B5FC00B0F08A4251ECB0F00000100E816EF6EC07
:10B60C007CF08A42BEECB0F08A6A6AECB0F00000C2
:10B61C008A86BEECB0F0100E816E93EC7CF08A4200
:10B62C0051ECB0F000008A46A1ECB0F08A6A000040
:10B63C000000000000008A864CECB0F000006FECBB
:10B64C00B0F00000100E816E100E816E36EC91F091
:10B65C00100E816E4CECB0F0000000008A6AC7EC52
:10B66C00B8F0100E816EB9EC91F0100E816E080ED0
:10B67C00816E6FECB0F0000051ECB0F08A6AA1EC76
:10B68C00B0F08A88A1ECB0F08A424CECB0F000002B
:10B69C000000100E816EF6EC7CF08A42BEECB0F02D
:10B6AC008A6A6AECB0F000008A86BEECB0F0100E2C
:10B6BC00816E93EC7CF08A424CECB0F00000000000
:10B6CC008A46A1ECB0F08A6AA1ECB0F08A864CEC08
:10B6DC00B0F0000000006FECB0F00000100E816EB6
:10B6EC00100E816E4FEC91F0100E816E4CECB0F0A0
:10B6FC00000000008A6AC7ECB8F0100E816EB9EC3D
:10B70C0091F0100E816E080E816E6FECB0F000009F
:10B71C0051ECB0F000008A6AA1ECB0F08A88A1EC80
:10B72C00B0F08A424CECB0F00000100E816EF6ECDA
:10B73C007CF08A42BEECB0F08A6A6AECB0F0000091
:10B74C008A86BEECB0F0100E816E93EC7CF08A42CF
:10B75C004CECB0F000008A46A1ECB0F08A6AA1EC87
:10B76C00B0F08A8651ECB0F06FECB0F00000100E27
:10B77C00816E100E816E4FEC91F0100E816E4CECC0
:10B78C00B0F0000000008A6AC7ECB8F0100E816EB1
:10B79C00B9EC91F0100E816E080E816E6FECB0F06A
:10B7AC0000004CECB0F08A4600008A420000000019
:10B7BC008A6AA1ECB0F08A88B2ECB0F08A4245EC0F
:10B7CC00B0F0100E816EF6EC7CF08A42BEECB0F05C
:10B7DC008A6A6AECB0F000008A86BEECB0F0100EFB
:10B7EC00816E93EC7CF08A4245ECB0F08A46B2EC68
:10B7FC00B0F08A6AA1ECB0F08A86000000008A469C
:10B80C0000008A4245ECB0F06FECB0F00000100E76
:10B81C00816E100E816E4FEC91F0100E816E4CEC1F
:10B82C00B0F0000000008A6AC7ECB8F0100E816E10
:10B83C00B9EC91F0100E816E080E816E6FECB0F0C9
:10B84C0000004CECB0F08A4600008A420000000078
:10B85C00000000008A6AA1ECB0F08A88A1ECB0F07C
:10B86C008A42C7ECB0F0100E816EF6EC7CF08A4286
:10B87C00BEECB0F08A6A6AECB0F000008A86BEECCE
:10B88C00B0F0100E816E93EC7CF08A42C7ECB0F0F5
:10B89C008A46A1ECB0F08A6AA1ECB0F08A8600006E
:10B8AC000000000000008A4600008A4245ECB0F01F
:10B8BC006FECB0F00000100E816E100E816E4FEC2C
:10B8CC0091F0100E816E4CECB0F0000000008A6A12
:10B8DC00C7ECB8F0100E816EB9EC91F0100E816EC1
:10B8EC00080E816E6FECB0F000004CECB0F08A46A4
:10B8FC0000008A42A1ECB0F08A6AA1ECB0F08A8810
:10B90C00B2ECB0F08A42BEECB0F0100E816EF6ECE8
:10B91C007CF08A42BEECB0F08A6A6AECB0F00000AF
:10B92C008A86BEECB0F0100E816E93EC7CF08A42ED
:10B93C00BEECB0F08A46B2ECB0F08A6AA1ECB0F082
:10B94C008A86A1ECB0F08A4600008A4245ECB0F041
:10B95C006FECB0F00000100E816E100E816E4FEC8B
:10B96C0091F0100E816E4CECB0F0000000008A6A71
:10B97C00C7ECB8F0100E816EB9EC91F0100E816E20
:10B98C00080E816E6FECB0F000004CECB0F08A4603
:10B99C0000008A42B2ECB0F08A6AB2ECB0F08A884D
:10B9AC00B2ECB0F08A42A1ECB0F0100E816EF6EC65
:10B9BC007CF08A42BEECB0F08A6A6AECB0F000000F
:10B9CC008A86BEECB0F0100E816E93EC7CF08A424D
:10B9DC00A1ECB0F08A46B2ECB0F08A6AB2ECB0F0EE
:10B9EC008A86B2ECB0F08A4600008A4245ECB0F090
:10B9FC006FECB0F00000100E816E100E816E4FECEB
:10BA0C0091F0100E816E4CECB0F0000000008A6AD0
:10BA1C00C7ECB8F000008A6A00005FEC91F0100EE1
:10BA2C00816E080E816E6FECB0F000004CECB0F043
:10BA3C008A4600008A42C2ECB0F08A6AB2ECB0F0DE
:10BA4C008A88B2ECB0F08A42000000000000100EB0
:10BA5C00816EF6EC7CF08A428DECB0F000000000B8
:10BA6C00100E816E93EC7CF08A4200000000000006
:10BA7C008A46B2ECB0F08A6AB2ECB0F08A86C2ECBC
:10BA8C00B0F08A4600008A4245ECB0F06FECB0F0A2
:10BA9C000000100E816E100E816E09EC91F000000A
:10BAAC0000008A6A4CECB0F0000000008A6AC7EC17
:10BABC00B8F000008A6A00005FEC91F0100E816E05
:10BACC00080E816E6FECB0F000004CECB0F08A46C2
:10BADC0000008A4245ECB0F08A6AB2ECB0F08A8879
:10BAEC00B2ECB0F08A420000100E816EF6EC7CF0E5
:10BAFC008A428DECB0F000000000100E816E93ECC9
:10BB0C007CF08A4200008A46B2ECB0F08A6AB2EC51
:10BB1C00B0F08A8645ECB0F08A4600008A4245ECCB
:10BB2C00B0F06FECB0F00000100E816E100E816E54
:10BB3C0009EC91F0000000008A6A4CECB0F00000B7
:10BB4C0000008A6AC7ECB8F000008A6A00005FEC5B
:10BB5C0091F0100E816E080E816E6FECB0F000004B
:10BB6C004CECB0F08A4600008A424CECB0F000007D
:10BB7C008A6AB2ECB0F08A88B2ECB0F0100E816E2A
:10BB8C00F6EC7CF08A428DECB0F000000000100E58
:10BB9C00816E93EC7CF08A88B2ECB0F08A6AB2ECDD
:10BBAC00B0F08A864CECB0F000008A4600008A4265
:10BBBC0045ECB0F06FECB0F00000100E816E100E82
:10BBCC00816E09EC91F0000000008A6A4CECB0F038
:10BBDC00000000008A6AC7ECB8F000008A6A000016
:10BBEC005FEC91F0100E816E080E816E6FECB0F070
:10BBFC0000004CECB0F08A4600008A424CECB0F0ED
:10BC0C00000000008A6ABEECB0F08A8800000000D8
:10BC1C0000000000100E816EF6EC7CF08A428DEC78
:10BC2C00B0F000000000100E816E93EC7CF08A885E
:10BC3C0000000000000000008A6ABEECB0F08A86AA
:10BC4C004CECB0F0000000008A4600008A4245EC43
:10BC5C00B0F06FECB0F00000100E816E100E816E23
:10BC6C0009EC91F0000000008A6A4CECB0F0000086
:10BC7C0000008A6AC7ECB8F000008A6A00005FEC2A
:10BC8C0091F0100E816E080E816E6FECB0F000001A
:10BC9C004CECB0F08A4600008A4251ECB0F0000047
:10BCAC008A6ABEECB0F08A8800000000100E816E2B
:10BCBC00F6EC7CF08A428DECB0F000000000100E27
:10BCCC00816E93EC7CF08A88000000008A6ABEECDE
:10BCDC00B0F08A8651ECB0F000008A4600008A422F
:10BCEC0045ECB0F06FECB0F00000100E816E100E51
:10BCFC00816E09EC91F0000000008A6A4CECB0F007
:10BD0C00000000008A6AC7ECB8F000008A6A0000E4
:10BD1C005FEC91F0100E816E080E816E6FECB0F03E
:10BD2C0000004CECB0F08A4600008A4256ECB0F0B1
:10BD3C0000008A6AB2ECB0F08A88100E816E7EEC3C
:10BD4C00B0F000008A428DECB0F000000000100E44
:10BD5C00816E7EECB0F000008A888A6AB2ECB0F09A
:10BD6C008A8656ECB0F000008A4600008A4245EC08
:10BD7C00B0F06FECB0F00000100E816E100E816E02
:10BD8C0009EC91F0000000008A6A4CECB0F0000065
:10BD9C0000008A6AC7ECB8F000008A6A4CECB0F07C
:10BDAC0000000000100E816E97ECB0F00000000057
:10BDBC0000008DECB0F0100E816E6FECB0F0000056
:10BDCC006FECB0F0000000008A42000000008A6AAC
:10BDDC00BEECB0F08A88C2ECB0F08A4297ECB0F0BE
:10BDEC0000000000000097ECB0F08A46C2ECB0F006
:10BDFC008A6ABEECB0F08A86000000008A4651ECDC
:10BE0C00B0F00000000051ECB0F06FECB0F00000AE
:10BE1C00100E816E97ECB0F00000000000008DEC6D
:10BE2C00B0F00000000000008A6A4CECB0F000009A
:10BE3C0000008A6AC7ECB8F000008A6A000085EC42
:10BE4C0091F0100E816E080E816E6FECB0F0000058
:10BE5C004CECB0F08A4600008A425BECB0F000007B
:10BE6C0000008A6AC2ECB0F08A88C2ECB0F08A4258
:10BE7C0097ECB0F00000000000008DECB0F08A46AA
:10BE8C00C2ECB0F08A6AC2ECB0F08A865BECB0F01F
:10BE9C00000000008A4600008A4245ECB0F06FECCE
:10BEAC00B0F00000100E816E080E816E27EC91F040
:10BEBC00000000008A6A4CECB0F0000000008A6AB6
:10BECC00C7ECB8F000008A6A000085EC91F0100E07
:10BEDC00816E080E816E6FECB0F000004CECB0F08F
:10BEEC008A4600008A4265ECB0F0000000008A6AC5
:10BEFC00BEECB0F08A8845ECB0F08A4297ECB0F01A
:10BF0C0000000000000079ECB0F000008A4645EC1F
:10BF1C00B0F08A6ABEECB0F08A8665ECB0F0000036
:10BF2C0000008A4600008A4245ECB0F06FECB0F09D
:10BF3C000000100E816E080E816E27EC91F000004F
:10BF4C0000008A6A4CECB0F0000000008A6AC7EC72
:10BF5C00B8F000008A6A000085EC91F0100E816E3A
:10BF6C00080E816E6FECB0F000004CECB0F08A461D
:10BF7C0000008A426AECB0F000008A6AC2ECB0F0B1
:10BF8C008A8845ECB0F08A4297ECB0F000000000D3
:10BF9C0000006AECB0F000008A4645ECB0F08A6A0A
:10BFAC00C2ECB0F08A866AECB0F000008A46000061
:10BFBC008A4245ECB0F06FECB0F00000100E816ED0
:10BFCC00080E816E27EC91F0000000008A6A4CECA0
:10BFDC00B0F0000000008A6AC7ECB8F000008A6A72
:10BFEC00000085EC91F0100E816E080E816E6FECE6
:10BFFC00B0F000004CECB0F08A4600008A426FECC6
:10C00C00B0F000008A6AC7ECB0F08A884CECB0F053
:10C01C008A4297ECB0F000000000000056ECB0F043
:10C02C008A464CECB0F08A6AC7ECB0F08A866FECAA
:10C03C00B0F000008A4600008A4245ECB0F06FEC8C
:10C04C00B0F00000100E816E080E816E27EC91F09E
:10C05C00000000008A6A4CECB0F0000000008A6A14
:10C06C00C7ECB8F000008A6A000085EC91F0100E65
:10C07C00816E080E816E6FECB0F000004CECB0F0ED
:10C08C008A4600008A4279ECB0F000008A6A45ECDE
:10C09C00B0F08A884CECB0F0000000008A4297ECBB
:10C0AC00B0F0000000000000A1ECB0F08A464CECAF
:10C0BC00B0F0000000008A6A45ECB0F08A8679EC9A
:10C0CC00B0F000008A4600008A4245ECB0F06FECFC
:10C0DC00B0F00000100E816E080E816E27EC91F00E
:10C0EC00000000008A6A4CECB0F0000000008A6A84
:10C0FC00C7ECB8F0100E816E000085EC91F0100EBC
:10C10C00816E080E816E6FECB0F000004CECB0F05C
:10C11C008A4600008A427EECB0F0000000008A6A79
:10C12C0045ECB0F08A8851ECB0F0000000008A4277
:10C13C008DECB0F08A4651ECB0F0000000008A6A39
:10C14C0045ECB0F08A867EECB0F0000000008A4628
:10C15C0000008A4245ECB0F06FECB0F00000100E1D
:10C16C00816E080E816E27EC91F00000100E816E2E
:10C17C004CECB0F0000000008A6AC7ECB8F0100E6E
:10C18C00816E000085EC91F0100E816E080E816EB0
:10C19C006FECB0F000004CECB0F08A4600008A4224
:10C1AC008DECB0F08A6A4CECB0F000008A885BEC45
:10C1BC00B0F0000000008A4256ECB0F08A465BEC0E
:10C1CC00B0F0000000008A6A4CECB0F000008A86E7
:10C1DC008DECB0F08A4600008A4245ECB0F06FEC72
:10C1EC00B0F00000100E816E080E816E27EC91F0FD
:10C1FC000000100E816E4CECB0F0000000008A6A5A
:10C20C00C7ECB8F0100E816E76EC91F0100E816ECA
:10C21C00080E816E51ECB0F00000100E816E000023
:10C22C000000080E816E56ECB0F000000000100EFD
:10C23C00816E080E816E6FECB0F000004CECB0F02B
:10C24C008A4600008A4292ECB0F000008A6A4CECFC
:10C25C00B0F0000000008A88000097ECB0F00000FD
:10C26C0000000000000000008A6A4CECB0F00000F6
:10C27C0000008A8692ECB0F000008A4600008A42E8
:10C28C0045ECB0F06FECB0F00000100E816E080EB3
:10C29C00816E5BECB0F00000100E816E00000000AF
:10C2AC00080E816E4CECB0F000000000100E816E98
:10C2BC00080E816E18EC91F000008A6AC7ECB8F099
:10C2CC00100E816E76EC91F0100E816E080E816E60
:10C2DC004CECB0F00000100E816E7CECBAF0100E3D
:10C2EC00816E080E816E51ECB0F000000000100E53
:10C2FC00816E080E816E6FECB0F000004CECB0F06B
:10C30C008A4600008A4297ECB0F000000000000062
:10C31C008A6A56ECB0F08A887EECB0F08A6A56ECE9
:10C32C00B0F08A8697ECB0F00000000000008A465E
:10C33C0000008A4245ECB0F06FECB0F00000100E3B
:10C34C00816E080E816E56ECB0F0000000008A463B
:10C35C00100E816E5EECBBF0080E816E45ECB0F0F9
:10C36C00100E816E080E816E18EC91F000008A6A36
:10C37C00C7ECB8F0100E816E76EC91F0100E816E59
:10C38C00080E816E45ECB0F0100E816E75ECBAF0B3
:10C39C00100E816E080E816E51ECB0F0100E816E95
:10C3AC00080E816E6FECB0F000004CECB0F08A46D9
:10C3BC0000008A428DECB0F08A4600008A424CECB8
:10C3CC00B0F08A6A97ECB0F00000000000004CEC72
:10C3DC00B0F08A864CECB0F08A4600008A428DECB4
:10C3EC00B0F08A4600008A4245ECB0F06FECB0F039
:10C3FC000000100E816E080E816E56ECB0F08A466D
:10C40C00100E816E57ECBBF0080E816EC2ECB0F0D2
:10C41C00100E816E080E816E18EC91F000008A6A85
:10C42C00C7ECB8F0100E816E76EC91F0100E816EA8
:10C43C00080E816EC2ECB0F0100E816E70ECBAF08A
:10C44C00100E816E080E816E4CECB0F00000100ED8
:10C45C00816E080E816E6FECB0F000004CECB0F009
:10C46C008A4600008A428DECB0F08A4600008A426F
:10C47C0056ECB0F0000000008A6A92ECB0F00000BC
:10C48C008A8656ECB0F0000000008A4600008A4212
:10C49C008DECB0F08A4600008A4245ECB0F06FECAF
:10C4AC00B0F00000100E816E080E816E51ECB0F0F1
:10C4BC0000008A46100E816E52ECBBF0080E816EA5
:10C4CC00B2ECB0F0100E816E080E816E18EC91F08B
:10C4DC0000008A6AC7ECB8F0100E816E76EC91F011
:10C4EC00100E816E080E816EB2ECB0F0100E816EE3
:10C4FC0067ECBAF0100E816E080E816E45ECB0F050
:10C50C00100E816E080E816E6FECB0F000004CECDA
:10C51C00B0F08A4600008A428DECB0F08A460000EA
:10C52C008A426FECB0F0000000008A6A5BECB0F05D
:10C53C0000008A866FECB0F0000000008A46000014
:10C54C008A428DECB0F08A4600008A4245ECB0F08D
:10C55C006FECB0F00000100E816E080E816E4CEC8A
:10C56C00B0F0000000008A46100E816E49ECBBF062
:10C57C00080E816E0000000000000000100E816E9D
:10C58C00080E816E18EC91F000008A6AC7ECB8F0C6
:10C59C00100E816E76EC91F0100E816E080E816E8D
:10C5AC000000000000000000100E816E5AECBAF082
:10C5BC00100E816E080E816EC2ECB0F0100E816E02
:10C5CC00080E816E83ECB0F000000000100E816E3E
:10C5DC00080E816E83ECB0F000000000100E816E2E
:10C5EC00080E816E92ECB0F083ECB0F0000000000D
:10C5FC00100E816E080E816E83ECB0F0000000000E
:10C60C00100E816E080E816E83ECB0F000000000FD
:10C61C00100E816E080E816E4CECB0F08A46100E36
:10C62C00816E3CECBBF0080E816E00000000100E19
:10C63C00816E080E816E18EC91F000008A6AC7ECCE
:10C64C00B8F0100E816E76EC91F0100E816E080E23
:10C65C00816E00000000100E816E55ECBAF0100EC9
:10C66C00816E080E816EB2ECB0F0100E816E080E69
:10C67C00816E01EC7EF0100E816E080E816EC7EC9F
:10C68C00B0F08A46100E816E37ECBBF0080E816E4E
:10C69C00100E816E080E816E18EC91F000008A6A03
:10C6AC00C7ECB8F0100E816E76EC91F0100E816E26
:10C6BC00080E816E100E816E4CECBAF0100E816E6D
:10C6CC00080E816E0000000000000000100E816E4C
:10C6DC00080E816E01EC7EF0100E816E080E816EDC
:10C6EC00BEECB0F08A46100E816E2EECBBF0100E34
:10C6FC00816E080E816E18EC91F000008A6AC7EC0E
:10C70C00B8F0100E816E76EC91F0100E816E100E5A
:10C71C00816E3FECBAF0100E816E080E816E000037
:10C72C000000100E816E080E816E01EC7EF0100E72
:10C73C00816E080E816EA1ECB0F08A46100E816EEF
:10C74C0021ECBBF0080E816E18EC91F000008A6AA7
:10C75C00C7ECB8F0100E816E76EC91F0100E816E75
:10C76C0034ECBAF0100E816E080E816E100E816ED4
:10C77C00080E816E01EC7EF0100E816E080E816E3B
:10C78C000000000000008A46100E816E16ECBBF013
:10C79C00080E816E83ECB0F0100E816E080E816E67
:10C7AC00000000000000100E816E4CECB0F0000098
:10C7BC0000008A6AE6EC91F00000000075ECB5F020
:10C7CC008DEF32F048ECAEF00E53D8A4E6D000005A
:10C7DC00BB0E8A6A0F6F0000000000008B9E8B86D8
:10C7EC0097ECB0F00000000000008B8E8B9697EC5D
:10C7FC00B0F000000000000003D08A6AC7ECB8F06B
:10C80C00080E816E97ECB0F0000000008A6AA1EC73
:10C81C00B0F0100E816E100E816EF6EC7CF0100EE6
:10C82C00816E00008A6AA1ECB0F0080E816E92EC69
:10C83C00B0F00000000000008A6AA1ECB0F0100E0D
:10C84C00816E100E816ED5EC7CF0100E816E0000A6
:10C85C008A6AA1ECB0F0080E816E92ECB0F0000088
:10C86C00000000008A6AA1ECB0F0100E816E100E70
:10C87C00816EB4EC7CF0100E816E00008A6AA1EC23
:10C88C00B0F0080E816E92ECB0F0000000000000D9
:10C89C008A6AA1ECB0F0100E816E0000100E816E51
:10C8AC0093EC7CF0000000008A6AA1ECB0F0080E5A
:10C8BC00816E97ECB0F0000000000000BEECB0F010
:10C8CC000F2F9BD700008A6AC7ECB8F0080E816E58
:10C8DC0097ECB0F0000000008A6AA1ECB0F0100EEA
:10C8EC00816E100E816EF6EC7CF0100E816E0000E5
:10C8FC008A6AA1ECB0F0080E816E92ECB0F00000E8
:10C90C00000000008A6AA1ECB0F0100E816E100ECF
:10C91C00816ED5EC7CF0100E816E00008A6AA1EC61
:10C92C00B0F0080E816E92ECB0F000000000000038
:10C93C008A6AA1ECB0F0100E816E100E816EB4EC10
:10C94C007CF0100E816E00008A6AA1ECB0F0080E2B
:10C95C00816E92ECB0F00000000000008A6AA1EC3D
:10C96C00B0F0100E816E0000100E816E93EC7CF016
:10C97C00000000008A6AA1ECB0F0080E816E97EC02
:10C98C00B0F0000000000000000082A05CEF78F026
:10C99C0082A26CEF6FF08A6AE1D0BB0E8A6A0F6FCD
:10C9AC000000000000008B9E8B8697ECB0F000001E
:10C9BC00000000008B8E8B9697ECB0F0000000000E
:10C9CC00000003D08A6AC7ECB8F0080E816E97ECB1
:10C9DC00B0F0000000008A6AA1ECB0F0100E816E7D
:10C9EC00100E816EF6EC7CF0100E816E00008A6ADF
:10C9FC00A1ECB0F0080E816E92ECB0F000000000DB
:10CA0C0000008A6AA1ECB0F0100E816E100E816EDF
:10CA1C00D5EC7CF0100E816E00008A6AA1ECB0F0AF
:10CA2C00080E816E92ECB0F00000000000008A6AE3
:10CA3C00A1ECB0F0100E816E100E816EB4EC7CF097
:10CA4C00100E816E00008A6AA1ECB0F0080E816EA7
:10CA5C0092ECB0F00000000000008A6AA1ECB0F08B
:10CA6C00100E816E0000100E816E93EC7CF00000B5
:10CA7C0000008A6AA1ECB0F0080E816E97ECB0F061
:10CA8C00000000000000BEECB0F00F2F9BD70000A0
:10CA9C008A6AC7ECB8F0080E816E97ECB0F0000013
:10CAAC0000008A6AA1ECB0F0100E816E100E816E3F
:10CABC00F6EC7CF0100E816E00008A6AA1ECB0F0EE
:10CACC00080E816E92ECB0F00000000000008A6A43
:10CADC00A1ECB0F0100E816E100E816ED5EC7CF0D6
:10CAEC00100E816E00008A6AA1ECB0F0080E816E07
:10CAFC0092ECB0F00000000000008A6AA1ECB0F0EB
:10CB0C00100E816E100E816EB4EC7CF0100E816EE6
:10CB1C0000008A6AA1ECB0F0080E816E92ECB0F0C5
:10CB2C000000000000008A6AA1ECB0F0100E816ECB
:10CB3C000000100E816E93EC7CF0000000008A6AFD
:10CB4C00A1ECB0F0080E816E97ECB0F00000000084
:10CB5C000000BEECB0F08A6A0000000075ECB5F085
:10CB6C0033D648ECAEF00E53D8A4B1D00000BB0EB7
:10CB7C008A6A0F6F0000000000008B9E8B8697EC7A
:10CB8C00B0F00000000000008B8E8B9697ECB0F09C
:10CB9C0000000000000003D08A6AC7ECB8F065EC16
:10CBAC00B0F0000000006FECB0F0000000008A2A2A
:10CBBC008A2A65ECB0F0000000006AECB0F08A2A1A
:10CBCC008A2A65ECB0F0000000006AECB0F08A2A0A
:10CBDC008A2A65ECB0F0000000006AECB0F08A2AFA
:10CBEC008A2A65ECB0F0000000006AECB0F08A2AEA
:10CBFC008A2A65ECB0F0000000006AECB0F08A2ADA
:10CC0C008A2A65ECB0F0000000006AECB0F08A2AC9
:10CC1C008A2A65ECB0F0000000006AECB0F08A2AB9
:10CC2C008A2A65ECB0F00000000065ECB0F00F2F24
:10CC3C00B3D700008A6AC7ECB8F065ECB0F000001E
:10CC4C0000006FECB0F0000000008A2A8A2A65EC24
:10CC5C00B0F0000000006AECB0F08A2A8A2A65EC79
:10CC6C00B0F0000000006AECB0F08A2A8A2A65EC69
:10CC7C00B0F0000000006AECB0F08A2A8A2A65EC59
:10CC8C00B0F0000000006AECB0F08A2A8A2A65EC49
:10CC9C00B0F0000000006AECB0F08A2A8A2A65EC39
:10CCAC00B0F0000000006AECB0F08A2A8A2A65EC29
:10CCBC00B0F0000000006AECB0F08A2A8A2A65EC19
:10CCCC00B0F00000000065ECB0F08A6AB6D0BB0E84
:10CCDC008A6A0F6F0000000000008B9E8B8697EC19
:10CCEC00B0F00000000000008B8E8B9697ECB0F03B
:10CCFC0000000000000003D08A6AC7ECB8F065ECB5
:10CD0C00B0F0000000006FECB0F0000000008A2AC8
:10CD1C008A2A65ECB0F0000000006AECB0F08A2AB8
:10CD2C008A2A65ECB0F0000000006AECB0F08A2AA8
:10CD3C008A2A65ECB0F0000000006AECB0F08A2A98
:10CD4C008A2A65ECB0F0000000006AECB0F08A2A88
:10CD5C008A2A65ECB0F0000000006AECB0F08A2A78
:10CD6C008A2A65ECB0F0000000006AECB0F08A2A68
:10CD7C008A2A65ECB0F0000000006AECB0F08A2A58
:10CD8C008A2A65ECB0F00000000065ECB0F00F2FC3
:10CD9C00B3D700008A6AC7ECB8F065ECB0F00000BD
:10CDAC0000006FECB0F0000000008A2A8A2A65ECC3
:10CDBC00B0F0000000006AECB0F08A2A8A2A65EC18
:10CDCC00B0F0000000006AECB0F08A2A8A2A65EC08
:10CDDC00B0F0000000006AECB0F08A2A8A2A65ECF8
:10CDEC00B0F0000000006AECB0F08A2A8A2A65ECE8
:10CDFC00B0F0000000006AECB0F08A2A8A2A65ECD8
:10CE0C00B0F0000000006AECB0F08A2A8A2A65ECC7
:10CE1C00B0F0000000006AECB0F08A2A8A2A56ECC6
:10CE2C00B0F00000000082A00BD082A28BEF32F099
:10CE3C0065ECB0F08A6A0000000075ECB5F093D692
:10CE4C0048ECAEF00E53D8A48DD00000BB0E8A6A0D
:10CE5C000F6F0000000000008B9E8B8697ECB0F0EB
:10CE6C000000000000008B8E8B9697ECB0F0000059
:10CE7C000000000003D08A6AC7ECB8F08A8897ECEF
:10CE8C00B0F08A6A97ECB0F08A2A8A2A92ECB0F059
:10CE9C00000000008A2A8A2A92ECB0F00000000000
:10CEAC008A2A8A2A92ECB0F0000000008A2A8A2A88
:10CEBC0092ECB0F0000000008A2A8A2A92ECB0F0C2
:10CECC00000000008A2A8A2A92ECB0F000000000D0
:10CEDC008A2A8A2A92ECB0F0000000008A2A8A2A58
:10CEEC008DECB0F0000000000F2FC5D700008A6A4F
:10CEFC00C7ECB8F08A8897ECB0F08A6A97ECB0F07F
:10CF0C008A2A8A2A92ECB0F0000000008A2A8A2A27
:10CF1C0092ECB0F0000000008A2A8A2A92ECB0F061
:10CF2C00000000008A2A8A2A92ECB0F0000000006F
:10CF3C008A2A8A2A92ECB0F0000000008A2A8A2AF7
:10CF4C0092ECB0F0000000008A2A8A2A92ECB0F031
:10CF5C00000000008A2A8A2A8DECB0F00000000044
:10CF6C008A6A91D0BB0E8A6A0F6F00000000000025
:10CF7C008B9E8B8697ECB0F00000000000008B8E2F
:10CF8C008B9697ECB0F000000000000003D08A6A8A
:10CF9C00C7ECB8F08A8897ECB0F08A6A97ECB0F0DE
:10CFAC008A2A8A2A92ECB0F0000000008A2A8A2A87
:10CFBC0092ECB0F0000000008A2A8A2A92ECB0F0C1
:10CFCC00000000008A2A8A2A92ECB0F000000000CF
:10CFDC008A2A8A2A92ECB0F0000000008A2A8A2A57
:10CFEC0092ECB0F0000000008A2A8A2A92ECB0F091
:10CFFC00000000008A2A8A2A8DECB0F000000000A4
:10D00C000F2FC5D700008A6AC7ECB8F08A8897EC56
:10D01C00B0F08A6A97ECB0F08A2A8A2A92ECB0F0C7
:10D02C00000000008A2A8A2A92ECB0F0000000006E
:10D03C008A2A8A2A92ECB0F0000000008A2A8A2AF6
:10D04C0092ECB0F0000000008A2A8A2A92ECB0F030
:10D05C00000000008A2A8A2A92ECB0F0000000003E
:10D06C008A2A8A2A92ECB0F0000000008A2A8A2AC6
:10D07C007EECB0F0000000008A6A82A007D082A289
:10D08C0070D50000000075ECB5F0DCD648ECAEF0C5
:10D09C000E53D8A404D000005BECB4F004D05BECCD
:10D0AC00B4F00000000075ECB5F0F2D748ECAEF02F
:10D0BC000E53D8A476D100008A6AA1ECB0F08B9EF6
:10D0CC008B8697ECB0F00000000000008B8E8B96E6
:10D0DC0097ECB0F0000000000000000000008A6A2D
:10D0EC0065ECB0F08A8800008A6A92ECB0F000001F
:10D0FC008A8800008A6A92ECB0F000008A880000EE
:10D10C008A6A92ECB0F000008A8800008A6A92EC7D
:10D11C00B0F000008A8800008A6A92ECB0F000003F
:10D12C008A8800008A6A92ECB0F000008A880000BD
:10D13C008A6A92ECB0F000008A8800008A6A92EC4D
:10D14C00B0F000008A8800008A6A92ECB0F000000F
:10D15C008A8800008A6A5BECB0F065ECAEF00000E7
:10D16C008A6AC7ECB8F08A6A4CECB0F000008A8886
:10D17C0088ECB0F00000000097ECB0F0000000006C
:10D18C0000000000000000008A6A45ECB0F08A6ADA
:10D19C0004ECAFF000008A6AC7ECB8F08A6A4CEC79
:10D1AC00B0F000008A8888ECB0F00000000097EC2A
:10D1BC00B0F00000000000000000000000008A6ACF
:10D1CC0045ECB0F08A6A04ECAFF000008A6AC7EC58
:10D1DC00B8F08A6A4CECB0F000008A8888ECB0F0A9
:10D1EC000000000097ECB0F0000000000000000010
:10D1FC00000000008A6A45ECB0F08A6A04ECAFF0DB
:10D20C0000008A6AC7ECB8F08A6A4CECB0F00000F7
:10D21C008A8888ECB0F00000000097ECB0F00000B9
:10D22C00000000000000000000008A6A45ECB0F02D
:10D23C008A6A04ECAFF000008A6AC7ECB8F08A6A1C
:10D24C004CECB0F000008A8888ECB0F000000000D4
:10D25C0097ECB0F00000000000000000000000009F
:10D26C008A6A45ECB0F08A6A04ECAFF000008A6A76
:10D27C00C7ECB8F08A6A4CECB0F000008A8888ECF5
:10D28C00B0F00000000097ECB0F0000000000000CF
:10D29C000000000000008A6A45ECB0F08A6A04ECD9
:10D2AC00AFF000008A6AC7ECB8F08A6A4CECB0F0B8
:10D2BC0000008A8888ECB0F00000000097ECB0F019
:10D2CC000000000000000000000000008A6A45EC2D
:10D2DC00B0F08A6A04ECAFF000008A6AC7ECB8F0D0
:10D2EC008A6A4CECB0F000008A8888ECB0F0000040
:10D2FC00000097ECB0F000000000000000000000FF
:10D30C0000008A6A45ECB0F08A6A65ECAEF0000069
:10D31C008A6AC7ECB8F08A6A65ECB0F08A880000BB
:10D32C008A6A92ECB0F000008A8800008A6A92EC5B
:10D33C00B0F000008A8800008A6A92ECB0F000001D
:10D34C008A8800008A6A92ECB0F000008A8800009B
:10D35C008A6A92ECB0F000008A8800008A6A92EC2B
:10D36C00B0F000008A8800008A6A92ECB0F00000ED
:10D37C008A8800008A6A92ECB0F000008A8800006B
:10D38C008A6A92ECB0F000008A8800008A6A4CEC41
:10D39C00B0F00000000082A07DD182A26DEF71F090
:10D3AC0076D18A6AA1ECB0F08B9E8B8697ECB0F0AC
:10D3BC000000000000008B8E8B9697ECB0F0000004
:10D3CC0000000000000000008A6A65ECB0F08A885A
:10D3DC0000008A6A92ECB0F000008A8800008A6A29
:10D3EC0092ECB0F000008A8800008A6A92ECB0F0EF
:10D3FC0000008A8800008A6A92ECB0F000008A88EB
:10D40C0000008A6A92ECB0F000008A8800008A6AF8
:10D41C0092ECB0F000008A8800008A6A92ECB0F0BE
:10D42C0000008A8800008A6A92ECB0F000008A88BA
:10D43C0000008A6A92ECB0F000008A8800008A6AC8
:10D44C005BECB0F065ECAEF000008A6AC7ECB8F0AB
:10D45C008A6A4CECB0F000008A8888ECB0F00000CE
:10D46C00000097ECB0F0000000000000000000008D
:10D47C0000008A6A45ECB0F08A6A04ECAFF0000058
:10D48C008A6AC7ECB8F08A6A4CECB0F000008A8863
:10D49C0088ECB0F00000000097ECB0F00000000049
:10D4AC0000000000000000008A6A45ECB0F08A6AB7
:10D4BC0004ECAFF000008A6AC7ECB8F08A6A4CEC56
:10D4CC00B0F000008A8888ECB0F00000000097EC07
:10D4DC00B0F00000000000000000000000008A6AAC
:10D4EC0045ECB0F08A6A04ECAFF000008A6AC7EC35
:10D4FC00B8F08A6A4CECB0F000008A8888ECB0F086
:10D50C000000000097ECB0F00000000000000000EC
:10D51C00000000008A6A45ECB0F08A6A04ECAFF0B7
:10D52C0000008A6AC7ECB8F08A6A4CECB0F00000D4
:10D53C008A8888ECB0F00000000097ECB0F0000096
:10D54C00000000000000000000008A6A45ECB0F00A
:10D55C008A6A04ECAFF000008A6AC7ECB8F08A6AF9
:10D56C004CECB0F000008A8888ECB0F000000000B1
:10D57C0097ECB0F00000000000000000000000007C
:10D58C008A6A45ECB0F08A6A04ECAFF000008A6A53
:10D59C00C7ECB8F08A6A4CECB0F000008A8888ECD2
:10D5AC00B0F00000000097ECB0F0000000000000AC
:10D5BC000000000000008A6A45ECB0F08A6A04ECB6
:10D5CC00AFF000008A6AC7ECB8F08A6A4CECB0F095
:10D5DC0000008A8888ECB0F00000000097ECB0F0F6
:10D5EC000000000000000000000000008A6A45EC0A
:10D5FC00B0F08A6A65ECAEF000008A6AC7ECB8F04D
:10D60C008A6A65ECB0F08A8800008A6A92ECB0F005
:10D61C0000008A8800008A6A92ECB0F000008A88C8
:10D62C0000008A6A92ECB0F000008A8800008A6AD6
:10D63C0092ECB0F000008A8800008A6A92ECB0F09C
:10D64C0000008A8800008A6A92ECB0F000008A8898
:10D65C0000008A6A92ECB0F000008A8800008A6AA6
:10D66C0092ECB0F000008A8800008A6A92ECB0F06C
:10D67C0000008A8800008A6A4CECB0F000000000C0
:10D68C0082A008D082A26DEF71F00000000075EC52
:10D69C00B5F00ED548ECAEF00E53D8A489D10000ED
:10D6AC008A6AA1ECB0F08B9E8B8697ECB0F00000F0
:10D6BC00000000008B8E8B9697ECB0F00000000001
:10D6CC000000000000008A6A8A865BECB0F0000063
:10D6DC0000008A4600008A4292ECB0F000008A46B4
:10D6EC0000008A4292ECB0F000008A4600008A42A8
:10D6FC0092ECB0F000008A4600008A4292ECB0F046
:10D70C0000008A4600008A4292ECB0F000008A4683
:10D71C0000008A4292ECB0F000008A4600008A4277
:10D72C0092ECB0F000008A4600008A4292ECB0F015
:10D73C0000008A4600008A4292ECB0F000008A4653
:10D74C0000008A4256ECB0F0000000008A6A00002B
:10D75C008A6AB4ECAEF000008A6AC7ECB8F08A6A48
:10D76C008A864CECB0F08A4688ECB0F000000000E1
:10D77C0097ECB0F00000000000000000000000007A
:10D78C008A424CECB0F000008A6A53ECAFF0000017
:10D79C008A6AC7ECB8F08A6A8A864CECB0F08A4682
:10D7AC0088ECB0F00000000097ECB0F00000000036
:10D7BC0000000000000000008A424CECB0F00000B9
:10D7CC008A6A53ECAFF000008A6AC7ECB8F08A6A38
:10D7DC008A864CECB0F08A4688ECB0F00000000071
:10D7EC0097ECB0F00000000000000000000000000A
:10D7FC008A424CECB0F000008A6A53ECAFF00000A7
:10D80C008A6AC7ECB8F08A6A8A864CECB0F08A4611
:10D81C0088ECB0F00000000097ECB0F000000000C5
:10D82C0000000000000000008A424CECB0F0000048
:10D83C008A6A53ECAFF000008A6AC7ECB8F08A6AC7
:10D84C008A864CECB0F08A4688ECB0F00000000000
:10D85C0097ECB0F000000000000000000000000099
:10D86C008A424CECB0F000008A6A53ECAFF0000036
:10D87C008A6AC7ECB8F08A6A8A864CECB0F08A46A1
:10D88C0088ECB0F00000000097ECB0F00000000055
:10D89C0000000000000000008A424CECB0F00000D8
:10D8AC008A6A53ECAFF000008A6AC7ECB8F08A6A57
:10D8BC008A864CECB0F08A4688ECB0F00000000090
:10D8CC0097ECB0F000000000000000000000000029
:10D8DC008A424CECB0F000008A6A53ECAFF00000C6
:10D8EC008A6AC7ECB8F08A6A8A864CECB0F08A4631
:10D8FC0088ECB0F00000000097ECB0F000000000E5
:10D90C0000000000000000008A424CECB0F0000067
:10D91C008A6AB4ECAEF000008A6AC7ECB8F08A6A86
:10D92C008A865BECB0F0000000008A4600008A4258
:10D93C0092ECB0F000008A4600008A4292ECB0F003
:10D94C0000008A4600008A4292ECB0F000008A4641
:10D95C0000008A4292ECB0F000008A4600008A4235
:10D96C0092ECB0F000008A4600008A4292ECB0F0D3
:10D97C0000008A4600008A4292ECB0F000008A4611
:10D98C0000008A4292ECB0F000008A4600008A4205
:10D99C0092ECB0F000008A4600008A424CECB0F0E9
:10D9AC0000008A6A82A090D182A25CEF68F089D1D3
:10D9BC008A6AA1ECB0F08B9E8B8697ECB0F00000DD
:10D9CC00000000008B8E8B9697ECB0F000000000EE
:10D9DC000000000000008A6A8A865BECB0F0000050
:10D9EC0000008A4600008A4292ECB0F000008A46A1
:10D9FC0000008A4292ECB0F000008A4600008A4295
:10DA0C0092ECB0F000008A4600008A4292ECB0F032
:10DA1C0000008A4600008A4292ECB0F000008A4670
:10DA2C0000008A4292ECB0F000008A4600008A4264
:10DA3C0092ECB0F000008A4600008A4292ECB0F002
:10DA4C0000008A4600008A4292ECB0F000008A4640
:10DA5C0000008A4256ECB0F0000000008A6A000018
:10DA6C008A6AB4ECAEF000008A6AC7ECB8F08A6A35
:10DA7C008A864CECB0F08A4688ECB0F000000000CE
:10DA8C0097ECB0F000000000000000000000000067
:10DA9C008A424CECB0F000008A6A53ECAFF0000004
:10DAAC008A6AC7ECB8F08A6A8A864CECB0F08A466F
:10DABC0088ECB0F00000000097ECB0F00000000023
:10DACC0000000000000000008A424CECB0F00000A6
:10DADC008A6A53ECAFF000008A6AC7ECB8F08A6A25
:10DAEC008A864CECB0F08A4688ECB0F0000000005E
:10DAFC0097ECB0F0000000000000000000000000F7
:10DB0C008A424CECB0F000008A6A53ECAFF0000093
:10DB1C008A6AC7ECB8F08A6A8A864CECB0F08A46FE
:10DB2C0088ECB0F00000000097ECB0F000000000B2
:10DB3C0000000000000000008A424CECB0F0000035
:10DB4C008A6A53ECAFF000008A6AC7ECB8F08A6AB4
:10DB5C008A864CECB0F08A4688ECB0F000000000ED
:10DB6C0097ECB0F000000000000000000000000086
:10DB7C008A424CECB0F000008A6A53ECAFF0000023
:10DB8C008A6AC7ECB8F08A6A8A864CECB0F08A468E
:10DB9C0088ECB0F00000000097ECB0F00000000042
:10DBAC0000000000000000008A424CECB0F00000C5
:10DBBC008A6A53ECAFF000008A6AC7ECB8F08A6A44
:10DBCC008A864CECB0F08A4688ECB0F0000000007D
:10DBDC0097ECB0F000000000000000000000000016
:10DBEC008A424CECB0F000008A6A53ECAFF00000B3
:10DBFC008A6AC7ECB8F08A6A8A864CECB0F08A461E
:10DC0C0088ECB0F00000000097ECB0F000000000D1
:10DC1C0000000000000000008A424CECB0F0000054
:10DC2C008A6AB4ECAEF000008A6AC7ECB8F08A6A73
:10DC3C008A865BECB0F0000000008A4600008A4245
:10DC4C0092ECB0F000008A4600008A4292ECB0F0F0
:10DC5C0000008A4600008A4292ECB0F000008A462E
:10DC6C0000008A4292ECB0F000008A4600008A4222
:10DC7C0092ECB0F000008A4600008A4292ECB0F0C0
:10DC8C0000008A4600008A4292ECB0F000008A46FE
:10DC9C0000008A4292ECB0F000008A4600008A42F2
:10DCAC0092ECB0F000008A4600008A424CECB0F0D6
:10DCBC0000008A6A82A008D082A25CEF68F00000A3
:10DCCC00000075ECB5F0E8D448ECAEF00E53D8A4D7
:10DCDC003DD00000BB0E8A6A0F6F000000000000F0
:10DCEC008B9E8B8697ECB0F00000000000008B8EB2
:10DCFC008B9697ECB0F000000000000003D08A6A0D
:10DD0C00C7ECB8F088ECB0F00000000097ECB0F075
:10DD1C000000000000006AECB0F000000F2FEFD7FD
:10DD2C0000008A6AC7ECB8F088ECB0F00000000084
:10DD3C0097ECB0F00000000000005BECB0F00000CD
:10DD4C00000082A03FD082A2A5D439D0BB0E8A6A33
:10DD5C000F6F0000000000008B9E8B8697ECB0F0DC
:10DD6C000000000000008B8E8B9697ECB0F000004A
:10DD7C000000000003D08A6AC7ECB8F088ECB0F061
:10DD8C000000000097ECB0F00000000000006AEC0E
:10DD9C00B0F000000F2FEFD700008A6AC7ECB8F084
:10DDAC0088ECB0F00000000097ECB0F00000000030
:10DDBC0000006AECB0F0000000000000000075EC00
:10DDCC00B5F084D748ECAEF00E53D8A440D0000088
:10DDDC00BB0E8A6A0F6F0000000000008B9E8B86C2
:10DDEC0097ECB0F00000000000008B8E8B9697EC47
:10DDFC00B0F000000000000003D08A6AC7ECB8F055
:10DE0C008A8888ECB0F00000000097ECB0F00000BD
:10DE1C000000000065ECB0F0000000008A6A0F2FD3
:10DE2C00ECD700008A6AC7ECB8F08A8888ECB0F0AE
:10DE3C000000000097ECB0F00000000000005BEC6C
:10DE4C00B0F08A6A82A042D082A23ED73CD0BB0EF0
:10DE5C008A6A0F6F0000000000008B9E8B8697EC87
:10DE6C00B0F00000000000008B8E8B9697ECB0F0A9
:10DE7C0000000000000003D08A6AC7ECB8F08A8862
:10DE8C0088ECB0F00000000097ECB0F0000000004F
:10DE9C00000065ECB0F0000000008A6A0F2FECD790
:10DEAC0000008A6AC7ECB8F08A8888ECB0F00000F1
:10DEBC00000097ECB0F00000000000006AECB0F03D
:10DECC008A6A0000000075ECB5F07ED748ECAEF025
:10DEDC00190E036F136B0E53D8A404D00000E1ECA1
:10DEEC00B0F004D0E1ECB0F00000000075ECB5F03F
:10DEFC00F2D748ECAEF00E53D8A4E9D000008A6AF1
:10DF0C00A1ECB0F08B9E8B8697ECB0F0000000007B
:10DF1C0000008B8E8B9697ECB0F000000000000098
:10DF2C00000000008A88CDECB0F000000000CDECC1
:10DF3C00B0F000008A6A97ECB0F00000000000001E
:10DF4C006FECB0F08A88CDECB0F00000000097ECDC
:10DF5C00B0F000000000000097ECB0F08A6A0000FE
:10DF6C008A6AC7ECB8F08A88CDECB0F000000000EB
:10DF7C00CDECB0F000008A6A97ECB0F00000000025
:10DF8C0000006FECB0F08A88CDECB0F0000000001F
:10DF9C0097ECB0F000000000000097ECB0F000002F
:10DFAC0000008A6A14ECB0F000008A6AC7ECB8F082
:10DFBC008A88CDECB0F000000000CDECB0F0000091
:10DFCC008A6A97ECB0F00000000000006FECB0F033
:10DFDC008A88CDECB0F00000000097ECB0F00000A7
:10DFEC000000000097ECB0F0000000008A6AF2EC30
:10DFFC00AFF000008A6AC7ECB8F08A88CDECB0F0BC
:10E00C0000000000CDECB0F000008A6A97ECB0F094
:10E01C000000000000006FECB0F08A88CDECB0F08E
:10E02C000000000097ECB0F000000000000097EC3E
:10E03C00B0F0000000008A6A14ECB0F000008A6AAC
:10E04C00C7ECB8F08A88CDECB0F000000000CDEC45
:10E05C00B0F000008A6A97ECB0F0000000000000FD
:10E06C006FECB0F08A88CDECB0F00000000097ECBB
:10E07C00B0F000000000000097ECB0F000000000D1
:10E08C008A6AC7ECB8F08A88CDECB0F000000000CA
:10E09C00CDECB0F000008A6A97ECB0F00000000004
:10E0AC0000006FECB0F08A88CDECB0F000000000FE
:10E0BC0097ECB0F000000000000083ECB0F0000022
:10E0CC00000082A004D182A2EED08A6AE9D08A6ACA
:10E0DC00A1ECB0F08B9E8B8697ECB0F000000000AA
:10E0EC0000008B8E8B9697ECB0F0000000000000C7
:10E0FC00000000008A88CDECB0F000000000CDECF0
:10E10C00B0F000008A6A97ECB0F00000000000004C
:10E11C006FECB0F08A88CDECB0F00000000097EC0A
:10E12C00B0F000000000000097ECB0F08A6A00002C
:10E13C008A6AC7ECB8F08A88CDECB0F00000000019
:10E14C00CDECB0F000008A6A97ECB0F00000000053
:10E15C0000006FECB0F08A88CDECB0F0000000004D
:10E16C0097ECB0F000000000000097ECB0F000005D
:10E17C0000008A6A14ECB0F000008A6AC7ECB8F0B0
:10E18C008A88CDECB0F000000000CDECB0F00000BF
:10E19C008A6A97ECB0F00000000000006FECB0F061
:10E1AC008A88CDECB0F00000000097ECB0F00000D5
:10E1BC000000000097ECB0F0000000008A6AF2EC5E
:10E1CC00AFF000008A6AC7ECB8F08A88CDECB0F0EA
:10E1DC0000000000CDECB0F000008A6A97ECB0F0C3
:10E1EC000000000000006FECB0F08A88CDECB0F0BD
:10E1FC000000000097ECB0F000000000000097EC6D
:10E20C00B0F0000000008A6A14ECB0F000008A6ADA
:10E21C00C7ECB8F08A88CDECB0F000000000CDEC73
:10E22C00B0F000008A6A97ECB0F00000000000002B
:10E23C006FECB0F08A88CDECB0F00000000097ECE9
:10E24C00B0F000000000000097ECB0F000000000FF
:10E25C008A6AC7ECB8F08A88CDECB0F000000000F8
:10E26C00CDECB0F000008A6A97ECB0F00000000032
:10E27C0000006FECB0F08A88CDECB0F0000000002C
:10E28C0097ECB0F000000000000083ECB0F0000050
:10E29C00000082A01CD082A206D08A6A0000000076
:10E2AC0075ECB5F028D648ECAEF00E53D8A406D0D9
:10E2BC0000008A6A23ECB1F08A6A06D08A6A23ECE1
:10E2CC00B1F08A6A0000000075ECB5F0EED748ECAE
:10E2DC00AEF00E53D8A473D300008A6AA1ECB0F050
:10E2EC008B9E8B8697ECB0F00000000000008B8EAC
:10E2FC008B9697ECB0F000000000000000000000CE
:10E30C008A6A9CECB0F00000000000008A6AC7EC3E
:10E31C00B8F08A8897ECB0F0000000000000C7EC61
:10E32C00B0F08A6A97ECB0F0000000000000C7EC77
:10E33C00B0F08A8897ECB0F0000000000000C7EC49
:10E34C00B0F08A6A97ECB0F0000000000000C7EC57
:10E35C00B0F08A8897ECB0F0000000000000C7EC29
:10E36C00B0F08A6A97ECB0F0000000000000C7EC37
:10E37C00B0F08A8897ECB0F0000000000000C7EC09
:10E38C00B0F08A6A97ECB0F0000000000000C2EC1C
:10E39C00B0F0FBECADF000008A6AC7ECB8F08A88EC
:10E3AC0097ECB0F0000000000000C7ECB0F08A6AF7
:10E3BC0097ECB0F0000000000000C7ECB0F08A88C9
:10E3CC0097ECB0F0000000000000C7ECB0F08A6AD7
:10E3DC0097ECB0F0000000000000C7ECB0F08A88A9
:10E3EC0097ECB0F0000000000000C7ECB0F08A6AB7
:10E3FC0097ECB0F0000000000000C7ECB0F08A8889
:10E40C0097ECB0F0000000000000C7ECB0F08A6A96
:10E41C0097ECB0F0000000000000C2ECB0F000007F
:10E42C008A6AC7ECB8F08A6A97ECB0F0000000007A
:10E43C000000C7ECB0F08A8897ECB0F00000000048
:10E44C000000C7ECB0F08A6A97ECB0F00000000056
:10E45C000000C7ECB0F08A8897ECB0F00000000028
:10E46C000000C7ECB0F08A6A97ECB0F00000000036
:10E47C000000C7ECB0F08A8897ECB0F00000000008
:10E48C000000C7ECB0F08A6A97ECB0F00000000016
:10E49C000000C7ECB0F08A8897ECB0F000000000E8
:10E4AC000000C2ECB0F000008A6AB0ECADF00000E5
:10E4BC008A6AC7ECB8F08A6A97ECB0F000000000EA
:10E4CC000000C7ECB0F08A8897ECB0F000000000B8
:10E4DC000000C7ECB0F08A6A97ECB0F000000000C6
:10E4EC000000C7ECB0F08A8897ECB0F00000000098
:10E4FC000000C7ECB0F08A6A97ECB0F000000000A6
:10E50C000000C7ECB0F08A8897ECB0F00000000077
:10E51C000000C7ECB0F08A6A97ECB0F00000000085
:10E52C000000C7ECB0F08A8897ECB0F00000000057
:10E53C000000C2ECB0F000008A6AC7ECB8F08A8820
:10E54C0097ECB0F0000000000000C7ECB0F08A6A55
:10E55C0097ECB0F0000000000000C7ECB0F08A8827
:10E56C0097ECB0F0000000000000C7ECB0F08A6A35
:10E57C0097ECB0F0000000000000C7ECB0F08A8807
:10E58C0097ECB0F0000000000000C7ECB0F08A6A15
:10E59C0097ECB0F0000000000000C7ECB0F08A88E7
:10E5AC0097ECB0F0000000000000C7ECB0F08A6AF5
:10E5BC0097ECB0F0000000000000C2ECB0F0FBECF7
:10E5CC00ADF000008A6AC7ECB8F08A8897ECB0F01E
:10E5DC00000000000000C7ECB0F08A6A97ECB0F0C5
:10E5EC00000000000000C7ECB0F08A8897ECB0F097
:10E5FC00000000000000C7ECB0F08A6A97ECB0F0A5
:10E60C00000000000000C7ECB0F08A8897ECB0F076
:10E61C00000000000000C7ECB0F08A6A97ECB0F084
:10E62C00000000000000C7ECB0F08A8897ECB0F056
:10E63C00000000000000C7ECB0F08A6A97ECB0F064
:10E64C00000000000000C2ECB0F000008A6AC7ECC9
:10E65C00B8F08A6A97ECB0F0000000000000C7EC3C
:10E66C00B0F08A8897ECB0F0000000000000C7EC16
:10E67C00B0F08A6A97ECB0F0000000000000C7EC24
:10E68C00B0F08A8897ECB0F0000000000000C7ECF6
:10E69C00B0F08A6A97ECB0F0000000000000C7EC04
:10E6AC00B0F08A8897ECB0F0000000000000C7ECD6
:10E6BC00B0F08A6A97ECB0F0000000000000C7ECE4
:10E6CC00B0F08A8897ECB0F0000000000000C2ECBB
:10E6DC00B0F000008A6AB0ECADF000008A6AC7ECBA
:10E6EC00B8F08A6A97ECB0F0000000000000C7ECAC
:10E6FC00B0F08A8897ECB0F0000000000000C7EC86
:10E70C00B0F08A6A97ECB0F0000000000000C7EC93
:10E71C00B0F08A8897ECB0F0000000000000C7EC65
:10E72C00B0F08A6A97ECB0F0000000000000C7EC73
:10E73C00B0F08A8897ECB0F0000000000000C7EC45
:10E74C00B0F08A6A97ECB0F0000000000000C7EC53
:10E75C00B0F08A8897ECB0F0000000000000C2EC2A
:10E76C00B0F000008A6AC7ECB8F08A8897ECB0F079
:10E77C00000000000000C7ECB0F08A6A97ECB0F023
:10E78C00000000000000C7ECB0F08A8897ECB0F0F5
:10E79C00000000000000C7ECB0F08A6A97ECB0F003
:10E7AC00000000000000C7ECB0F08A8897ECB0F0D5
:10E7BC00000000000000C7ECB0F08A6A97ECB0F0E3
:10E7CC00000000000000C7ECB0F08A8897ECB0F0B5
:10E7DC00000000000000C7ECB0F08A6A97ECB0F0C3
:10E7EC00000000000000C2ECB0F0FBECADF000004B
:10E7FC008A6AC7ECB8F08A8897ECB0F00000000089
:10E80C000000C7ECB0F08A6A97ECB0F00000000092
:10E81C000000C7ECB0F08A8897ECB0F00000000064
:10E82C000000C7ECB0F08A6A97ECB0F00000000072
:10E83C000000C7ECB0F08A8897ECB0F00000000044
:10E84C000000C7ECB0F08A6A97ECB0F00000000052
:10E85C000000C7ECB0F08A8897ECB0F00000000024
:10E86C000000C7ECB0F08A6A97ECB0F00000000032
:10E87C000000C2ECB0F000008A6AC7ECB8F08A6AFB
:10E88C0097ECB0F0000000000000C7ECB0F08A88F4
:10E89C0097ECB0F0000000000000C7ECB0F08A6A02
:10E8AC0097ECB0F0000000000000C7ECB0F08A88D4
:10E8BC0097ECB0F0000000000000C7ECB0F08A6AE2
:10E8CC0097ECB0F0000000000000C7ECB0F08A88B4
:10E8DC0097ECB0F0000000000000C7ECB0F08A6AC2
:10E8EC0097ECB0F0000000000000C7ECB0F08A8894
:10E8FC0097ECB0F0000000000000C2ECB0F000009B
:10E90C008A6AB0ECADF000008A6AC7ECB8F08A6A8B
:10E91C0097ECB0F0000000000000C7ECB0F08A8863
:10E92C0097ECB0F0000000000000C7ECB0F08A6A71
:10E93C0097ECB0F0000000000000C7ECB0F08A8843
:10E94C0097ECB0F0000000000000C7ECB0F08A6A51
:10E95C0097ECB0F0000000000000C7ECB0F08A8823
:10E96C0097ECB0F0000000000000C7ECB0F08A6A31
:10E97C0097ECB0F0000000000000C7ECB0F08A8803
:10E98C0097ECB0F0000000000000C2ECB0F000000A
:10E99C008A6AC7ECB8F08A6A88ECB0F00000000014
:10E9AC0097ECB0F00000000000005BECB0F0000051
:10E9BC0082A05CEF68F082A27FEF6FF073D38A6A5B
:10E9CC00A1ECB0F08B9E8B8697ECB0F000000000B1
:10E9DC0000008B8E8B9697ECB0F0000000000000CE
:10E9EC00000000008A6A9CECB0F0000000000000FF
:10E9FC008A6AC7ECB8F08A8897ECB0F00000000087
:10EA0C000000C7ECB0F08A6A97ECB0F00000000090
:10EA1C000000C7ECB0F08A8897ECB0F00000000062
:10EA2C000000C7ECB0F08A6A97ECB0F00000000070
:10EA3C000000C7ECB0F08A8897ECB0F00000000042
:10EA4C000000C7ECB0F08A6A97ECB0F00000000050
:10EA5C000000C7ECB0F08A8897ECB0F00000000022
:10EA6C000000C7ECB0F08A6A97ECB0F00000000030
:10EA7C000000C2ECB0F0FBECADF000008A6AC7EC11
:10EA8C00B8F08A8897ECB0F0000000000000C7ECEA
:10EA9C00B0F08A6A97ECB0F0000000000000C7EC00
:10EAAC00B0F08A8897ECB0F0000000000000C7ECD2
:10EABC00B0F08A6A97ECB0F0000000000000C7ECE0
:10EACC00B0F08A8897ECB0F0000000000000C7ECB2
:10EADC00B0F08A6A97ECB0F0000000000000C7ECC0
:10EAEC00B0F08A8897ECB0F0000000000000C7EC92
:10EAFC00B0F08A6A97ECB0F0000000000000C2ECA5
:10EB0C00B0F000008A6AC7ECB8F08A6A97ECB0F0F3
:10EB1C00000000000000C7ECB0F08A8897ECB0F061
:10EB2C00000000000000C7ECB0F08A6A97ECB0F06F
:10EB3C00000000000000C7ECB0F08A8897ECB0F041
:10EB4C00000000000000C7ECB0F08A6A97ECB0F04F
:10EB5C00000000000000C7ECB0F08A8897ECB0F021
:10EB6C00000000000000C7ECB0F08A6A97ECB0F02F
:10EB7C00000000000000C7ECB0F08A8897ECB0F001
:10EB8C00000000000000C2ECB0F000008A6AB0EC9B
:10EB9C00ADF000008A6AC7ECB8F08A6A97ECB0F066
:10EBAC00000000000000C7ECB0F08A8897ECB0F0D1
:10EBBC00000000000000C7ECB0F08A6A97ECB0F0DF
:10EBCC00000000000000C7ECB0F08A8897ECB0F0B1
:10EBDC00000000000000C7ECB0F08A6A97ECB0F0BF
:10EBEC00000000000000C7ECB0F08A8897ECB0F091
:10EBFC00000000000000C7ECB0F08A6A97ECB0F09F
:10EC0C00000000000000C7ECB0F08A8897ECB0F070
:10EC1C00000000000000C2ECB0F000008A6AC7ECF3
:10EC2C00B8F08A8897ECB0F0000000000000C7EC48
:10EC3C00B0F08A6A97ECB0F0000000000000C7EC5E
:10EC4C00B0F08A8897ECB0F0000000000000C7EC30
:10EC5C00B0F08A6A97ECB0F0000000000000C7EC3E
:10EC6C00B0F08A8897ECB0F0000000000000C7EC10
:10EC7C00B0F08A6A97ECB0F0000000000000C7EC1E
:10EC8C00B0F08A8897ECB0F0000000000000C7ECF0
:10EC9C00B0F08A6A97ECB0F0000000000000C2EC03
:10ECAC00B0F0FBECADF000008A6AC7ECB8F08A88D3
:10ECBC0097ECB0F0000000000000C7ECB0F08A6ADE
:10ECCC0097ECB0F0000000000000C7ECB0F08A88B0
:10ECDC0097ECB0F0000000000000C7ECB0F08A6ABE
:10ECEC0097ECB0F0000000000000C7ECB0F08A8890
:10ECFC0097ECB0F0000000000000C7ECB0F08A6A9E
:10ED0C0097ECB0F0000000000000C7ECB0F08A886F
:10ED1C0097ECB0F0000000000000C7ECB0F08A6A7D
:10ED2C0097ECB0F0000000000000C2ECB0F0000066
:10ED3C008A6AC7ECB8F08A6A97ECB0F00000000061
:10ED4C000000C7ECB0F08A8897ECB0F0000000002F
:10ED5C000000C7ECB0F08A6A97ECB0F0000000003D
:10ED6C000000C7ECB0F08A8897ECB0F0000000000F
:10ED7C000000C7ECB0F08A6A97ECB0F0000000001D
:10ED8C000000C7ECB0F08A8897ECB0F000000000EF
:10ED9C000000C7ECB0F08A6A97ECB0F000000000FD
:10EDAC000000C7ECB0F08A8897ECB0F000000000CF
:10EDBC000000C2ECB0F000008A6AB0ECADF00000CC
:10EDCC008A6AC7ECB8F08A6A97ECB0F000000000D1
:10EDDC000000C7ECB0F08A8897ECB0F0000000009F
:10EDEC000000C7ECB0F08A6A97ECB0F000000000AD
:10EDFC000000C7ECB0F08A8897ECB0F0000000007F
:10EE0C000000C7ECB0F08A6A97ECB0F0000000008C
:10EE1C000000C7ECB0F08A8897ECB0F0000000005E
:10EE2C000000C7ECB0F08A6A97ECB0F0000000006C
:10EE3C000000C7ECB0F08A8897ECB0F0000000003E
:10EE4C000000C2ECB0F000008A6AC7ECB8F08A8807
:10EE5C0097ECB0F0000000000000C7ECB0F08A6A3C
:10EE6C0097ECB0F0000000000000C7ECB0F08A880E
:10EE7C0097ECB0F0000000000000C7ECB0F08A6A1C
:10EE8C0097ECB0F0000000000000C7ECB0F08A88EE
:10EE9C0097ECB0F0000000000000C7ECB0F08A6AFC
:10EEAC0097ECB0F0000000000000C7ECB0F08A88CE
:10EEBC0097ECB0F0000000000000C7ECB0F08A6ADC
:10EECC0097ECB0F0000000000000C2ECB0F0FBECDE
:10EEDC00ADF000008A6AC7ECB8F08A8897ECB0F005
:10EEEC00000000000000C7ECB0F08A6A97ECB0F0AC
:10EEFC00000000000000C7ECB0F08A8897ECB0F07E
:10EF0C00000000000000C7ECB0F08A6A97ECB0F08B
:10EF1C00000000000000C7ECB0F08A8897ECB0F05D
:10EF2C00000000000000C7ECB0F08A6A97ECB0F06B
:10EF3C00000000000000C7ECB0F08A8897ECB0F03D
:10EF4C00000000000000C7ECB0F08A6A97ECB0F04B
:10EF5C00000000000000C2ECB0F000008A6AC7ECB0
:10EF6C00B8F08A6A97ECB0F0000000000000C7EC23
:10EF7C00B0F08A8897ECB0F0000000000000C7ECFD
:10EF8C00B0F08A6A97ECB0F0000000000000C7EC0B
:10EF9C00B0F08A8897ECB0F0000000000000C7ECDD
:10EFAC00B0F08A6A97ECB0F0000000000000C7ECEB
:10EFBC00B0F08A8897ECB0F0000000000000C7ECBD
:10EFCC00B0F08A6A97ECB0F0000000000000C7ECCB
:10EFDC00B0F08A8897ECB0F0000000000000C2ECA2
:10EFEC00B0F000008A6AB0ECADF000008A6AC7ECA1
:10EFFC00B8F08A6A97ECB0F0000000000000C7EC93
:10F00C00B0F08A8897ECB0F0000000000000C7EC6C
:10F01C00B0F08A6A97ECB0F0000000000000C7EC7A
:10F02C00B0F08A8897ECB0F0000000000000C7EC4C
:10F03C00B0F08A6A97ECB0F0000000000000C7EC5A
:10F04C00B0F08A8897ECB0F0000000000000C7EC2C
:10F05C00B0F08A6A97ECB0F0000000000000C7EC3A
:10F06C00B0F08A8897ECB0F0000000000000C2EC11
:10F07C00B0F000008A6AC7ECB8F08A6A88ECB0F08D
:10F08C000000000097ECB0F00000000000005BEC0A
:10F09C00B0F0000082A05CEF68F082A27FEF6FF00E
:10F0AC000000000075ECB5F06FEF71F048ECAEF0BD
:10F0BC000E53D8A4B0D000008A6AA1ECB0F08B9E9D
:10F0CC008B8697ECB0F00000000000008B8E8B96C6
:10F0DC0097ECB0F0000000000000000000008A6A0D
:10F0EC0065ECB0F08A8800008A6A92ECB0F00000FF
:10F0FC008A8800008A6A92ECB0F000008A880000CE
:10F10C008A6A92ECB0F000008A8800008A6A92EC5D
:10F11C00B0F000008A8800008A6A92ECB0F000001F
:10F12C008A8800008A6A92ECB0F000008A8800009D
:10F13C008A6A92ECB0F000008A8800008A6A92EC2D
:10F14C00B0F000008A8800008A6A92ECB0F00000EF
:10F15C008A8800008A6A5BECB0F0A3ECAFF071EC2B
:10F16C00B8F0A3ECAFF071ECB8F071ECB8F0A3EC24
:10F17C00AFF071ECB8F071ECB8F071ECB8F0A3EC46
:10F18C00AFF000008A6AC7ECB8F08A6A65ECB0F0A0
:10F19C008A8800008A6A92ECB0F000008A8800002D
:10F1AC008A6A92ECB0F000008A8800008A6A92ECBD
:10F1BC00B0F000008A8800008A6A92ECB0F000007F
:10F1CC008A8800008A6A92ECB0F000008A880000FD
:10F1DC008A6A92ECB0F000008A8800008A6A92EC8D
:10F1EC00B0F000008A8800008A6A92ECB0F000004F
:10F1FC008A8800008A6A92ECB0F000008A880000CD
:10F20C008A6A4CECB0F00000000082A0B7D082A259
:10F21C00E8EF63F0B0D08A6AA1ECB0F08B9E8B86DD
:10F22C0097ECB0F00000000000008B8E8B9697ECF2
:10F23C00B0F0000000000000000000008A6A65ECDD
:10F24C00B0F08A8800008A6A92ECB0F000008A88DC
:10F25C0000008A6A92ECB0F000008A8800008A6A8A
:10F26C0092ECB0F000008A8800008A6A92ECB0F050
:10F27C0000008A8800008A6A92ECB0F000008A884C
:10F28C0000008A6A92ECB0F000008A8800008A6A5A
:10F29C0092ECB0F000008A8800008A6A92ECB0F020
:10F2AC0000008A8800008A6A92ECB0F000008A881C
:10F2BC0000008A6A5BECB0F0A3ECAFF071ECB8F034
:10F2CC00A3ECAFF071ECB8F071ECB8F0A3ECAFF0CC
:10F2DC0071ECB8F071ECB8F071ECB8F0A3ECAFF0E5
:10F2EC0000008A6AC7ECB8F08A6A65ECB0F08A88CC
:10F2FC0000008A6A92ECB0F000008A8800008A6AEA
:10F30C0092ECB0F000008A8800008A6A92ECB0F0AF
:10F31C0000008A8800008A6A92ECB0F000008A88AB
:10F32C0000008A6A92ECB0F000008A8800008A6AB9
:10F33C0092ECB0F000008A8800008A6A92ECB0F07F
:10F34C0000008A8800008A6A92ECB0F000008A887B
:10F35C0000008A6A92ECB0F000008A8800008A6A89
:10F36C004CECB0F00000000082A008D082A2E8EFC4
:10F37C0063F00000000075ECB5F09AD648ECAEF0E6
:10F38C000E53D8A462D100008A6AA1ECB0F08B9E17
:10F39C008B8697ECB0F00000000000008B8E8B96F3
:10F3AC0097ECB0F0000000000000000000008A6A3A
:10F3BC0065ECB0F08A8800008A6A92ECB0F000002C
:10F3CC008A8800008A6A92ECB0F000008A880000FB
:10F3DC008A6A92ECB0F000008A8800008A6A92EC8B
:10F3EC00B0F000008A8800008A6A92ECB0F000004D
:10F3FC008A8800008A6A92ECB0F000008A880000CB
:10F40C008A6A92ECB0F000008A8800008A6A92EC5A
:10F41C00B0F000008A8800008A6A92ECB0F000001C
:10F42C008A8800008A6A5BECB0F0A3ECAFF0D9ECF0
:10F43C00B8F0A3ECAFF00000000000008B9E97EC3E
:10F44C00B0F000000000000000008B8E97ECB0F0D4
:10F45C00000000000000BEECB0F08A6A65ECB0F071
:10F46C008A8800008A6A92ECB0F000008A8800005A
:10F47C008A6A92ECB0F000008A8800008A6A92ECEA
:10F48C00B0F000008A8800008A6A51ECB0F08A88DB
:10F49C0051ECB0F000008A6A51ECB0F08A880000A0
:10F4AC008A6A92ECB0F000008A8800008A6A51ECFB
:10F4BC00B0F08A8851ECB0F000008A6A51ECB0F0E0
:10F4CC008A8800008A6A92ECB0F000008A880000FA
:10F4DC008A6A92ECB0F000008A8800008A6A92EC8A
:10F4EC00B0F000008A8800008A6A5BECB0F037EC60
:10F4FC00B9F0A3ECAFF000008B9E97ECB0F00000DD
:10F50C000000000000008B8E97ECB0F000000000B3
:10F51C000000C7ECB0F08A6A65ECB0F08A88000095
:10F52C008A6A92ECB0F000008A8800008A6A92EC39
:10F53C00B0F000008A8800008A6A92ECB0F00000FB
:10F54C008A8800008A6A51ECB0F08A8851ECB0F0DD
:10F55C0000008A6A51ECB0F08A8800008A6A92EC4A
:10F56C00B0F000008A8800008A6A51ECB0F08A88FA
:10F57C0051ECB0F000008A6A51ECB0F08A880000BF
:10F58C008A6A92ECB0F000008A8800008A6A92ECD9
:10F59C00B0F000008A8800008A6A92ECB0F000009B
:10F5AC008A8800008A6A5BECB0F037ECB9F037EC73
:10F5BC00B9F0A3ECAFF000008A6AC7ECB8F08A6A25
:10F5CC0065ECB0F08A8800008A6A92ECB0F000001A
:10F5DC008A8800008A6A92ECB0F000008A880000E9
:10F5EC008A6A92ECB0F000008A8800008A6A92EC79
:10F5FC00B0F000008A8800008A6A92ECB0F000003B
:10F60C008A8800008A6A92ECB0F000008A880000B8
:10F61C008A6A92ECB0F000008A8800008A6A92EC48
:10F62C00B0F000008A8800008A6A92ECB0F000000A
:10F63C008A8800008A6A4CECB0F00000000082A0BE
:10F64C002EEF00F082A232D563D18A6AA1ECB0F021
:10F65C008B9E8B8697ECB0F00000000000008B8E28
:10F66C008B9697ECB0F0000000000000000000004A
:10F67C008A6A65ECB0F08A8800008A6A92ECB0F075
:10F68C0000008A8800008A6A92ECB0F000008A8838
:10F69C0000008A6A92ECB0F000008A8800008A6A46
:10F6AC0092ECB0F000008A8800008A6A92ECB0F00C
:10F6BC0000008A8800008A6A92ECB0F000008A8808
:10F6CC0000008A6A92ECB0F000008A8800008A6A16
:10F6DC0092ECB0F000008A8800008A6A92ECB0F0DC
:10F6EC0000008A8800008A6A5BECB0F0A3ECAFF0F3
:10F6FC00D9ECB8F0A3ECAFF00000000000008B9E3A
:10F70C0097ECB0F000000000000000008B8E97EC2E
:10F71C00B0F0000000000000BEECB0F08A6A65ECAE
:10F72C00B0F08A8800008A6A92ECB0F000008A88F7
:10F73C0000008A6A92ECB0F000008A8800008A6AA5
:10F74C0092ECB0F000008A8800008A6A51ECB0F0AC
:10F75C008A8851ECB0F000008A6A51ECB0F08A88CB
:10F76C0000008A6A92ECB0F000008A8800008A6A75
:10F77C0051ECB0F08A8851ECB0F000008A6A51EC80
:10F78C00B0F08A8800008A6A92ECB0F000008A8897
:10F79C0000008A6A92ECB0F000008A8800008A6A45
:10F7AC0092ECB0F000008A8800008A6A5BECB0F042
:10F7BC0037ECB9F0A3ECAFF000008B9E97ECB0F0F7
:10F7CC0000000000000000008B8E97ECB0F00000F1
:10F7DC0000000000C7ECB0F08A6A65ECB0F08A88D3
:10F7EC0000008A6A92ECB0F000008A8800008A6AF5
:10F7FC0092ECB0F000008A8800008A6A92ECB0F0BB
:10F80C0000008A8800008A6A51ECB0F08A8851ECBA
:10F81C00B0F000008A6A51ECB0F08A8800008A6A65
:10F82C0092ECB0F000008A8800008A6A51ECB0F0CB
:10F83C008A8851ECB0F000008A6A51ECB0F08A88EA
:10F84C0000008A6A92ECB0F000008A8800008A6A94
:10F85C0092ECB0F000008A8800008A6A92ECB0F05A
:10F86C0000008A8800008A6A5BECB0F037ECB9F0D3
:10F87C0037ECB9F0A3ECAFF000008A6AC7ECB8F033
:10F88C008A6A65ECB0F08A8800008A6A92ECB0F063
:10F89C0000008A8800008A6A92ECB0F000008A8826
:10F8AC0000008A6A92ECB0F000008A8800008A6A34
:10F8BC0092ECB0F000008A8800008A6A92ECB0F0FA
:10F8CC0000008A8800008A6A92ECB0F000008A88F6
:10F8DC0000008A6A92ECB0F000008A8800008A6A04
:10F8EC0092ECB0F000008A8800008A6A92ECB0F0CA
:10F8FC0000008A8800008A6A4CECB0F0000000001E
:10F90C0082A02EEF00F082A25CEF78F000000000E5
:10F91C0075ECB5F035D50300FED7000000008A6AFF
:10F92C00000000008A88000000008A6A00000000C5
:10F93C008A88000000008A6A000000008A880000A3
:10F94C0000008A6A000000008A88000000008A6AB1
:10F95C00000000008A8800000000120000008A6A83
:10F96C0000008A8800008A6A00008A8800008A6A7F
:10F97C0000008A8800008A6A00008A8800008A6A6F
:10F98C0000008A8800008A6A00008A8800008A6A5F
:10F99C0000008A8800008A6A8A88000012008A881F
:10F9AC008A6A8A868A368A6A8A868A368A6A8A86BF
:10F9BC008A368A6A8A868A368A6A8A868A368A6AFF
:10F9CC008A868A368A6A8A868A368A6A8A868A36D3
:10F9DC008A6A8A868A368A6A8A868A360000120081
:10F9EC008A888A6A8A888A6A8A888A6A8A888A6AF3
:10F9FC008A888A6A8A888A6A8A888A6A8A888A6AE3
:10FA0C008A888A6A8A888A6A8A888A6A8A888A6AD2
:10FA1C008A888A6A8A888A6A8A888A6A8A880000B6
:10FA2C00120083ECB0F0100E816E080E816E83EC28
:10FA3C00B0F000000000100E816E080E816E83EC99
:10FA4C00B0F000000000100E816E080E816E83EC89
:10FA5C00B0F000000000100E816E080E816E83EC79
:10FA6C00B0F000000000100E816E080E816E7EEC6E
:10FA7C00B0F00000000000001200C2ECB0F0100E5C
:10FA8C00816E080E816E5BECB0F0100E816E65EC31
:10FA9C00B0F00000000000008A6A97ECB0F00000A3
:10FAAC000000000065ECB0F00000100E816E65ECFB
:10FABC00B0F000000000080E816E5BECB0F0100E90
:10FACC00816E080E816EBEECB0F00000120083EC6B
:10FADC00B0F0100E816E080E816E5BECB0F0100E63
:10FAEC00816E65ECB0F00000000000008A6A97ECB3
:10FAFC00B0F000000000000065ECB0F00000100E4B
:10FB0C00816E65ECB0F000000000080E816E5BECBD
:10FB1C00B0F0100E816E080E816E7EECB0F000001D
:10FB2C00000000001200C2ECB0F0100E816E080E46
:10FB3C00816E5BECB0F0100E816ECDECB0F000007D
:10FB4C0000006AECB0F000000000080E816E5BEC67
:10FB5C00B0F0100E816E080E816EBEECB0F000009D
:10FB6C00120083ECB0F0100E816E080E816E5BEC0F
:10FB7C00B0F0100E816ECDECB0F0000000006AEC1D
:10FB8C00B0F000000000080E816E5BECB0F0100EBF
:10FB9C00816E080E816E7EECB0F00000000000005B
:10FBAC001200C2ECB0F0100E816E080E816E83EC68
:10FBBC00B0F000000000100E816E080E816E83EC18
:10FBCC00B0F000000000100E816E080E816E83EC08
:10FBDC00B0F000000000100E816E080E816E83ECF8
:10FBEC00B0F000000000100E816E080E816EC2ECA9
:10FBFC00B0F00000120083ECB0F0100E816E080E15
:10FC0C00816E83ECB0F000000000100E816E080EC7
:10FC1C00816E83ECB0F000000000100E816E080EB7
:10FC2C00816E83ECB0F000000000100E816E080EA7
:10FC3C00816E83ECB0F000000000100E816E080E97
:10FC4C00816E7EECB0F000000000000012006AEC47
:10FC5C00B0F000000000A1ECB0F08A6A00000000D7
:10FC6C00000000008A868A460000000000008A42DC
:10FC7C0065ECB0F00000100E816E70DE8A42BEECB6
:10FC8C00B0F08A846AECB0F000008A94BEECB0F05C
:10FC9C00100E816E84DE8A4265ECB0F000008A465C
:10FCAC000000000000008A428A6A00000000000088
:10FCBC0000008A8600000000000000006AECB0F032
:10FCCC000000000012006AECB0F000000000000020
:10FCDC008A6A00000000000000008A868A46000044
:10FCEC000000000000008A426AECB0F00000100E28
:10FCFC00816E34DE8A42BEECB0F08A846AECB0F0DD
:10FD0C0000008A94BEECB0F0100E816E48DE8A4280
:10FD1C006AECB0F000008A46000000000000000011
:10FD2C008A428A6A00000000000000008A866AECA1
:10FD3C00B0F00000000012006AECB0F0000000000F
:10FD4C00B2ECB0F08A6A0000000000008A868A4695
:10FD5C0000000000000000008A4265ECB0F0100EBC
:10FD6C00816EFCDD8A42BEECB0F08A846AECB0F0A5
:10FD7C0000008A94BEECB0F0100E816E10DE8A4248
:10FD8C0065ECB0F08A4600000000000000008A42DA
:10FD9C008A6A0000000000008A86A1ECB0F06AECD0
:10FDAC00B0F00000000012006AECB0F0000000009F
:10FDBC00000000008A6A00000000000000008A8831
:10FDCC0000000000000000008A426AECB0F0000065
:10FDDC00100E816EC3DD8A42BEECB0F08A846AECF0
:10FDEC00B0F000008A94BEECB0F0100E816ED7DD3E
:10FDFC008A426AECB0F000008A4600000000000065
:10FE0C0000008A6A00000000000000008A860000E2
:10FE1C006AECB0F00000000012006AECB0F00000D8
:10FE2C00000000008A6A00000000000000008A88C0
:10FE3C00A1ECB0F08A426AECB0F00000100E816EBA
:10FE4C008DDD8A42BEECB0F08A846AECB0F0000022
:10FE5C008A94BEECB0F0100E816EA1DD8A426AEC81
:10FE6C00B0F000008A46A1ECB0F08A6A00000000F5
:10FE7C00000000008A866AECB0F00000000012005E
:10FE8C006AECB0F000000000A1ECB0F08A6A00004F
:10FE9C000000000000008A88000000000000000044
:10FEAC008A4265ECB0F00000100E816E57DD8A427C
:10FEBC00BEECB0F08A846AECB0F000008A94BEEC20
:10FECC00B0F0100E816E6BDD8A4265ECB0F0000074
:10FEDC008A4600000000000000008A6A0000000052
:10FEEC00000000008A8600000000000000006AECA0
:10FEFC00B0F00000000012006AECB0F0000000004E
:10FF0C0000008A6A00000000000000008A880000DF
:10FF1C000000000000008A426AECB0F00000000013
:10FF2C00100E816E1BDD8A42BEECB0F08A846AEC46
:10FF3C00B0F000008A94BEECB0F0100E816E2FDD94
:10FF4C008A426AECB0F0000000008A460000000013
:10FF5C00000000008A6A00000000000000008A8691
:10FF6C006AECB0F00000000012006AECB0F0000087
:10FF7C00000045ECB0F08A6A0000000000000000B0
:10FF8C008A88A1ECB0F08A4256ECB0F00000100E5A
:10FF9C00816EE4DC8A42BEECB0F08A846AECB0F08C
:10FFAC0000008A94BEECB0F0100E816EF8DC8A4230
:10FFBC0056ECB0F000008A46A1ECB0F08A6A000062
:10FFCC000000000000008A86C7ECB0F06AECB0F0CC
:10FFDC000000000012006AECB0F000000000B2EC6F
:10FFEC00B0F08A6AA1ECB0F08A8800000000000032
:10FFFC0000008A425BECB0F000000000100E816E35
:020000040001F9
:10000C00ADDC8A42BEECB0F08A846AECB0F0000041
:10001C008A94BEECB0F0100E816EC1DC8A425BECAF
:10002C00B0F0000000008A46000000000000000054
:10003C008A6AA1ECB0F08A86A1ECB0F06AECB0F060
:10004C000000000012006AECB0F00000000045EC6B
:10005C00B0F08A6AA1ECB0F08A88000000000000C1
:10006C0000008A4256ECB0F00000100E816E76DC77
:10007C008A42BEECB0F08A846AECB0F000008A943C
:10008C00BEECB0F0100E816E8ADC8A4256ECB0F0F9
:10009C0000008A4600000000000000008A6AA1EC03
:1000AC00B0F08A86C7ECB0F06AECB0F0000000004B
:1000BC0012006AECB0F000000000BEECB0F08A6AEE
:1000CC0000000000000000008A88A1ECB0F08A4219
:1000DC005BECB0F00000100E816E40DC8A42BEEC8E
:1000EC00B0F08A846AECB0F000008A94BEECB0F0F8
:1000FC00100E816E54DC8A425BECB0F000008A4634
:10010C00A1ECB0F08A6A00000000000000008A86B2
:10011C00B2ECB0F06AECB0F00000000012006AEC37
:10012C00B0F000000000C7ECB0F08A6A00000000DC
:10013C00000000008A868A460000000000000000D3
:10014C008A4256ECB0F000000000100E816E06DC06
:10015C008A42BEECB0F08A846AECB0F000008A945B
:10016C00BEECB0F0100E816E1ADC8A4256ECB0F088
:10017C00000000008A4600000000000000008A42D7
:10018C008A6A00000000000000008A86C2ECB0F011
:10019C006AECB0F00000000012006AECB0F0000055
:1001AC000000B2ECB0F08A6A000000000000000011
:1001BC008A88A1ECB0F08A425BECB0F00000000041
:1001CC00100E816EB4EC7CF08A42BEECB0F08A84E6
:1001DC006AECB0F000008A94BEECB0F0100E816EA8
:1001EC00D5EC7CF08A425BECB0F0000000008A4653
:1001FC00A1ECB0F08A6A00000000000000008A86C2
:10020C00A1ECB0F06AECB0F00000000012006AEC57
:10021C00B0F00000000045ECB0F08A6A000000006D
:10022C00000000008A8800000000000000008A42E4
:10023C0056ECB0F000000000100E816EB4EC7CF0B7
:10024C008A42BEECB0F08A846AECB0F000008A946A
:10025C00BEECB0F0100E816ED5EC7CF08A4256EC00
:10026C00B0F0000000008A46000000000000000012
:10027C008A6A00000000000000008A86C7ECB0F01B
:10028C006AECB0F00000000012006AECB0F0000064
:10029C000000C2ECB0F08A6A000000000000000010
:1002AC008A868A4600000000000000008A425BEC4F
:1002BC00B0F0100E816EB4EC7CF08A42BEECB0F063
:1002CC008A846AECB0F000008A94BEECB0F0100E98
:1002DC00816ED5EC7CF08A425BECB0F08A46000073
:1002EC000000000000008A428A6A00000000000042
:1002FC0000008A86BEECB0F06AECB0F000000000A2
:10030C0012006AECB0F000000000A1ECB0F08A6AB8
:10031C0000000000000000008A88000000000000BF
:10032C0000008A4265ECB0F00000100E816EB4EC57
:10033C007CF08A42BEECB0F08A846AECB0F000002B
:10034C008A94BEECB0F0100E816ED5EC7CF08A4233
:10035C0065ECB0F000008A460000000000000000D0
:10036C008A6A00000000000000008A86000000007D
:10037C00000000006AECB0F00000000012006AEC13
:10038C00B0F000000000C7ECB0F08A6A000000007A
:10039C00000000008A8800000000000000008A4273
:1003AC005BECB0F0100E816EB4EC7CF08A42BEECCB
:1003BC00B0F08A846AECB0F000008A94BEECB0F025
:1003CC00100E816ED5EC7CF08A425BECB0F08A4664
:1003DC0000000000000000008A6A0000000000001D
:1003EC0000008A86C2ECB0F06AECB0F000000000AD
:1003FC0012006AECB0F000000000A1ECB0F08A6AC8
:10040C0000000000000000008A868A460000000000
:10041C00000000008A4265ECB0F0100E816EB4EC66
:10042C007CF08A42BEECB0F08A846AECB0F000003A
:10043C008A94BEECB0F0100E816ED5EC7CF08A4242
:10044C0065ECB0F08A4600000000000000008A4213
:10045C008A6A00000000000000008A86000000008C
:10046C00000000006AECB0F00000000012006AEC22
:10047C00B0F000000000C2ECB0F08A6A000000008E
:10048C00000000008A8800000000000000008A4282
:10049C005BECB0F00000100E816EB4EC7CF08A4284
:1004AC00BEECB0F08A846AECB0F000008A94BEEC2A
:1004BC00B0F0100E816ED5EC7CF08A425BECB0F0A3
:1004CC0000008A4600000000000000008A6A00005C
:1004DC000000000000008A86BEECB0F06AECB0F0C0
:1004EC000000000012006AECB0F0000000000000F8
:1004FC000000000000008A6AA1ECB0F08A880000BD
:10050C000000000000008A4265ECB0F00000100E04
:10051C00816EB4EC7CF08A42BEECB0F08A846AEC5A
:10052C00B0F000008A94BEECB0F0100E816ED5ECE9
:10053C007CF08A4265ECB0F000008A4600000000B6
:10054C00000000008A6AA1ECB0F08A86000000006E
:10055C0000006AECB0F00000000012006AECB0F091
:10056C0000000000C2ECB0F08A6A0000000000003D
:10057C0000008A8800000000000000008A425BEC4A
:10058C00B0F00000100E816EB4EC7CF08A42BEEC30
:10059C00B0F08A846AECB0F000008A94BEECB0F043
:1005AC00100E816ED5EC7CF08A425BECB0F0000052
:1005BC008A4600000000000000008A6A000000006B
:1005CC00000000008A86BEECB0F06AECB0F00000CF
:1005DC00000012006AECB0F000000000A1ECB0F0DA
:1005EC008A6A00000000000000008A8800000000F9
:1005FC00000000008A4265ECB0F00000100E816E25
:10060C00B4EC7CF08A42BEECB0F08A846AECB0F0B8
:10061C0000008A94BEECB0F0100E816ED5EC7CF02C
:10062C008A4265ECB0F000008A4600000000000031
:10063C0000008A6A00000000000000008A860000AA
:10064C000000000000006AECB0F000000000120096
:10065C006AECB0F000000000BEECB0F08A6A00005A
:10066C000000000000008A868A460000000000009E
:10067C0000008A425BECB0F00000100E816EB4EC0E
:10068C007CF08A42BEECB0F08A846AECB0F00000D8
:10069C008A94BEECB0F0100E816ED5EC7CF08A42E0
:1006AC005BECB0F000008A46000000000000000087
:1006BC008A428A6A00000000000000008A86B2ECC0
:1006CC00B0F06AECB0F00000000012006AECB0F080
:1006DC000000000000000000000000008A6A00001A
:1006EC000000000000008A880000000000000000EC
:1006FC008A4265ECB0F000000000100E816EB4EC84
:10070C007CF08A42BEECB0F08A846AECB0F0000057
:10071C008A94BEECB0F0100E816ED5EC7CF08A425F
:10072C0065ECB0F0000000008A46000000000000FC
:10073C0000008A6A00000000000000008A860000A9
:10074C00000000006AECB0F00000000012006AEC3F
:10075C00B0F000000000C2ECB0F08A6A00000000AB
:10076C00000000008A8800000000000000008A429F
:10077C005BECB0F00000100E816EB4EC7CF08A42A1
:10078C00BEECB0F08A846AECB0F000008A94BEEC47
:10079C00B0F0100E816ED5EC7CF08A425BECB0F0C0
:1007AC0000008A4600000000000000008A6A000079
:1007BC000000000000008A86BEECB0F06AECB0F0DD
:1007CC000000000012006AECB0F000000000000015
:1007DC000000000000008A6A000000000000000019
:1007EC008A868A4600000000000000008A4265EC00
:1007FC00B0F00000100E816EB4EC7CF08A42BEECBE
:10080C00B0F08A846AECB0F000008A94BEECB0F0D0
:10081C00100E816ED5EC7CF08A4265ECB0F00000D5
:10082C008A4600000000000000008A428A6A00002C
:10083C000000000000008A860000000000006AEC46
:10084C00B0F00000000012006AECB0F000000000F4
:10085C00BEECB0F08A6A00000000000000008A883C
:10086C0000000000000000008A425BECB0F00000C9
:10087C000000100E816EB4EC7CF08A42BEECB0F03D
:10088C008A846AECB0F000008A94BEECB0F0100ED2
:10089C00816ED5EC7CF08A425BECB0F0000000007D
:1008AC008A4600000000000000008A6A0000000078
:1008BC00000000008A86B2ECB0F06AECB0F00000E8
:1008CC00000012006AECB0F0000000000000000014
:1008DC0000008A6A00000000000000008A88A1EC79
:1008EC00B0F08A4265ECB0F000000000100E816E92
:1008FC00B4EC7CF08A42BEECB0F08A846AECB0F0C6
:10090C0000008A94BEECB0F0100E816ED5EC7CF039
:10091C008A4265ECB0F0000000008A46A1ECB0F011
:10092C008A6A00000000000000008A8600000000B7
:10093C006AECB0F00000000012006AECB0F00000AD
:10094C0000000000000000008A6A000000000000A7
:10095C0000008A868A4600000000000000008A42DF
:10096C0065ECB0F000000000100E816EB4EC7CF071
:10097C008A42BEECB0F08A846AECB0F000008A9433
:10098C00BEECB0F0100E816ED5EC7CF08A4265ECBA
:10099C00B0F0000000008A460000000000000000DB
:1009AC008A428A6A00000000000000008A8600006B
:1009BC0000006AECB0F00000000012006AECB0F02D
:1009CC0000000000A1ECB0F08A4200008A6A00002E
:1009DC000000000000008A880000000000000000F9
:1009EC008A425BECB0F000000000100E816EB4EC9B
:1009FC007CF08A42BEECB0F08A846AECB0F0000065
:100A0C008A94BEECB0F0100E816ED5EC7CF08A426C
:100A1C005BECB0F0000000008A4600000000000013
:100A2C0000008A6A00000000000000008A860000B6
:100A3C008A4600000000000000006AECB0F00000E4
:100A4C00000012006AECB0F0000000008A420000C6
:100A5C0000008A6A00000000000000008A88000084
:100A6C000000000000008A426AECB0F0100E816EAB
:100A7C00B4EC7CF08A42BEECB0F08A846AECB0F044
:100A8C0000008A94BEECB0F0100E816ED5EC7CF0B8
:100A9C008A426AECB0F08A460000000000000000B8
:100AAC008A6A00000000000000008A860000000036
:100ABC008A466AECB0F0000012006AECB0F000005C
:100ACC0000008A42000000008A6A0000000000005A
:100ADC0000008A88A1ECB0F08A4265ECB0F000000E
:100AEC000000100E816EB4EC7CF08A42BEECB0F0CB
:100AFC008A846AECB0F000008A94BEECB0F0100E60
:100B0C00816ED5EC7CF08A4265ECB0F00000000000
:100B1C008A46A1ECB0F08A6A0000000000000000D8
:100B2C008A86000000008A466AECB0F000001200D1
:100B3C006AECB0F000000000000000008A6A0000BF
:100B4C000000000000008A88A1ECB0F08A426AEC38
:100B5C00B0F0100E816EB4EC7CF08A42BEECB0F0BA
:100B6C008A846AECB0F000008A94BEECB0F0100EEF
:100B7C00816ED5EC7CF08A426AECB0F08A46A1EC2E
:100B8C00B0F08A6A00000000000000008A860000B5
:100B9C006AECB0F00000000012006AECB0F000004B
:100BAC000000B2ECB0F08A6A000000000000000007
:100BBC008A868A4600000000000000008A425BEC36
:100BCC00B0F000000000100E816EB4EC7CF08A4294
:100BDC00BEECB0F08A846AECB0F000008A94BEECF3
:100BEC00B0F0100E816ED5EC7CF08A425BECB0F06C
:100BFC00000000008A4600000000000000008A424D
:100C0C008A6A00000000000000008A86A1ECB0F0A7
:100C1C006AECB0F00000000012006AECB0F00000CA
:100C2C000000000000008A6A0000000000000000C4
:100C3C008A868A4600000000000000008A426AECA6
:100C4C00B0F0100E816EB4EC7CF08A42BEECB0F0C9
:100C5C008A846AECB0F000008A94BEECB0F0100EFE
:100C6C00816ED5EC7CF08A426AECB0F08A460000CA
:100C7C000000000000008A428A6A000000000000A8
:100C8C0000008A8600006AECB0F000000000120040
:100C9C006AECB0F000000000B2ECB0F08A6A000020
:100CAC000000000000008A88000000000000000026
:100CBC008A4265ECB0F0100E816EB4EC7CF08A4286
:100CCC00BEECB0F08A846AECB0F000008A94BEEC02
:100CDC00B0F0100E816ED5EC7CF08A4265ECB0F071
:100CEC008A4600000000000000008A6A0000000034
:100CFC00000000008A86A1ECB0F06AECB0F00000B5
:100D0C00000012006AECB0F00000000000000000CF
:100D1C008A6A00000000000000008A8800000000C1
:100D2C00000000008A426AECB0F00000100E816EE8
:100D3C00B4EC7CF08A42BEECB0F08A846AECB0F081
:100D4C0000008A94BEECB0F0100E816ED5EC7CF0F5
:100D5C008A426AECB0F000008A46000000000000F5
:100D6C0000008A6A00000000000000008A86000073
:100D7C006AECB0F00000000012006AECB0F0000069
:100D8C0000008A6A00000000000000008A88A1ECC4
:100D9C00B0F08A426AECB0F000000000100E816ED8
:100DAC00D5EC7CF08A426AECB0F00000000051EC0B
:100DBC00B0F00000100E816EB4EC7CF08A426AEC4C
:100DCC00B0F0000000008A46A1ECB0F08A6A000086
:100DDC000000000000008A866AECB0F000001200EF
:100DEC006AECB0F000000000000000000000000001
:100DFC008A6A00000000000000008A868A46000013
:100E0C00000000008A4265ECB0F000000000100EFB
:100E1C00816ED5EC7CF08A426AECB0F000000000E8
:100E2C0051ECB0F00000100E816EB4EC7CF08A42F4
:100E3C0065ECB0F0000000008A46000000000000E5
:100E4C008A428A6A00000000000000008A860000C6
:100E5C00000000006AECB0F00000000012006AEC28
:100E6C00B0F00000000000000000000000008A6AE2
:100E7C0000000000000000008A868A460000000086
:100E8C00000000008A4265ECB0F00000100E816E8C
:100E9C00D5EC7CF08A426AECB0F00000000051EC1A
:100EAC00B0F00000100E816EB4EC7CF08A4265EC60
:100EBC00B0F000008A4600000000000000008A42EA
:100ECC008A6A00000000000000008A860000000012
:100EDC0000006AECB0F00000000012006AECB0F008
:100EEC0000000000A1ECB0F08A6A000000000000D5
:100EFC0000008A8800000000000000008A4265ECB7
:100F0C00B0F00000100E816ED5EC7CF08A426AECD9
:100F1C00B0F00000000051ECB0F00000100E816E3B
:100F2C00B4EC7CF08A4265ECB0F000008A4600001C
:100F3C000000000000008A6A0000000000000000B1
:100F4C008A8600000000000000006AECB0F000008F
:100F5C00000012006AECB0F00000000000008A6A89
:100F6C0000000000000000008A8800000000000063
:100F7C0000008A426AECB0F000000000100E816E96
:100F8C00D5EC7CF08A426AECB0F00000000051EC29
:100F9C00B0F00000100E816EB4EC7CF08A426AEC6A
:100FAC00B0F0000000008A460000000000000000C5
:100FBC008A6A00000000000000008A866AECB0F02B
:100FCC000000000012006AECB0F000000000A1EC80
:100FDC00B0F08A6A00000000000000008A8800005F
:100FEC000000000000008A4265ECB0F00000100E1A
:100FFC00816ED5EC7CF08A426AECB0F00000000007
:10100C0051ECB0F00000100E816EB4EC7CF08A4212
:10101C0065ECB0F000008A46000000000000000003
:10102C008A6A00000000000000008A8600000000B0
:10103C00000000006AECB0F00000000012006AEC46
:10104C00B0F000000000A1ECB0F08A6A00000000D3
:10105C00000000008A8800000000000000008A42A6
:10106C0065ECB0F00000100E816EB4EC7CF08A429E
:10107C006AECB0F00000000051ECB0F00000100E73
:10108C00816ED5EC7CF08A4265ECB0F000008A46AB
:10109C0000000000000000008A6A00000000000050
:1010AC0000008A8600000000000000006AECB0F02E
:1010BC000000000012006AECB0F00000000000001C
:1010CC008A6A0000000000008A868A460000000040
:1010DC00000000008A426AECB0F000000000100E24
:1010EC00816EB4EC7CF08A426AECB0F00000000037
:1010FC0051ECB0F00000100E816ED5EC7CF08A4201
:10110C006AECB0F0000000008A460000000000000D
:10111C0000008A428A6A0000000000008A866AEC9D
:10112C00B0F00000000012006AECB0F0000000000B
:10113C00A1ECB0F08A6A00000000000000008A8870
:10114C0000000000000000008A4265ECB0F00000D6
:10115C00100E816EB4EC7CF08A426AECB0F00000A8
:10116C00000051ECB0F00000100E816ED5EC7CF05C
:10117C008A4265ECB0F000008A46000000000000D6
:10118C0000008A6A00000000000000008A8600004F
:10119C000000000000006AECB0F00000000012003B
:1011AC006AECB0F0000000008A6A00000000000049
:1011BC0000008A88A1ECB0F08A426AECB0F0000022
:1011CC000000100E816EB4EC7CF08A426AECB0F038
:1011DC000000000051ECB0F00000100E816ED5EC58
:1011EC007CF08A426AECB0F0000000008A46A1EC68
:1011FC00B0F08A6A00000000000000008A866AECE9
:10120C00B0F0000012006AECB0F00000000000002A
:10121C000000000000008A6A0000000000000000CE
:10122C008A868A460000000000008A4265ECB0F015
:10123C0000000000100E816EB4EC7CF08A426AEC67
:10124C00B0F00000000051ECB0F00000100E816E08
:10125C00D5EC7CF08A4265ECB0F0000000008A46C8
:10126C000000000000008A428A6A000000000000B2
:10127C0000008A860000000000006AECB0F000005C
:10128C00000012006AECB0F000000000000000004A
:10129C00000000008A6A00000000000000008A863E
:1012AC008A4600000000000000008A4265ECB0F0A5
:1012BC000000100E816EB4EC7CF08A426AECB0F047
:1012CC000000000051ECB0F00000100E816ED5EC67
:1012DC007CF08A4265ECB0F000008A460000000009
:1012EC00000000008A428A6A000000000000000032
:1012FC008A860000000000006AECB0F000000000DC
:10130C0012006AECB0F0000000008A6A00000000D5
:10131C00000000008A8800000000000000008A42E3
:10132C006FECB0F0100E816EB4EC7CF08A426AEC7B
:10133C00B0F00000000051ECB0F00000100E816E17
:10134C00D5EC7CF08A426FECB0F08A4600000000CD
:10135C00000000008A6A00000000000000008A867D
:10136C006AECB0F0000012006AECB0F00000000073
:10137C0000000000000000008A6A0000000000006D
:10138C0000008A8800000000000000008A4265EC22
:10139C00B0F000000000100E816E7EECB0F000008A
:1013AC008A426AECB0F00000000051ECB0F0000092
:1013BC00100E816E7EECB0F000008A4265ECB0F04D
:1013CC00000000008A4600000000000000008A6A4D
:1013DC0000000000000000008A86000000000000F1
:1013EC006AECB0F00000000012006AECB0F00000F3
:1013FC0000008A6A00000000000000008A880000DB
:10140C000000000000008A426FECB0F0100E816EFC
:10141C007EECB0F000008A426AECB0F000000000F4
:10142C0051ECB0F00000100E816E7EECB0F00000BC
:10143C008A426FECB0F08A46000000000000000009
:10144C008A6A00000000000000008A866AECB0F096
:10145C00000012006AECB0F0000000000000000078
:10146C00000000008A6A00000000000000008A886A
:10147C0000000000000000008A4265ECB0F00000A3
:10148C000000100E816E7EECB0F000008A426AEC17
:10149C00B0F00000000051ECB0F00000100E816EB6
:1014AC007EECB0F000008A4265ECB0F00000000069
:1014BC008A4600000000000000008A6A000000005C
:1014CC00000000008A860000000000006AECB0F00A
:1014DC000000000012006AECB0F0000000008A6A04
:1014EC0000000000000000008A88000000000000DE
:1014FC0000008A426FECB0F0100E816ED5EC7CF0DF
:10150C008A426AECB0F00000000051ECB0F0000030
:10151C00100E816EB4EC7CF08A426FECB0F08A460F
:10152C0000000000000000008A6A000000000000BB
:10153C0000008A866AECB0F0000012006AECB0F091
:10154C000000000000000000000000008A6A00009B
:10155C000000000000008A8800000000000000006D
:10156C008A4265ECB0F000000000100E816ED5ECE4
:10157C007CF08A426AECB0F00000000051ECB0F054
:10158C000000100E816EB4EC7CF08A4265ECB0F079
:10159C00000000008A4600000000000000008A6A7B
:1015AC0000000000000000008A860000000000001F
:1015BC006AECB0F00000000012006AECB0F0000021
:1015CC00000000000000000000008A6A000000001B
:1015DC00000000008A8800000000000000008A4221
:1015EC0065ECB0F000000000100E816ED5EC7CF0C4
:1015FC008A426AECB0F00000000051ECB0F0000040
:10160C00100E816EB4EC7CF08A4265ECB0F00000F8
:10161C0000008A4600000000000000008A6A0000FA
:10162C000000000000008A860000000000006AEC48
:10163C00B0F00000000012006AECB0F000000000F6
:10164C0000000000000000008A6A0000000000009A
:10165C0000008A8800000000000000008A4265EC4F
:10166C00B0F000000000100E816EB4EC7CF08A42E9
:10167C006AECB0F00000000051ECB0F00000100E6D
:10168C00816ED5EC7CF08A4265ECB0F00000000075
:10169C008A4600000000000000008A6A000000007A
:1016AC00000000008A860000000000006AECB0F028
:1016BC000000000012006AECB0F000000000000016
:1016CC000000000000008A6A00000000000000001A
:1016DC008A8800000000000000008A4265ECB0F02F
:1016EC0000000000100E816EB4EC7CF08A426AECB3
:1016FC00B0F00000000051ECB0F00000100E816E54
:10170C00D5EC7CF08A4265ECB0F0000000008A4613
:10171C0000000000000000008A6A000000000000C9
:10172C0000008A860000000000006AECB0F00000A7
:10173C00000012006AECB0F000000000C7ECB0F042
:10174C008A6A00000000000000008A880000000087
:10175C00000000008A425BECB0F0100E816ED5ECFC
:10176C007CF08A42BEECB0F08A326AECB0F0000039
:10177C008A36BEECB0F0100E816EB4EC7CF08A426E
:10178C005BECB0F08A4600000000000000008A6AA2
:10179C0000000000000000008A86C2ECB0F06AEC89
:1017AC00B0F00000000012006AECB0F00000000085
:1017BC00A1ECB0F08A6A00000000000000008A86EC
:1017CC008A4600000000000000008A4265ECB0F080
:1017DC00100E816ED5EC7CF08A42BEECB0F08A32F1
:1017EC006AECB0F000008A36BEECB0F0100E816EE0
:1017FC00B4EC7CF08A4265ECB0F08A460000000044
:10180C00000000008A428A6A00000000000000000C
:10181C008A8600000000000000006AECB0F00000B6
:10182C00000012006AECB0F000000000B2ECB0F066
:10183C008A6A00000000000000008A88A1ECB0F069
:10184C008A425BECB0F000000000100E816ED5EC0B
:10185C007CF08A42BEECB0F08A326AECB0F0000048
:10186C008A36BEECB0F0100E816EB4EC7CF08A427D
:10187C005BECB0F0000000008A46A1ECB0F08A6A84
:10188C0000000000000000008A86A1ECB0F06AECB9
:10189C00B0F00000000012006AECB0F00000000094
:1018AC0045ECB0F08A6A00000000000000008A8855
:1018BC0000000000000000008A4256ECB0F000006E
:1018CC000000100E816ED5EC7CF08A42BEECB0F0BC
:1018DC008A326AECB0F000008A36BEECB0F0100E22
:1018EC00816EB4EC7CF08A4256ECB0F00000000043
:1018FC008A4600000000000000008A6A0000000018
:10190C00000000008A86C7ECB0F06AECB0F0000072
:10191C00000012006AECB0F00000000045ECB0F0E2
:10192C008A6AA1ECB0F08A88000000000000000078
:10193C008A4256ECB0F00000100E816E7EECB0F0D6
:10194C0000008A42BEECB0F08A326AECB0F00000C3
:10195C008A36BEECB0F0100E816E7EECB0F000005A
:10196C008A4256ECB0F000008A46000000000000ED
:10197C0000008A6AA1ECB0F08A86C7ECB0F06AEC81
:10198C00B0F00000000012006AECB0F000000000A3
:10199C00BEECB0F08A6A00000000000000008A88EB
:1019AC00A1ECB0F08A425BECB0F00000100E816E3E
:1019BC007EECB0F000008A42BEECB0F08A326AECE9
:1019CC00B0F000008A36BEECB0F0100E816E7EECEA
:1019DC00B0F000008A425BECB0F000008A46A1EC4B
:1019EC00B0F08A6A00000000000000008A86B2ECA9
:1019FC00B0F06AECB0F00000000012006AECB0F03D
:101A0C0000000000A1ECB0F08A6A000000000000A9
:101A1C0000008A8800000000000000008A4265EC8B
:101A2C00B0F00000100E816ED5EC7CF08A42BEEC5A
:101A3C00B0F08A326AECB0F000008A36BEECB0F03E
:101A4C00100E816EB4EC7CF08A4265ECB0F00000B4
:101A5C008A4600000000000000008A6A00000000B6
:101A6C00000000008A8600000000000000006AEC04
:101A7C00B0F00000000012006AECB0F000000000B2
:101A8C0000008A6A00000000000000008A88000044
:101A9C000000000000008A426AECB0F00000000078
:101AAC00100E816ED5EC7CF08A42BEECB0F08A321E
:101ABC006AECB0F000008A36BEECB0F0100E816E0D
:101ACC00B4EC7CF08A426AECB0F0000000008A466C
:101ADC0000000000000000008A6A00000000000006
:101AEC0000008A866AECB0F00000000012006AEC7C
:101AFC00B0F00000000000008A6A00000000000046
:101B0C0000008A88A1ECB0F08A426AECB0F00000C8
:101B1C00100E816ED5EC7CF08A42BEECB0F08A32AD
:101B2C006AECB0F000008A36BEECB0F0100E816E9C
:101B3C00B4EC7CF08A426AECB0F000008A46A1EC6E
:101B4C00B0F08A6A00000000000000008A866AEC8F
:101B5C00B0F00000000012006AECB0F000000000D1
:101B6C00B2ECB0F08A6A0000000000008A868A4657
:101B7C0000000000000000008A4265ECB0F0100E7E
:101B8C00816ED5EC7CF08A42BEECB0F08A326AEC05
:101B9C00B0F000008A36BEECB0F0100E816EB4ECE2
:101BAC007CF08A4265ECB0F08A4600000000000030
:101BBC0000008A428A6A0000000000008A86A1ECBC
:101BCC00B0F06AECB0F00000000012006AECB0F06B
:101BDC0000000000000000008A6A00000000000005
:101BEC0000008A8800000000000000008A426AECB5
